:100000000C94830B0C9441BE0C9472BE0C94A3BE52
:100010000C94D4BE0C9405BF0C9436BF0C9467BFEF
:100020000C9498BF0C94AE0B0C945AB80C94AE0B75
:100030000C94AE0B0C94AE0B0C94AE0B0C94CB7ECC
:100040000C94AE0B0C94AE0B0C94AE0B0C94AE0B4C
:100050000C94F97E0C94AE0B0C94AE0B0C94C9BFAF
:100060000C94AE0B0C9404C20C94FDC30C94AE0B18
:100070000C94AE0B0C94AE0B0C94AE0B0C94AF80A6
:100080000C941C800C9462810C94AE0B0C94AE0BFF
:100090000C94AE0B0C94AE0B77559355BD55D955BA
:1000A000FF5553567C56A056B856E95619573F5738
:1000B0009B57BF573C5862588858E55817593F59C5
:1000C0006359875992599D599D5FC459FD590F5ADB
:1000D0002C5A495A625A885A9D5F9D5F9D5F9D5F69
:1000E0009D5F9D5FA75AD05AF45A9D5F9D5F9D5FAB
:1000F0009D5F9D5F9D5F9D5F185B305B5E5B9D5F5D
:100100009D5F9D5F9D5F9D5F9D5F9D5F9D5F9D5F0F
:100110009D5F9D5F9D5F9D5F9D5F9D5F9D5F9D5FFF
:100120009D5F9D5F9D5F9D5F9D5F9D5F9D5F9D5FEF
:100130009D5F9D5F9D5F9D5F9D5F9D5F9D5F9D5FDF
:100140009D5F9D5F9D5F9D5F9D5F9D5F9D5F9D5FCF
:100150009D5F9D5F9D5F9D5F9D5F9D5F005C265CD9
:100160004B5C715C975CC05CE05C215D475D665DEB
:10017000895DAF5DD05DF65D175E385E595E7A5E73
:10018000955EAC5ECD5EE05E065F1E5F495F4765D3
:100190006E2E004D6F742E0043616D2E004B662E47
:1001A0000056656C206F66207265717565737465A5
:1001B00064204B463A2000506F73206F66207265B2
:1001C00071756573746564204B463A200054696DFF
:1001D00065206F6620726571756573746564204B68
:1001E000463A200050726F672E202520636F6D7095
:1001F0006C6574653A20004D61782070726F67728B
:10020000616D2074696D652028696E636C2E2073A2
:10021000746172742064656C6179293A20004B46E0
:100220002043757272656E742072756E2074696DEC
:10023000653A200052756E2073746174653A20002F
:10024000436F6E742E2076696420647572617469E0
:100250006F6E3A2000416363656C2076616C69645F
:100260003A200056656C2076616C69643A20004142
:100270006363656C2061742074696D6520783A2031
:100280000056656C2061742074696D6520783A2091
:1002900000506F736974696F6E2061742074696DAA
:1002A0006520783A20004D6F746F722076656C205F
:1002B000757064617465207261746520286D73299E
:1002C0003A20004B6579206672616D6520636F7519
:1002D0006E743A200054616B696E672075702062FD
:1002E00061636B6C6173680053746F7070696E67E3
:1002F000206B662070726F6772616D00506175735C
:10030000696E67206B662070726F6772616D005254
:10031000756E6E696E672F726573756D696E672095
:100320006B662070726F6772616D005365747469DB
:100330006E6720636F6E742E207669642E206D6F59
:1003400076652074696D653A2000456E64696E6754
:10035000204B46207472616E736D697373696F6EA2
:100360000053657474696E672075647061746520EC
:10037000726174653A200053657474696E67207603
:10038000656C6F636974793A200053657474696EA3
:100390006720706F736974696F6E3A2000536574DB
:1003A00074696E672061627363697373613A2000D8
:1003B00053657474696E67206B6579206672616D30
:1003C0006520636F756E743A200053656C656374C5
:1003D000696E6720617869733A200041766F6964BD
:1003E000206F66667365743A2000496E7465727694
:1003F000616C6F6D65746572206D6F64653F203A46
:1004000020004B6565702D616C6976653F203A2050
:100410000054657374206D6F64653F203A2000536B
:10042000686F74732066697265643A2000496E745F
:10043000657276616C2074696D653A20004D697251
:10044000726F722075703F203A2000466F6375739B
:1004500020772F20736875747465723F203A2000EE
:1004600044656C61792074696D653A20004D61784E
:100470002073686F74733A2000466F63757320743D
:10048000696D653A20005472696767657220746906
:100490006D653A200042757379206578706F7369D5
:1004A0006E673F203A2000456E61626C65643F20B4
:1004B0003A200053657474696E6720696E746572C2
:1004C00076616C6F6D65746572206D6F64653A203E
:1004D0000053657474696E67206B6565702D616C7F
:1004E0006976653A200053657474696E6720746597
:1004F0007374206D6F64653A200053657474696E7F
:100500006720696E74657276616C2074696D653AF6
:10051000200053657474696E67207265706561743C
:10052000206379636C65733A200053657474696E57
:100530006720666F63757320772F206578706F73FF
:100540007572653A200053657474696E672064653E
:100550006C61792074696D653A2000536574746923
:100560006E67206D61782073686F74733A20005352
:10057000657474696E6720666F6375732074696D46
:10058000653A200053657474696E672074726967F8
:100590006765722074696D653A20004578706F73E5
:1005A000696E67206E6F77210053657420656E61F8
:1005B000626C65643A200049732073656E64696EED
:1005C000673F3A2000506C6174666F726D207261F3
:1005D00074696F3A200047656172626F78207261BA
:1005E00074696F3A2000556E697420636F64653AD0
:1005F0002000436865636B696E6720322D7074203C
:1006000076656C2076616C69646974793A20004C77
:100610006561642D6F75743A200049732070726FA4
:100620006772616D2076616C69643F203A200053E7
:100630006C6565703A200050726F6772616D20645E
:100640006563656C206C656E6774683A2000507253
:100650006F6772616D20616363656C206C656E67A6
:1006600074683A20004C6561642D696E3A2000542C
:10067000726176656C206C656E6774683A20005311
:10068000746F7020706F733A20005374617274201D
:10069000706F733A2000456173696E673A200041BC
:1006A0006363656C3A200053706565643A200052BC
:1006B000756E6E696E673F203A20004375727265F1
:1006C0006E7420706F733A2000456E6420706F73F3
:1006D0003A20004D61782073706565643A200044CB
:1006E0006972656374696F6E3A20004D6963726F59
:1006F00073746570733A20004261636B6C61736858
:100700003A2000456E61626C65643A20005365745E
:1007100074696E672073746F702D6D6F74696F6E7E
:10072000206D6F64653A200053657474696E6720AC
:10073000706C6174666F726D20726174696F3A20BB
:100740000053657474696E672067656172626F78C3
:1007500020726174696F3A200053657474696E6722
:1007600020756E6974733A200053657474696E67FE
:1007700020656E6420706F736974696F6E20746F8A
:100780003A200053657474696E67206375727265F0
:100790006E7420706F736974696F6E20746F3A2085
:1007A0000053656E64696E6720746F3A200053656C
:1007B0007474696E672073746F7020686572650069
:1007C00053657474696E6720737461727420686510
:1007D0007265004175746F2D73657474696E67205E
:1007E0006D6963726F737465707320005265736511
:1007F00074696E67206C696D69747320616E642022
:1008000073746172742F73746F7020706F696E747B
:10081000730053657474696E67206C656164206F42
:1008200075743A200053656E64696E6720746F209A
:1008300073746F70200053656E64696E6720746F07
:100840002073746172740053657474696E672064F8
:100850006563656C206C656E6774683A200053654B
:100860007474696E6720616363656C206C656E6784
:1008700074683A200053657474696E6720747261FD
:1008800076656C206C656E6774683A2000536574F9
:1008900074696E67206C6561642D696E3A2000533F
:1008A000657474696E6720656173696E67206D6F2A
:1008B00064653A200053657474696E672073746FC1
:1008C000703A200053657474696E672073746172A6
:1008D000743A2000436F6D6D616E646564207374BB
:1008E0006570733A200053657474696E67206163A4
:1008F00063656C65726174696F6E3A20005365744C
:1009000074696E6720636F6E742E20737065656402
:100910003A200053657474696E67206A6F79737446
:1009200069636B2073706565643A200053656E647B
:10093000696E6720746F20656E640053656E64692C
:100940006E6720746F20686F6D65005365747469FD
:100950006E6720656E6420686572653A2000536595
:100960007474696E6720686F6D65206865726500D4
:1009700053657474696E6720646972656374696F26
:100980006E3A20004E6577206D6178207370656542
:10099000643A200053657474696E67206D696372F0
:1009A0006F73746570733A200053657474696E6771
:1009B000206261636B6C6173683A200053746F70DE
:1009C00070696E67206D6F746F720053657474691F
:1009D0006E6720656E61626C653A200053657474C1
:1009E000696E6720736C6565703A200052756E6998
:1009F0006E672073656C6620646961676E6F7374DF
:100A000069630046726565206D656D6F72793A2085
:100A1000004772616666696B206D6F64653A2000FD
:100A200050726F6772616D2072756E20737461749D
:100A300075733A2000436F6E74726F6C6C65722030
:100A4000636F756E743A2000456E6420706F73207A
:100A5000726573746F72653A200053746172742FFB
:100A600073746F7020706F7320726573746F72652A
:100A70003A200043757220706F7320726573746F33
:100A800072653A2000416C6C206D6F746F72207338
:100A90006C656570207374617465733A20005072E0
:100AA0006F6772616D2076616C69643F3A20004126
:100AB0006E79206D6F746F72732072756E6E696ED1
:100AC000673F3A200046505320666C61673A200029
:100AD00049732070726F6772616D20636F6D706C07
:100AE0006574653F3A2000546F74616C2070726FBA
:100AF0006772616D2074696D653A2000546F74618E
:100B00006C2070726F6772616D2074696D653A2038
:100B1000002520436F6D706C6574653A2000576145
:100B2000746368646F67206D6F64653F203A2000CE
:100B300050696E67706F6E67206D6F64653A200054
:100B40004A6F79737469636B206D6F64653A200036
:100B5000506C616E20747970653A20005374617234
:100B6000742064656C61793A2000416C7420696E70
:100B70007075742065646765206465746563746965
:100B80006F6E3A2000537570706C792063757272C5
:100B9000656E743A2000537570706C7920766F6CB6
:100BA000746167653A200043757272656E742072D5
:100BB000756E2074696D653A200052756E207374ED
:100BC000617475733A200053657474696E672061AF
:100BD0007070206D6F64653A200053657474696E9F
:100BE00067204772616666696B206D6F64653A20A5
:100BF0000053657474696E6720636F6E74726F6CF6
:100C00006C657220636F756E743A2000536574745E
:100C1000696E6720656E6420706F732072657374EF
:100C20006F72653A200053657474696E672073743F
:100C30006172742F73746F7020706F73207265739C
:100C4000746F72653A200053657474696E6720632F
:100C5000757220706F7320726573746F72653A20BD
:100C600000526576657273696E6720737461727481
:100C70002F73746F7020706F696E74730053657496
:100C800074696E672046505320666C61673A200095
:100C900053657474696E672073746F7020706F731E
:100CA000206865726520666F7220616C6C206D6FC4
:100CB000746F72732E2E2E0053656E64696E6720FA
:100CC0006D6F746F727320746F207374617274200F
:100CD000706F736974696F6E0053657474696E67C1
:100CE0002070696E672D706F6E67206D6F64652070
:100CF0000053657474696E67206A6F7973746963F1
:100D00006B206D6F6465200053657474696E672095
:100D100070726F6772616D206D6F64653A20005369
:100D2000657474696E672073746172742064656C95
:100D300061793A200053657474696E672077617435
:100D40006368646F67206D6F64653A200053657453
:100D500074696E67206C696D697420737769746358
:100D6000682065646765206D6F64653A200053658F
:100D70006E64696E6720616C6C206D6F746F727346
:100D800020686F6D650053657474696E67206164D7
:100D900064726573733A2000546F67676C696E679D
:100DA000206465627567204C45440053746F707011
:100DB000696E672070726F6772616D005061757344
:100DC000696E672070726F6772616D005374617233
:100DD00074696E67202F20726573756D696E672068
:100DE00070726F6772616D0053657474696E67200D
:100DF0006E657720616464726573732100426C755F
:100E000065746F6F746820004D6F636F4275732057
:100E100000537562616464723A0020636F6D6D61A6
:100E20006E643A00206275665B305D3A2000206295
:100E300075665B315D3A2000206275665B325D3A13
:100E40002000206275665B335D3A20002062756683
:100E50005B345D3A200074696D65200053656E64F3
:100E6000696E67206D6F746F7220007265766572AF
:100E70007365537461727453746F702829004D6FD9
:100E8000742E3133202D204175746F2D737461726F
:100E900074696E6720636F6E74696E756F75732009
:100EA0006D6F7665004A6F79737469636B3A2000E1
:100EB0004D6F746F7273206172652072756E6E690A
:100EC0006E672C2063616E2774206175746F2D73BB
:100ED0006574206D6963726F737465707300526519
:100EE00071756573746564204D6963726F737465A1
:100EF00070733A2000547279696E6720746F2061B4
:100F000075746F2D736574206D6963726F7374658A
:100F100070730045786365737369766520737065D7
:100F200065642072657175657374656400546F70D3
:100F3000207370656564207265717565737465648E
:100F40003A20004D6963726F73746570733A2000C4
:100F50004F7574206F66206C6F6F7020616E642017
:100F60006D6F76696E67206F6E21004D6963726FD9
:100F700073746570733A200047657474696E6720F6
:100F8000766964206D6F76652074696D653A20001E
:100F900047657474696E6720544C206D6F766520C8
:100FA00074696D653A2000536875747465722064C5
:100FB0006F6E652C20726561647920666F72206D9A
:100FC0006F76650054696D65206174206578706F77
:100FD000737572653A200054696D652061742066EE
:100FE0006F6375733A20006B665F43616D65726174
:100FF000436865636B2829202D204261696C696E06
:10100000672066726F6D2063616D65726120637920
:10101000636C6520617420706F696E742032006BA0
:10102000665F43616D657261436865636B28292063
:101030002D20536B697070696E672073686F742C14
:101040002077616974696E6720666F7220657874B5
:1010500065726E616C2074726967676572005365B2
:101060006E64696E6720746F200041626F75742032
:10107000746F2073656E6420746F206C6F6361748D
:10108000696F6E20233A200053656E64696E672095
:101090006D6F746F727320746F206E6577206C6F44
:1010A000636174696F6E73005374617274696E6703
:1010B000206E6577206B6620626F756E63652070A9
:1010C000726F6772616D0053746F7070696E672024
:1010D0006B662070726F6772616D00537461727419
:1010E000696E67206B65657020616C69766520703C
:1010F00068617365005061757365206C656E677417
:10110000683A200053544F5050494E47204B4620D8
:1011100050524F4752414D0053746F7070696E6763
:10112000206D6F746F72200050415553494E472017
:101130004B462050524F4752414D00204B462070A5
:10114000726F6772616D005374617274696E6720AB
:101150006E6577207479706520002A2A2A205665EA
:101160006C6F636974696573202A2A2A002A2A2A07
:1011700020506F736974696F6E73202A2A2A002ABF
:101180002A2A20416273636973736173202A2A2AB1
:1011900000207E7E7E7E7E7E007E7E7E7E7E7E2027
:1011A000415849532000436F6E742E207669646560
:1011B0006F2074696D653A200050726F6772616DBF
:1011C000206D6F64653A200050657263656E74200F
:1011D000636F6D706C6574653A200043757272655B
:1011E0006E742072756E2074696D653A20005275B8
:1011F0006E207374617475733A20004D6178206DB0
:101200006F76652074696D653A20004D61782063C2
:10121000616D6572612074696D653A20007E7E7E25
:101220007E7E7E2047656E6572616C2050726F67AE
:1012300072616D20506172616D73207E7E7E7E7E54
:101240007E004175746F2070617573696E6721212E
:1012500021006379636C6553686F744F4B282920B4
:101260002D20616C74466F72636553686F74206ED5
:101270006F74206465746563746564006379636C7E
:101280006553686F744F4B2829202D20616C74467C
:101290006F72636553686F74206465746563746509
:1012A00064202A2A2A2A2A2A2A2A2A2A2A2A00635F
:1012B00079636C6553686F744F4B2829202D204546
:1012C00078742E20696E74657276616C206D6F641F
:1012D0006520616374697665006379636C65536842
:1012E0006F744F4B2829202D20456E74657220663F
:1012F000756E6374696F6E006379636C6543616DCD
:101300006572612829202D205374617274696E679B
:10131000206578706F73757265206379636C650002
:101320006379636C6543616D6572612829202D20A6
:1013300043616D65726120627573793A200063794B
:10134000636C6543616D6572612829202D204261BF
:10135000696C696E672066726F6D2063616D65727E
:1013600061206379636C6520617420706F696E74AD
:101370002033004D6F746F7220006379636C654396
:10138000616D6572612829202D2053686F74733A4E
:1013900020006379636C6543616D65726128292063
:1013A0002D204261696C696E672066726F6D2063E3
:1013B000616D657261206379636C65206174207072
:1013C0006F696E742032006379636C6543616D658B
:1013D00072612829202D20536B697070696E672017
:1013E00073686F742C2077616974696E6720666F0B
:1013F000722065787465726E616C207472696767BB
:101400006572006379636C6543616D65726128295B
:10141000202D204261696C696E672066726F6D20B5
:1014200063616D657261206379636C65206174200E
:10143000706F696E742031006D73206F66206C656B
:1014400061642D6F75742072656D61696E696E6778
:10145000006379636C6543616D6572612829202D95
:101460002054686572652061726520006379636C41
:101470006543616D6572612829202D20416C6C20C7
:101480006D6F7420646F6E65206D6F76696E670096
:101490006379636C6543616D6572612829202D2035
:1014A00050617573696E67006379636C6543616D44
:1014B0006572612829202D20537461727400636164
:1014C0006D43616C6C4261636B2829202D2053743D
:1014D0006F700063616D43616C6C4261636B2829BE
:1014E000202D20537461727400206C656164496E14
:1014F0003A20002073686F74733A2000205479708A
:10150000653A200020656E61626C653A20002072A9
:10151000756E6E696E673A200020656E64506F7359
:101520003A20002073746F70506F733A200020735C
:1015300074617274506F733A2000206261636B6C47
:101540006173683A200020636F6E74696E696F750D
:10155000732053706565643A200043757272656E3E
:101560007420537465707320001201100102000092
:1015700008EB03442001000102030109023E0002BE
:101580000100C0320904000001020201000524002C
:101590001001042402060524060001070582030841
:1015A00000FF09040100020A000000070504021000
:1015B000000507058302100005040309042E0344F7
:1015C0000079006E0061006D00690063002000502A
:1015D0000065007200630065007000740069006FB0
:1015E000006E0020004C004C00430000003C03440F
:1015F0000079006E0061006D0069006300200050FA
:101600000065007200630065007000740069006F7F
:10161000006E00200043004400430020005300659A
:10162000007200690061006C0000000E03300030A1
:101630000034003500370033000000000021002492
:101640000027002A002D003000000022002500287D
:10165000002B002E0031000000200023002600296E
:10166000002C002F00010101010101010102020211
:10167000020202020203030303030303030404043C
:10168000040404040405050505050505050606060C
:101690000606060606010204081020408001020426
:1016A000081020408001020408102040800102043C
:1016B000081020408001020408102040800102042C
:1016C0000810204080000000000000000000000022
:1016D0000007030401000000000B0A0900020800D3
:1016E00000000000000000000000000000000000FA
:1016F0000000000000000102030405060700C418F2
:10170000B8C3E0C7BD1811241FBECFEFD0E2DEBFC3
:10171000CDBF14E0A0E0B1E0E6E6F5EA01E00BBFE2
:1017200002C007900D92A839B107D9F71BBE13E18B
:10173000A8E9B4E001C01D92A63AB107E1F716E1AD
:10174000C4E0D7E104C02297FE010E946BD2CE3FD5
:10175000D107C9F70E94D3C40C94A6D20C94000000
:10176000CF93DF93BC018230910510F462E070E00A
:10177000A0919E13B0919F13ED01E0E0F0E040E0F6
:1017800050E021C0888199818617970769F48A8182
:101790009B81309719F09383828304C090939F13A9
:1017A00080939E13FE0134C06817790738F4411501
:1017B000510519F08417950708F4AC01FE018A81E0
:1017C0009B819C01E9012097E9F641155105A9F19A
:1017D000CA01861B970B049708F4BA01E0E0F0E019
:1017E0002AC08D919C91119784179507F9F464177D
:1017F000750781F412968D919C911397309719F08B
:101800009383828304C090939F1380939E13FD0162
:1018100032964CC0CA01861B970BFD01E80FF91FD9
:101820006193719302978D939C9340C0FD018281D7
:1018300093819C01D9011097A1F680919C139091FE
:101840009D13892B41F48091A4039091A50390935B
:101850009D1380939C134091A6035091A7034115BB
:10186000510541F44DB75EB78091A2039091A30357
:10187000481B590B20919C1330919D13CA01821B68
:10188000930B8617970780F0AB014E5F5F4F84176D
:10189000950750F0420F531F50939D1340939C1394
:1018A000F9016193719302C0E0E0F0E0CF01DF91B4
:1018B000CF910895CF93DF93009709F450C0EC01C6
:1018C00022971B821A82A0919E13B0919F131097AA
:1018D00009F140E050E0AC17BD0708F1BB83AA83D3
:1018E000FE0121913191E20FF31FAE17BF0779F48A
:1018F0008D919C911197280F391F2E5F3F4F39838F
:10190000288312968D919C9113979B838A8341150E
:10191000510571F4D0939F13C0939E1320C012966B
:101920008D919C911397AD01009711F0DC01D3CFFD
:10193000FA01D383C28321913191E20FF31FCE17B5
:10194000DF0769F488819981280F391F2E5F3F4F87
:10195000FA01318320838A819B8193838283DF9183
:10196000CF910895A0E0B0E0E8EBFCE00C9471D2D8
:101970006C01009729F4CB010E94B00B6C01C1C02F
:101980008EEF882E8FEF982E8C0C9D1C8601060FF3
:10199000171F0815190508F4B2C0F401A081B18120
:1019A000A617B707B8F0A530B10508F4AAC0CD0155
:1019B00004978617970708F4A4C01297A61BB70BC5
:1019C000F801A193B193D4016D937C93CF010E9450
:1019D0005A0C97C07B01EA1AFB0AEEEFFFEFEE0EFE
:1019E000FF1E36016A0E7B1EC0919E13D0919F137D
:1019F00044245524AA24BB244AC0C615D705E1F5C2
:101A0000488159814E155F05B8F1CA0104978E15BA
:101A10009F05B0F41296A40FB51FF401B183A08303
:101A20002A813B814114510431F0D20113963C9339
:101A30002E93129766C030939F1320939E1361C01C
:101A40008A819B81F80193838283425050404E19D2
:101A50005F09518340834114510431F0D201139640
:101A60001C930E93129704C010939F1300939E1320
:101A7000F4017183608345C088819981A816B906F5
:101A800008F45C012E018A819B819C01E901209769
:101A900009F0B3CF80919C1390919D138615970503
:101AA000E9F4A616B706D0F42091A6033091A70357
:101AB0002115310541F42DB73EB78091A2039091D5
:101AC000A303281B390B02171307C8F410939D13A7
:101AD00000939C13D4016D937C9313C0CB010E949F
:101AE000B00BEC01009759F0F40140815181B6012F
:101AF0000E948E0DC6010E945A0C6E0102C0CC24B9
:101B0000DD24C601CDB7DEB7E0E10C948DD2FB0138
:101B1000DC0105900D920020E1F70895FB01DC0146
:101B200002C001900D9241505040D8F70895FB013A
:101B3000DC0101900D920020E1F70895FB019F0167
:101B4000E8944230C4F04532B4F44A3029F497FBAB
:101B50001EF4909581959F4F642F77270E9405D2A0
:101B6000805D8A330CF0895D8193CB010097A1F7EA
:101B700016F45DE251931082C9010C940110FA0130
:101B8000CF93FF93EF932230CCF02532BCF4C22FD9
:101B90002C2F332744275527FF93EF930E942CD2F5
:101BA000EF91FF91605D6A330CF0695D6193B9015B
:101BB000CA01605070408040904051F710828F9170
:101BC0009F91CF910C940110FB019F01423074F062
:101BD000453264F4642F77270E9405D2805D8A33F2
:101BE0000CF0895D8193CB010097A1F71082C901A8
:101BF0000C940110A0E0B0E0E0E0FEE00C947FD295
:101C00009E01275F3F4F8D819E816F817885A9015D
:101C10000E940E0E2096E2E00C949BD2ABE0B0E066
:101C2000E4E1FEE00C946FD23C012B015A01FC016F
:101C300017821682838181FD03C06FEF7FEFC6C1DB
:101C40009AE0892E1E010894211C311CF301238186
:101C5000F20123FD859123FF81912F01882309F44F
:101C6000B2C1853239F423FD859123FF81912F0183
:101C7000853229F490E0B3010E941110E7CF982F2C
:101C8000FF24EE249924FFE1FF15D0F09B3269F088
:101C90009C3228F4903259F0933291F40EC09D3268
:101CA00049F0903369F441E024C052E0F52A84E021
:101CB000F82A28C098E0F92A25C0E0E1FE2A22C0CF
:101CC000F7FC29C0892F80538A3070F4F6FE05C0D6
:101CD000989C902C1124980E15C0E89CE02C11249F
:101CE000E80EF0E2FF2A0EC09E3229F4F6FC6BC12A
:101CF00040E4F42A07C09C3619F450E8F52A02C0E3
:101D0000983649F4F20123FD959123FF91912F011B
:101D1000992309F0B8CF892F8554833018F0805269
:101D2000833038F444E050E0A40EB51E5FE35983DD
:101D30000FC0933631F0933779F0933509F056C0E0
:101D400020C0F5018081898342E050E0A40EB51ED9
:101D5000610101E010E012C0F501C080D180F6FC05
:101D600003C06FEF7FEF02C0692D70E042E050E0EA
:101D7000A40EB51EC6010E94F60F8C015FE7F52286
:101D800014C0F501C080D180F6FC03C06FEF7FEF77
:101D900002C0692D70E042E050E0A40EB51EC601FD
:101DA0000E94EB0F8C0150E8F52AF3FE07C01AC021
:101DB00080E290E0B3010E941110EA948E2D90E031
:101DC00008171907A8F30EC0F601F7FC8591F7FE76
:101DD00081916F0190E0B3010E941110E110EA942B
:101DE000015010400115110579F7EAC0943611F041
:101DF000993669F5F7FE08C0F501208131814281ED
:101E0000538184E090E00AC0F501808191819C01BA
:101E1000442737FD4095542F82E090E0A80EB91E6C
:101E20009FE6F92257FF09C05095409530952195BE
:101E30003F4F4F4F5F4FE0E8FE2ACA01B901A101B1
:101E40002AE030E00E943D10D82ED21840C09537CD
:101E500029F41F2D1F7E2AE030E01DC01F2D197FA1
:101E60009F3661F0903720F4983509F0ACC00FC070
:101E7000903739F0983709F0A6C004C028E030E068
:101E80000AC0106114FD146020E130E004C014FDAC
:101E9000166020E132E017FF08C0F5016081718112
:101EA0008281938144E050E008C0F50180819181F6
:101EB000BC0180E090E042E050E0A40EB51EA1011C
:101EC0000E943D10D82ED2188FE7F82EF122F6FE90
:101ED0000BC05EEFF522D91438F4F4FE07C0F2FC13
:101EE00005C08FEEF82202C01D2D01C0192DF4FE91
:101EF0000DC0FE01ED0DF11D8081803319F499EEC6
:101F0000F92208C01F5FF2FE05C003C08F2D86783E
:101F100009F01F5F0F2DF3FC14C0F0FE0FC01E155B
:101F200010F09D2C0BC09D2C9E0C911A1E2D06C0EE
:101F300080E290E0B3010E9411101F5F1E15C0F3F4
:101F400004C01E1510F4E11A01C0EE2404FF0FC0F6
:101F500080E390E0B3010E94111002FF1DC001FD5B
:101F600003C088E790E00EC088E590E00BC0802FAA
:101F7000867891F001FF02C08BE201C080E2F7FC9D
:101F80008DE290E0B3010E94111006C080E390E062
:101F9000B3010E9411109A94D914C0F3DA94F1019C
:101FA000ED0DF11D808190E0B3010E941110DD2044
:101FB000A9F706C080E290E0B3010E941110EA94F4
:101FC000EE20C1F743CEF30166817781CB012B96DA
:101FD000E2E10C948BD2FC0105906150704001103D
:101FE000D8F7809590958E0F9F1F0895FC01615042
:101FF000704001900110D8F7809590958E0F9F1F2B
:102000000895DC01FC01672F71917723E1F7329786
:1020100004C07C916D9370836291AE17BF07C8F3C3
:1020200008950F931F93CF93DF938C01EB018B8166
:1020300081FF1BC082FF0DC02E813F818C819D815D
:102040002817390764F4E881F9810193F983E8835B
:1020500006C0E885F985802F0995892B31F48E819A
:102060009F8101969F838E8302C00FEF1FEFC801EF
:10207000DF91CF911F910F910895FA01AA2728307F
:1020800051F1203181F1E8946F936E7F6E5F7F4F45
:102090008F4F9F4FAF4FB1E03ED0B4E03CD0670FC1
:1020A000781F891F9A1FA11D680F791F8A1F911D14
:1020B000A11D6A0F711D811D911DA11D20D009F464
:1020C00068943F912AE0269F11243019305D3193A6
:1020D000DEF6CF010895462F4770405D4193B3E08F
:1020E0000FD0C9F7F6CF462F4F70405D4A3318F036
:1020F000495D31FD4052419302D0A9F7EACFB4E0E7
:10210000A6959795879577956795BA95C9F700979E
:102110006105710508959B01AC010A2E069457953F
:10212000479537952795BA95C9F7620F731F841F96
:10213000951FA01D0895FC01108281E08183128209
:102140000895FC01748363830E949B100895FC0131
:1021500080810895FC016183862F0895FC016283CC
:10216000862F08951F93CF93DF93EC01162F68837A
:102170008981882399F089E793E160E071E00E940A
:10218000B8C689E793E1612F42E050E00E942DC676
:1021900089E793E167E171E00E9468C78A8188233B
:1021A00099F08B819C8160E071E00E94B8C68B81C0
:1021B0009C81612F42E050E00E942DC68B819C8162
:1021C00067E171E00E9468C7DF91CF911F91089588
:1021D0008091A20408958091DA041092DA0408959F
:1021E0008091060410920604089580939B0488232E
:1021F00011F010929C04089580919B04089580939F
:102200009C04882311F010929B04089580919C04F3
:1022100008958093DB048093DC0408958091DB04AF
:10222000811181E0089581E08093C70D08950F9397
:102230001F93CF93DF93EC018EE46132780718F09F
:1022400060E27EE405C06436710510F464E670E077
:1022500080E090E00E9468D02FEF30E0C29F8001C4
:10226000C39F100DD29F100D11240253124F0F5017
:102270001F4FF80161937193819391938F0120E037
:1022800030E040E05FE30E941ED1F801608371837B
:1022900082839383DF91CF911F910F9108952F92A5
:1022A0003F924F925F926F927F928F929F92AF92E6
:1022B000BF92CF92DF92EF92FF920F931F93DF9323
:1022C000CF9300D000D0CDB7DEB73C018FEF90E0C8
:1022D000689EB001699E700D789E700D1124FB01FF
:1022E000E253F24FDF01A751BF4FE351FF4F20816F
:1022F0003181428153818D919D910D90BC91A02D92
:10230000281739074A075B0709F43FC1FB01E0536F
:10231000F24F80E090E020E030E040E050E02083A9
:1023200031834283538320AF31AF42AF53AF148E1A
:10233000158E168E178E019634968730910579F793
:102340008FEF90E0689E8001699E100D789E100DC1
:1023500011240253124F05501F4FD8016D917D91EA
:102360008D919C9120E030E040EA51E40E941ED122
:102370002FE632E143E852E40E94CFCF6B017C01AB
:1023800006501040D8018D919D910D90BC91A02DCB
:1023900089839A83AB83BC83F801B290A290929018
:1023A0008290C701B601A50194010E941AD11816A6
:1023B00014F4750164018FEF90E0689EF001699E4E
:1023C000F00D789EF00D1124EA54F14F808188239E
:1023D00021F4F7FAF094F7F8F094C701B6012981D7
:1023E0003A814B815C810E94CFCF1B012C01E89484
:1023F00057F88FEF90E0689EF001699EF00D789E8F
:10240000F00D1124E253F24F22823382448255822E
:10241000E751FF4F80819181A281B381E95EF04055
:10242000868F978FA0A3B1A3C2AED3AEE4AEF5AEB4
:10243000C701B60120E030E040E050E00E941AD130
:1024400018164CF489819A81AB81BC81B05889837C
:102450009A83AB83BC838FEF90E0689E8001699E76
:10246000100D789E100D11240253124F86E5682E30
:10247000712C600E711E89819A81AB81BC81F30140
:1024800080839183A283B3830F2EF0E08F2EF0E040
:102490009F2EF0E0AF2EF0E0BF2EF02DD801169663
:1024A0008D929D92AD92BC9219975E966D917D91A1
:1024B0008D919C9191970E946AD06B017C01C20121
:1024C000B101F80122AD33AD44AD55AD0E941ED12E
:1024D0009B01AC01C701B6010E9467CF6B017C0173
:1024E00069817A818B819C8120E030E040E05FE36C
:1024F0000E941ED1A20191010E941ED1A201910150
:102500000E941ED19B01AC01C701B6010E9467CF9A
:102510000E9437D06B017C01D80192966D937D9318
:102520008D939C939597025C1F4FF8018082918256
:10253000A282B382045E1F4FD8018D929D92AD920C
:10254000BC921397F301608171818281938120E0B5
:1025500030E040E05FE30E941ED1D3016D937D9394
:102560008D939C9313970D561F4FF801C082D18213
:10257000E282F38209501040D8018D929D92AD9273
:10258000BC921397F801129212920F900F900F9035
:102590000F90CF91DF911F910F91FF90EF90DF90FF
:1025A000CF90BF90AF909F908F907F906F905F90F3
:1025B0004F903F902F90089580E090E00E944F113F
:1025C00081E090E00E944F1182E090E00E944F1164
:1025D000089520E0039708F421E0822F08952F92B8
:1025E0003F924F925F926F927F928F929F92AF92A3
:1025F000BF92CF92DF92EF92FF920F931F93DF93E0
:10260000CF93CDB7DEB760970FB6F894DEBF0FBE9D
:10261000CDBF8C0149875A876B877C873E872D8782
:102620008FEF90E0089FF001099FF00D189FF00DCB
:102630001124EA54F14F8081882359F40F2EF0E0E1
:10264000CF2EF0E0DF2EF0EAEF2EF1ECFF2EF02D92
:102650000AC00F2EF0E0CF2EF0E0DF2EF0EAEF2ED2
:10266000F1E4FF2EF02D8FEF90E0089F9001099F7D
:10267000300D189F300D11242253324F25503F4FFB
:10268000D9012D903D904D905C9022513040D90160
:102690008D919D910D90BC91A02D8D839E83AF83D4
:1026A000B88729853A854B855C8582179307A407EF
:1026B000B5072CF04FEF5FEF588B4F8704C081E0D8
:1026C00090E0988B8F87C201B10120E030E040E0BC
:1026D00050E00E94CBCF882309F44BC18FEF90E0EC
:1026E000089FF001099FF00D189FF00D1124EA5486
:1026F000F14F808190E0AF85B889FC01AE9FC001A9
:10270000AF9F900DBE9F900D112497FF32C1C8015D
:102710000E944F113CC18FEF90E0089FF001099F8C
:10272000F00D189FF00D1124E253F24FEF50FF4FC0
:10273000619071908190919080819181A281B3810B
:1027400089839A83AB83BC83C701B601A20191013F
:102750000E941ED12FE632E143E852E40E94CFCF1F
:102760007B018C01E89417F9C801B701A40193011A
:102770000E94CBCF87FD15C00F2EF0E06F2EF0E04A
:102780007F2EF0E08F2EF0E09F2EF02D0F2EF0E048
:102790002F2EF0E03F2EF0E04F2EFFE35F2EF02DC6
:1027A00035C0C401B301A80197010E9466CF2981F9
:1027B0003A814B815C810E94CFCF3B014C0120E0EC
:1027C00030E040E05FE30E94CBCF87FD15C00F2EC5
:1027D000F0E06F2EF0E07F2EF0E08F2EFFE39F2ED3
:1027E000F02D0F2EF0E02F2EF0E03F2EF0E04F2ED8
:1027F000F0E05F2EF02D0AC060E070E080E09FE323
:10280000A40193010E9466CF1B012C0169817A818A
:102810008B819C81A40193010E941ED19B01AC017C
:10282000C801B7010E9467CF5B016C01C801B70105
:10283000A40193010E941ED17B018C0169817A81E0
:102840008B819C8120E030E040E05FE30E941ED15C
:10285000A40193010E941ED1A40193010E941ED1E4
:102860009B01AC01C801B7010E9467CF0E9437D01D
:102870000E946AD07B018C01C201B101A6019501C1
:102880000E941ED19B01AC01C801B7010E9467CF15
:102890000E9437D00E946AD07B018C01C601B5012D
:1028A000A60195010E941ED120E030E040E05FE3E8
:1028B0000E941ED129813A814B815C810E94CFCF39
:1028C0009B01AC01C801B7010E9467CF0E9437D0BD
:1028D000EF85F8899F01442737FD4095542F0E94CA
:1028E000E6D12D813E814F815885620F731F841F71
:1028F000951F4F8558894130510551F429853A85F6
:102900004B855C8526173707480759078CF40EC09E
:102910004F8558894F5F5F4F59F429853A854B851C
:102920005C85621773078407950714F4CA01B9011F
:10293000AD85BE856D937D938D939C93139781E0B8
:1029400060960FB6F894DEBF0FBECDBFCF91DF917A
:102950001F910F91FF90EF90DF90CF90BF90AF90BD
:102960009F908F907F906F905F904F903F902F90AF
:10297000089529853A854B855C858D819E81AF813F
:10298000B885281739074A075B0709F0C4CE80E0ED
:10299000D7CF8091A50408958091C104882339F48C
:1029A00080918205882319F420E030E00AC020914C
:1029B000CC043091CD048091A3049091A404280FFD
:1029C000391FC90108951092A4041092A304109213
:1029D000CD041092CC0408958091D11091E0892704
:1029E0008093D11008951092D11008958091D11044
:1029F00008952091C4043091C5044091C6045091BB
:102A0000C7048091B9049091BA04A091BB04B0911D
:102A1000BC04280F391F4A1F5B1FB901CA01089562
:102A200080918205882319F420E030E00BC080916A
:102A30008305882319F421E030E004C0813011F4CB
:102A400022E030E0C90108952091C8043091C90402
:102A50004091CA045091CB0480916E0590916F050E
:102A6000A0917005B0917105280F391F4A1F5B1F97
:102A7000B901CA010895813039F0813018F08230EF
:102A800051F406C083E001C082E08093C003089542
:102A900081E08093C0030895E091E010F091E1108F
:102AA000309709F0099508958091E10408958230E6
:102AB00010F48093C30408958091C3040895809115
:102AC000A60408951F938091C104882311F011E09A
:102AD00007C080918205882311F015E001C010E045
:102AE0008091D704882311F0136004C0809183057E
:102AF000811116608091D604811118600E945F15C3
:102B0000811110610E945C1581111062812F1F914B
:102B10000895FC0110820895FC0180810895FC0154
:102B200080E880934C1180934D1180934E118093D7
:102B30004F111286138608951F93FC01808188230C
:102B400009F455C070E0615070402581368147819D
:102B50005085DA01C901062E04C0B695A795979550
:102B600087950A94D2F7182F117081819281A381E1
:102B7000B481062E04C0B695A795979587950A94BB
:102B8000D2F780FF17C081E090E0A0E0B0E004C081
:102B9000880F991FAA1FBB1F6A95D2F7822B932B10
:102BA000A42BB52B85839683A783B0871130E9F4D6
:102BB00081E01EC081E090E0A0E0B0E004C0880F9A
:102BC000991FAA1FBB1F6A95D2F780959095A09573
:102BD000B09582239323A423B52385839683A7836B
:102BE000B087113021F482E003C083E001C080E0AF
:102BF0001F910895FC018081882341F1862F90E088
:102C000001972581368147815085082E04C056954D
:102C10004795379527950A94D2F7922F9170218185
:102C200032814381548104C0569547953795279545
:102C30008A95D2F720FF06C0913011F481E0089503
:102C400083E00895913011F482E0089580E00895C2
:102C5000FC01E45BFF4F80810895FC01E25BFF4FC4
:102C600080810895FC01E15BFF4F80810895089504
:102C70001092001108950895AF92BF92CF92DF9203
:102C8000EF92FF920F931F935A016B01CB01BA0190
:102C900020E030E040E053E40E9466CF7B018C01ED
:102CA00020E030E040E050E00E941AD118165CF4B9
:102CB000C801B70120E030E040E251E40E94CBCFF0
:102CC0001816ACF00AC0C801B70120E030E040E2BD
:102CD00051EC0E941AD1882354F00F2EF0E0AF2E51
:102CE000F0E0BF2EF0E0CF2EF3E4DF2EF02DB501A3
:102CF000C6011F910F91FF90EF90DF90CF90BF9092
:102D0000AF900895FC0113A20895FC01E60FF11D98
:102D100043870895CF93DF93EC01222319F40E9497
:102D2000821612C081E08BA32EA31FA25FA74EA71D
:102D30005BA74AA779A768A71DA61CA60E9411C079
:102D400068AB79AB8AAB9BABDF91CF91089566E915
:102D500070E044E650E021E00E948A1608957F92D8
:102D60008F929F92AF92BF92CF92DF92EF92FF929B
:102D70000F931F93CF93DF934C01742EE90180E0F2
:102D800091E10E949C15833019F5BE0180E090E02E
:102D90000E9468D07B018C012AE939E949E15EE3B0
:102DA0000E941ED10E943CD05B016C01C801B7019A
:102DB0002AE939E949E55FE30E941ED10E943CD02F
:102DC0009B01AC01C401B501A901272D0E948A16FF
:102DD000DF91CF911F910F91FF90EF90DF90CF90F7
:102DE000BF90AF909F908F907F9008956F927F9249
:102DF0008F929F92AF92BF92CF92DF92EF92FF920B
:102E00000F931F93CF93DF93EC01162FA42E49014C
:102E1000702E6C2C80E091E1642F0E949C15982FFD
:102E200080919A11882329F080919911A81609F0B0
:102E30008DC0933009F063C01123A9F5A0929911B8
:102E400081E080939A110E9411C060939511709354
:102E50009611809397119093981110929411B70145
:102E600080E090E00E9468D07B018C012AE939E97A
:102E700049E15EE30E941ED10E943CD05B016C01DF
:102E8000C801B7012AE939E949E55FE30E941ED18B
:102E90000E943CD09B01AC01CE01B501A9012FEFEE
:102EA0000E948A1645C0133019F0113009F040C055
:102EB000B70180E090E00E9468D07B018C012AE994
:102EC00039E949E15EE30E941ED10E943CD05B01DA
:102ED0006C01C801B7012AE939E949E55FE30E94BD
:102EE0001ED10E943CD09B01AC01CE01B501A901CD
:102EF000272D0E948A1681E080939B1127C0923073
:102F0000B9F480919B11813019F410929B111EC06D
:102F1000882371F480919411882319F4CE010E94C2
:102F2000821610929A118FA1F401808381E00FC064
:102F30008FA1861558F080919411882339F4CE0121
:102F40000E94821681E0809394116FA280E0DF914D
:102F5000CF911F910F91FF90EF90DF90CF90BF9096
:102F6000AF909F908F907F906F9008958F929F92D7
:102F7000AF92BF92CF92DF92EF92FF920F931F9387
:102F8000CF93DF93EC018130910509F0C4C06F5FEE
:102F90007F4F09F0E5C082EE94E00E949E898EE0AA
:102FA00095E00E949E898AE395E00E949E89109296
:102FB00087051092860588EE93E0A0E0B0E080934C
:102FC000880590938905A0938A05B0938B058AE5BF
:102FD00094E090938505809384054091B4035091CB
:102FE000B50380E995E064E875E026E630E00CE39F
:102FF00014E00E9454B54091B4035091B50382EFA0
:1030000095E069E773E126E630E00E9454B540910F
:10301000B4035091B50384E596E067E573E126E6D5
:1030200030E00E9454B586EB96E00E944A9387EB0D
:1030300096E00E946BB0A1B200D0EDB7FEB712824D
:1030400011828CEC96E06DE270E040E150E020E20D
:1030500030E001E110E0E2E1EE2EF12CB3E1CB2E05
:10306000D12CBB24A5E08A2E912C0E9489ACA1B260
:10307000EDB7FEB7D283C18386EC98E06EE270E0D4
:1030800045E150E024E130E00DE110E0FEE1EF2EFB
:10309000F12CEFE1CE2ED12CB6E08B2E912C0E949C
:1030A00089ACA1B282E090E0EDB7FEB79283818354
:1030B00080EC9AE06FE270E042E250E021E230E022
:1030C0000FE010E0ABE2EA2EF12CFCE2CF2ED12C87
:1030D000E7E08E2E912C0E9489AC0F900F908AEB26
:1030E0009CE067E00E94CDAE8DED9CE064E576E06B
:1030F0000E940C7E83EE9CE06DED7CE00E94A110AE
:103100000E9411C06093DC107093DD108093DE107C
:103110009093DF1025C0009719F56F5F7F4F01F581
:1031200080EC9AE00E94A79386EC98E00E94A79317
:103130008CEC96E00E94A7938AE594E09093850535
:10314000809384050E94EC818AE395E00E94928935
:103150008EE095E00E94928982EE94E00E9492892E
:10316000DF91CF911F910F91FF90EF90DF90CF9063
:10317000BF90AF909F908F90089580E090E06FEFA8
:103180007FEF0E94B617089581E090E06FEF7FEF28
:103190000E94B61708958CEC96E00E9492968823C0
:1031A00089F086EC98E00E949296882359F080EC92
:1031B0009AE00E94929690E0882309F491E081E0E1
:1031C000982701C090E0892F089541E00E9481B5C1
:1031D000089542E00E9481B5089541E00E9481B5C2
:1031E000089541E00E9481B5089544E00E9481B5B0
:1031F000089544E00E9481B5089542E00E9481B59F
:10320000089541E00E94D8B508950F931F93CF937E
:10321000DF938FE0689F80011124065A1F4FC4E896
:10322000D1E107C0C801BE010E9401190F5F1F4F05
:10323000219681E1C339D807A9F7DF91CF911F917A
:103240000F91089541E00E94D8B5089542E00E9490
:10325000D8B508958093B4031092B50380E090E050
:1032600064EB73E00E942619089541E00E94D8B5EE
:10327000089544E00E94D8B5089542E00E94D8B570
:10328000089544E00E94D8B50895CF93DF93EC01F0
:103290008CEC96E00E944394882369F486EC98E0D5
:1032A0000E944394882339F480EC9AE00E9443946E
:1032B000882309F41882DF91CF9108958CEC96E071
:1032C0000E944394882371F486EC98E00E94439412
:1032D000882341F480EC9AE00E944394882319F0FB
:1032E00081E0089581E00895AF92BF92CF92DF927E
:1032F000EF92FF920F931F93DF93CF9300D0CDB740
:10330000DEB700E010E0A4E2EA2EF12CFAEFAF2ED7
:10331000F1E0BF2E6E010894C11CD11C0A9DC001B2
:103320000B9D900D1A9D900D11248453994F0E946E
:1033300058949A838983C701B6010E943D190F5F93
:103340001F4F88E190E0E80EF91E0330110531F7B8
:103350000F900F90CF91DF911F910F91FF90EF9001
:10336000DF90CF90BF90AF9008950E9420B708954E
:1033700021E22093931329E02093941321E032E07B
:1033800030939613209395131092981310929713DD
:1033900020E330E030939A13209399131092A70002
:1033A0000E94E8BB90E0882309F491E0892F0895FA
:1033B000FC0180818823C9F0628743874093D7034B
:1033C0008285813021F48FEF8093D80302C0109260
:1033D000D8031092D9031092DA0381858093DF031A
:1033E00086ED93E060E30E94B8190895CF93DF93D0
:1033F000EC018BA1882329F480919311813009F08D
:103400005CC00E9411C09B01AC0188A999A9AAA91E
:10341000BBA9281B390B4A0B5B0B6EA57FA5611559
:10342000710501F1CB01A0E0B0E0281739074A0788
:103430005B0798F01FA61EA688A599A59DA78CA737
:103440008FA18F5F8FA381E08093931180E091E142
:1034500061E04EEF0E94D8192AC0621B730B7FA750
:103460006EA725C06CA57DA56115710501F1CB0185
:10347000A0E0B0E0281739074A075B07A0F08EA14B
:1034800081508EA3882311F41BA204C08AA59BA59A
:103490009FA78EA780E091E160E04EEF0E94D819CF
:1034A0001092931104C0621B730B7DA76CA70E943E
:1034B00011C068AB79AB8AAB9BABDF91CF9108951C
:1034C000FC0180818823F1F02185413049F481E0BD
:1034D00090E002C0880F991F6A95E2F7282B09C077
:1034E00081E090E002C0880F991F6A95E2F780950D
:1034F0002823218781858093DF0386ED93E060E3B5
:103500000E94B8190895EF92FF920F931F93CF93E3
:10351000DF937C018FE0689F80011124065A1F4FC2
:10352000C4E8D1E107C0C801BE010E94E5180F5FE1
:103530001F4F219681E1C339D807A9F740E0F70171
:1035400084A9882309F441E080E091E162E00E94CF
:10355000601ADF91CF911F910F91FF90EF90089526
:10356000FC018AE085AB16AA17AA10AE14AA81E066
:1035700083AF15AE82E081AF12AE16AE17AE14AEB9
:10358000EE5BFF4F808312921292E054F04080E88D
:1035900083838483858380E091E162E041E00E943F
:1035A000601A08950F931F938C0180E091E10E94AF
:1035B0008915F801118280E883838483858312A2B0
:1035C0001186128613A2C8010E94B01AF801128255
:1035D00087EB96E061E00E9410AF81E08093CB061C
:1035E000F80110821F910F9108950F931F93CF93AD
:1035F000DF93EC018B01888184FF0FC089818823D0
:1036000021F089E793E10E9468C78A81882329F025
:103610008B819C81B8010E9468C7DF91CF911F9177
:103620000F9108950F931F93CF93DF93EC018B01BC
:10363000888183FF0FC08981882321F089E793E186
:103640000E9468C78A81882329F08B819C81B801F8
:103650000E9468C7DF91CF911F910F9108959C013F
:1036600081E08093A7008091A9008F7B8093A900BF
:103670008091A60080FD06C08091A900806480939F
:10368000A9000BC06091F6007091F700C90140E0FD
:1036900050E00E941BB6882311F080E008958091CD
:1036A000A6008E778093A6008091A9008064809305
:1036B000A90081E00895CF93DF93EC0180919B13E3
:1036C0008B3051F58881882339F11FC08E859F8505
:1036D000A889B98989839A83AB83BC838A89C45BAF
:1036E000DF4F8883CC54D0408B89C35BDF4F888306
:1036F000CD54D0408C89C25BDF4F8883CE54D040FC
:103700008D89C15BDF4F888307C0CE010C9660E3D3
:103710000E942F1B8823D1F6DF91CF9108950F933C
:1037200081E863E041E020E430E000E00E9474B60C
:1037300082E063E042E020E430E00E9474B60F9142
:103740000895DF93CF93CDB7DEB7C851D2400FB6FF
:10375000F894DEBF0FBECDBF81E060E0AE01495FEF
:103760005F4F22E10E94F8BC882309F050C081E03D
:10377000BE016F5F7F4FAE01475E5F4F20E032E0DA
:103780000E94E2B9882309F042C08F8598898C5441
:103790009540E9F589899A8988569240C1F581E07A
:1037A0000E9415BD882399F50E948F1B82E48B83AC
:1037B0008CE08C831D821E8281E28093931389E0CA
:1037C0008093941384EF93E09093961380939513D2
:1037D000109298131092971384E090E090939A13AC
:1037E000809399131092A700CE0103960E94E8BB24
:1037F000882369F480E091E10E948F1581E0809335
:10380000001183EE9CE068E171E00E94F51AC85E49
:10381000DD4F0FB6F894DEBF0FBECDBFCF91DF9165
:103820000895A82FFB019A018091A803823041F0EE
:10383000833019F0813089F40AC082EF95E002C02C
:1038400080E995E06A2FAF010E94C1B3089584E535
:1038500096E06A2FAF010E94C1B30895E82F9A0144
:10386000AB018091A803823041F0833019F08130A0
:1038700079F409C082EF95E002C080E995E06E2FEF
:103880000E9439B4089584E596E06E2F0E9439B401
:103890000895E82F9A01AB018091A803823041F08E
:1038A000833019F0813079F409C082EF95E002C0CD
:1038B00080E995E06E2F0E9412B4089584E596E0A9
:1038C0006E2F0E9412B40895282FAB018091A80397
:1038D000823041F0833019F0813079F409C082EFF1
:1038E00095E002C080E995E0622F0E9460B40895DF
:1038F00084E596E0622F0E9460B40895282FAB0102
:103900008091A803823041F0833019F0813079F43E
:1039100009C082EF95E002C080E995E0622F0E9425
:1039200081B4089584E596E0622F0E9481B40895E1
:10393000282F462F8091A803823041F0833019F060
:10394000813079F409C082EF95E002C080E995E00A
:10395000622F0E94EDB3089584E596E0622F0E94E5
:10396000EDB30895682F8091A803823041F0833031
:1039700019F0813069F408C082EF95E002C080E957
:1039800095E00E940CB4089584E596E00E940CB482
:1039900008950F931F93CF93DF93EC018B018881E0
:1039A00083FF0FC08981882321F089E793E10E947A
:1039B0007CC78A81882329F08B819C81B8010E9471
:1039C0007CC7DF91CF911F910F910895EF92FF92E5
:1039D0000F931F93CF93DF93EC017A018B018881C2
:1039E00084FF14C08981882331F089E793E122E0C4
:1039F00030E00E9454C78A81882341F08B819C81EA
:103A0000B801A70122E030E00E9454C7DF91CF91B6
:103A10001F910F91FF90EF90089590E02AEF31E011
:103A2000AC01429FC001439F900D529F900D112405
:103A30008453994F0E94DE930895EF92FF921F9353
:103A4000CF93DF9310E0C0E0D0E041E0E42EF12C12
:103A50008C2F0E940D1D813041F4C7010C2E02C035
:103A6000880F991F0A94E2F7182B2196C330D105CD
:103A700079F7812FDF91CF911F91FF90EF900895FB
:103A80009C01C397C197E0F48CEC96E060E021E0E4
:103A900030E040E050E00E9427A886EC98E060E02B
:103AA00021E030E040E050E00E9427A880EC9AE05E
:103AB00060E021E030E040E050E00E9427A8089557
:103AC00025363105D8F08CEC96E061E021E030E05D
:103AD00040E050E00E9427A886EC98E061E021E0F9
:103AE00030E040E050E00E9427A880EC9AE061E0DE
:103AF00021E030E040E050E00E9427A808954F9276
:103B00005F926F927F928F929F92AF92BF92CF926D
:103B1000DF92EF92FF920F931F93CF93DF930E9458
:103B20004296882381F566247724C0E0D0E05AEFDE
:103B3000452E51E0552EC49D8001C59D100DD49D8C
:103B4000100D11240453194FC8010E9474964B01A3
:103B50005C01C8010E944B966B017C01C8010E9468
:103B60008796C601880D991D860F971F68167906DE
:103B700008F43C012196C330D105E9F687EB96E0C5
:103B8000B3010E9419AFDF91CF911F910F91FF9068
:103B9000EF90DF90CF90BF90AF909F908F907F90ED
:103BA0006F905F904F9008952F923F924F925F9247
:103BB0006F927F928F929F92AF92BF92CF92DF923D
:103BC000EF92FF920F931F93DF93CF9300D000D01B
:103BD000CDB7DEB72224332421011A82198249810C
:103BE0005A818AEF91E0489F9001499F300D589F7C
:103BF000300D11242453394F3C832B83C9010E947B
:103C0000D493882309F44CC00E944296882339F546
:103C100087EB96E00E94EEAE3B014C018B819C81CC
:103C20000E9474965B016C018B819C810E944B9673
:103C30007B018C018B819C810E948796EA0CFB1C86
:103C40000C1D1D1DE60EF71E081F191FC801B70128
:103C5000A40193010E94E6D19B01AC011AC08B81A3
:103C60009C810E9474965B016C018B819C810E94F7
:103C70004B967B018C018B819C810E948796A801C9
:103C800097012A0D3B1D4C1D5D1D260F371F481F38
:103C9000591F221633064406550610F419012A014D
:103CA000E981FA813196FA83E983339709F097CF56
:103CB0002091D2043091D3044091D4045091D50482
:103CC000220D331D441D551DB901CA010F900F90DF
:103CD0000F900F90CF91DF911F910F91FF90EF9078
:103CE000DF90CF90BF90AF909F908F907F906F901C
:103CF0005F904F903F902F9008952F923F924F9258
:103D00005F926F927F928F929F92AF92BF92CF926B
:103D1000DF92EF92FF920F931F93CF93DF930E9456
:103D200011C0662477244301442455246AEF262ECB
:103D300061E0362E429CE001439CD00D529CD00D98
:103D40001124C453D94FCE010E94D4938823F1F09B
:103D5000CE010E9474965B016C01CE010E944B96CD
:103D60007B018C01CE010E948796A80197012A0D44
:103D70003B1D4C1D5D1D260F371F481F591F621626
:103D800073068406950610F439014A010894411C13
:103D9000511C83E04816510469F60E94429688231C
:103DA00091F487EB96E00E941DAFA0E0B0E086158D
:103DB0009705A805B90538F487EB96E00E941DAF7A
:103DC0003C01882499240E944296882339F460910A
:103DD000A3047091A40480E090E014C06091B50445
:103DE0007091B6048091B7049091B8042091D204E8
:103DF0003091D3044091D4045091D504621B730BCD
:103E0000840B950B0E9468D07B018C01C401B30127
:103E10000E9468D09B01AC01C801B7010E94CFCFBE
:103E200020E030E048EC52E40E941ED17B018C017E
:103E300020E030E040E050E00E941AD188234CF0AE
:103E4000C801B70120E030E040E05FE30E9467CFA7
:103E500008C0C801B70120E030E040E05FE30E9405
:103E600066CF0E9437D0162F662301F58091C711C7
:103E70008823E1F00E94FC108823C1F484E680933B
:103E8000C7118091C711DF91CF911F910F91FF90C2
:103E9000EF90DF90CF90BF90AF909F908F907F90EA
:103EA0006F905F904F903F902F9008951093C7119F
:103EB000E8CFAF92BF92CF92DF92EF92FF920F9333
:103EC0001F93DF93CF9300D000D0CDB7DEB700E0D3
:103ED00010E0E6E2EE2EF12C7AEFA72E71E0B72E7D
:103EE0006E010894C11CD11C0A9DC0010B9D900D50
:103EF0001A9D900D11248453994F0E943594698323
:103F00007A838B839C83C701B6010E9441190F5F9E
:103F10001F4F88E190E0E80EF91E0330110521F7EC
:103F20000F900F900F900F90CF91DF911F910F91F5
:103F3000FF90EF90DF90CF90BF90AF9008958AE20E
:103F40000E94EEC0AA2797FDA095BA2FBC01CD0113
:103F50000E946AD020E030EC4FE754E40E94CFCFBB
:103F600020E030E048EC51E40E941ED108951F93F8
:103F7000CF93DF93EC01162F888184FF13C08981D2
:103F8000882331F089E793E14AE050E00E942DC692
:103F90008A81882339F08B819C81612F4AE050E02F
:103FA0000E942DC6DF91CF911F9108951F93CF934B
:103FB000DF93EC01162F888183FF13C0898188234A
:103FC00031F089E793E14AE050E00E941BC68A8104
:103FD000882339F08B819C81612F4AE050E00E9458
:103FE0001BC6DF91CF911F9108951F93CF93DF934D
:103FF000EC01162F888180FF13C08981882331F05E
:1040000089E793E14AE050E00E941BC68A81882339
:1040100039F08B819C81612F4AE050E00E941BC6E1
:10402000DF91CF911F910895FF920F931F93CF932C
:10403000DF93EC01F62E8A01888180FF10C0898110
:10404000882321F089E793E10E941BC68A81882397
:1040500031F08B819C816F2DA8010E941BC6DF91DE
:10406000CF911F910F91FF9008951F93CF93DF93EE
:10407000EC01162F888184FF13C08981882331F0D9
:1040800089E793E14AE050E00E941BC68A818823B9
:1040900039F08B819C81612F4AE050E00E941BC661
:1040A000DF91CF911F9108950F931F93CF93DF93CB
:1040B000EC018B01888183FF0FC08981882321F067
:1040C00089E793E10E94B8C68A81882329F08B8111
:1040D0009C81B8010E94B8C6DF91CF911F910F91CA
:1040E00008950F931F93CF93DF93EC018B01888189
:1040F00080FF0FC08981882321F089E793E10E9426
:10410000B8C68A81882329F08B819C81B8010E94DE
:10411000B8C6DF91CF911F910F9108950F931F9310
:10412000CF93DF93EC018B01888180FF0FC08981E1
:10413000882321F089E793E10E94B8C68A81882309
:1041400029F08B819C81B8010E94B8C6DF91CF9184
:104150001F910F9108950F931F93CF93DF93EC015D
:104160008B01888184FF0FC08981882321F089E732
:1041700093E10E94B8C68A81882329F08B819C81B3
:10418000B8010E94B8C6DF91CF911F910F91089599
:10419000DF92EF92FF920F931F93CF93DF93D82E6E
:1041A00080910B0D90910C0D8230910509F49FC008
:1041B0008330910534F4009769F0019709F046C106
:1041C00028C08330910509F42EC18436910509F089
:1041D0003DC12EC18DE0D81609F43CC19AE0D91634
:1041E00009F438C181E090E090930C0D80930B0DA1
:1041F00090930E0D80930D0D10920F0D1092100DD7
:104200001092110D1092120D1092130D1092140DA8
:1042100021C180910A0D883631F4E9E6DE1609F0F5
:1042200015C18AE00DC08D3629F4F3E7DF1659F485
:104230008EE106C0833761F481E6D81609F582E382
:1042400080930F0DF2C09DE6D91651F488E246C066
:104250008E3661F4E0E7DE1609F0F8C08FE13EC06B
:10426000F0E7DF1609F0F2C08BE238C08A3731F48C
:104270008DE6D81609F0EAC08CE230C0833731F4FD
:104280009DE6D91609F0E2C08AE228C0803731F4F1
:10429000E2E7DE1609F0DAC089E220C0823631F4A6
:1042A000F6E6DF1609F0D2C08CE318C0873631F489
:1042B0008FE6D81609F0CAC08DE3C2CF8A3631F432
:1042C0009DE6D91609F0C2C086E408C0893609F017
:1042D000BDC0EDE6DE1609F0B9C087E480930F0D8E
:1042E00082E090E090930C0D80930B0DB3C09D2D58
:1042F00090539A3020F0FDE2DF1609F065C08091FE
:104300000A0D8032C1F58091100D8F5F8093100DE2
:10431000883248F089E793E168E271E00E94B8C60C
:1043200083E090E0DFCFE82FF0E0EE0FFF1FEE0F0D
:10433000FF1FE35FF24F10821182128213828DE21F
:10434000D81639F48FEF9FEF90930E0D80930D0DDB
:1043500081C081E090E090930E0D80930D0D8D2D26
:1043600090E0C097AA2797FDA095BA2F80839183EC
:10437000A283B3836FC09A3038F56091100DC62FB9
:10438000D0E0CC0FDD1FCC0FDD1FC35FD24FED2C73
:10439000FF24E0EDFFEFEE0EFF1E0027F7FC009577
:1043A000102F688179818A819B812AE030E040E08A
:1043B00050E00E94E6D1E60EF71E081F191FE882A2
:1043C000F9820A831B8346C0F0E2DF1621F08DE0FC
:1043D000D81609F03FC080910A0D80538A30F8F456
:1043E0000091100D0023D9F010E0000F111F000FF5
:1043F000111F035F124F20910D0D30910E0D4427B8
:1044000037FD4095542FF80160817181828193813D
:104410000E94E6D1F8016083718382839383FDE07B
:10442000DF16C1F402C010920F0D84E690E05ACF5F
:104430008AE0D81679F480910A0D8D3059F4809174
:104440000F0D10920C0D10920B0D05C010920C0D5B
:1044500010920B0D80E0D0920A0DDF91CF911F9149
:104460000F91FF90EF90DF900895EF92FF920F93DE
:104470001F93CF93DF93EC017A018B01888183FF37
:1044800014C08981882331F089E793E12AE030E084
:104490000E947DC68A81882341F08B819C81B8016E
:1044A000A7012AE030E00E947DC6DF91CF911F91E5
:1044B0000F91FF90EF900895EF92FF920F931F934B
:1044C000CF93DF93EC017A018B01888184FF14C0C4
:1044D0008981882331F089E793E12AE030E00E9466
:1044E0007DC68A81882341F08B819C81B801A70118
:1044F0002AE030E00E947DC6DF91CF911F910F919D
:10450000FF90EF900895EF92FF920F931F93CF9338
:10451000DF93EC017A018B01888184FF14C08981CB
:10452000882331F089E793E12AE030E00E94F6C564
:104530008A81882341F08B819C81B801A7012AE000
:1045400030E00E94F6C5DF91CF911F910F91FF904F
:10455000EF900895EF92FF920F931F93382F562FED
:10456000742FE22F780184E596E0632F452F272FE3
:104570000E2F0E949CB31F910F91FF90EF90089512
:10458000EF92FF920F931F93382F562F742FE22F25
:10459000780184E596E0632F452F272F0E2F0E9488
:1045A0009CB31F910F91FF90EF9008958F929F926F
:1045B000AF92BF92CF92DF92EF92FF920F931F9331
:1045C000B82EA62E942E822E680180E995E06B2DE0
:1045D0004A2D292D082D76010E949CB382EF95E08B
:1045E0006B2D4A2D292D0E949CB31F910F91FF9096
:1045F000EF90DF90CF90BF90AF909F908F900895F5
:104600000F931F93BC0102EE10E1C8010E94870DB9
:10461000C8011F910F9108954F925F927F928F92E0
:104620009F92AF92BF92CF92DF92EF92FF920F9341
:104630001F93DF93CF93CDB7DEB7CB57D0400FB6E4
:10464000F894DEBF0FBECDBF782E4B012A01EC9649
:104650000CAF1DAF2EAF3FAFEC97B8E0CB2ED12CF7
:10466000CC0EDD1EC6016FE371E00E9460C90E949E
:1046700011C0AB01BC017E010894E11CF11CC70113
:104680002AE00E9493C9C601B7010E940FC966E4DF
:1046900071E00E94F3C8BC018E01015F1F4FC80189
:1046A0000E943FCA83EE9CE0B8010E94C91CC80169
:1046B0000E9450CAC7010E944ACAC6010E9450CA3D
:1046C00083E0871520F081E07816B0F509C084E01A
:1046D000781609F473C085E0781609F0FEC0A9C009
:1046E0008EE891E00E940023BC01ADE1CA2ED12CDE
:1046F000CC0EDD1EC6010E9460C9F6E1EF2EF12C42
:10470000EC0EFD1EC701B4014AE00E94C5C9C601F6
:10471000B7010E940FC966E471E00E94F3C88C01E2
:10472000C2010E940023BC01C8010E94F3C8BC0161
:104730008E010C5D1F4F6DC083E991E00E94002344
:10474000BC01E2E3AE2EB12CAC0EBD1EC5010E9431
:1047500060C96BE2C62ED12CCC0EDD1EC601B401A1
:104760004AE00E94C5C9C501B6010E940FC96AE4AA
:1047700071E00E94F3C88C0159E3E52EF12CEC0E98
:10478000FD1E672D70E061507040C7014AE00E9435
:10479000C5C9C801B7010E940FC966E471E00E9453
:1047A000F3C88C01C2010E940023BC01C8010E9411
:1047B000F3C8BC018E01005C1F4F7BC088E991E00B
:1047C0000E940023BC014EE4C42ED12CCC0EDD1E71
:1047D000C6010E9460C937E4E32EF12CEC0EFD1EE9
:1047E000C701B4014AE00E94C5C9C601B7010E94D1
:1047F0000FC966E471E00E94F3C88C01C2010E94F7
:104800000023BC01C8010E94F3C8BC018E010B5AF1
:104810001F4FC8010E943FCA83EE9CE0B8010E946E
:10482000C91CC8010E9450CAC7010E944ACAC601D9
:1048300052C08DE991E00E940023BC0123E6A22E24
:10484000B12CAC0EBD1EC5010E9460C99CE5C92EED
:10485000D12CCC0EDD1EC601B4014AE00E94C5C9B0
:10486000C501B6010E940FC964E571E00E94F3C85A
:104870008C010E945A86BC018AE6E82EF12CEC0ECF
:10488000FD1EC7014AE00E94C5C9C801B7010E94C8
:104890000FC966E471E00E94F3C88C01C2010E9456
:1048A0000023BC01C8010E94F3C8BC018E010F584F
:1048B0001F4FC8010E943FCA83EE9CE0B8010E94CE
:1048C000C91CC8010E9450CAC7010E944ACAC60139
:1048D0000E944ACAC5010E9450CAEC966CAD7DADDB
:1048E0008EAD9FADEC9728E23BE64EE65EEC0E9473
:1048F000CBCF882339F483EE9CE06DE571E00E9414
:10490000121B26C08091E30C83FF22C08091E40C2F
:10491000882361F089E793E1EC964CAD5DAD6EAD17
:104920007FADEC9722E030E00E9454C78091E50C07
:10493000882371F08091E60C9091E70CEC964CADD9
:104940005DAD6EAD7FADEC9722E030E00E9454C7C4
:10495000C558DF4F0FB6F894DEBF0FBECDBFCF9165
:10496000DF911F910F91FF90EF90DF90CF90BF905C
:10497000AF909F908F907F905F904F9008950F938E
:104980001F9308E21BE62EE63EEC0E940C231F91CB
:104990000F910895EF92FF920F931F93F82EE62E3A
:1049A0008A0181E19EE00E940023BC0183EE9CE02D
:1049B0000E948E2083EE9CE06F2D0E94F51F8AE1FD
:1049C0009EE00E940023BC0183EE9CE00E948E20AA
:1049D00083EE9CE06E2D0E94F51F84E29EE00E9413
:1049E0000023BC0183EE9CE00E948E2083EE9CE0BD
:1049F000F801608140E150E00E9414208EE29EE0C8
:104A00000E940023BC0183EE9CE00E948E2083EE76
:104A10009CE0F801618140E150E00E94142088E3AD
:104A20009EE00E940023BC0183EE9CE00E948E2049
:104A300083EE9CE0F801628140E150E00E94142086
:104A400082E49EE00E940023BC0183EE9CE00E9471
:104A50008E2083EE9CE0F801638140E150E00E94EB
:104A600014208CE49EE00E940023BC0183EE9CE0B5
:104A70000E948E2083EE9CE0F801648140E150E0CA
:104A80000E94142086E59EE00E940023BC0183EE74
:104A90009CE00E948E20E090DD04F090DE04009106
:104AA000DF041091E0048091E30C80FF1AC0809134
:104AB000E40C882341F089E793E1B801A7012AE0DB
:104AC00030E00E94F6C58091E50C882351F080917A
:104AD000E60C9091E70CB801A7012AE030E00E94B3
:104AE000F6C58091E30C80FF16C08091E40C88230A
:104AF00031F089E793E16DE571E00E9468C780912C
:104B0000E50C882341F08091E60C9091E70C6DE56F
:104B100071E00E9468C71F910F91FF90EF90089578
:104B20000F931F93CF93DF93EC018B01888184FF58
:104B30000FC08981882321F089E793E10E941AC57B
:104B40008A81882329F08B819C81B8010E941AC533
:104B5000DF91CF911F910F9108950F931F93CF93E2
:104B6000DF93EC018B01888183FF0FC0898188234B
:104B700021F089E793E10E945BC58A81882329F0AF
:104B80008B819C81B8010E945BC5DF91CF911F9101
:104B90000F9108952F923F924F925F926F927F9262
:104BA0008F929F92AF92BF92CF92DF92EF92FF923D
:104BB0000F931F93DF93CF93CDB7DEB76A970FB6EE
:104BC000F894DEBF0FBECDBF83EE9CE06BE67EE0C7
:104BD0000E94AD251A8E198E9AEF292E91E0392E5A
:104BE000298D3A8D229D8001239D100D329D100D3F
:104BF00011240453194FC8010E9415966F87788BB2
:104C0000898B9A8BC8010E9425966B017C01C80193
:104C10000E9457966B877C878D879E87C8010E946C
:104C200063964B015C01C8010E9474966F8378877C
:104C300089879A87C8010E9487962B013C01C80189
:104C4000B701A6010E940D96C8014F855889698950
:104C50007A890E941D96C801B501A4010E9451964F
:104C6000C8014B855C856D857E850E945D96C80177
:104C7000B2010E946996C8016F8178850E947C9676
:104C8000898D9A8D01969A8F898F039709F0A8CF05
:104C90001E821D828D819E810E945586ED81FE813E
:104CA0002CE230E0E29F7001E39FF00CF29FF00CE9
:104CB000112482EE94E0E80EF91EC7010E946E8670
:104CC0002C01009709F4AAC09A8F898F8C01000FDC
:104CD000111F000F111FC8010E94B00B9E8B3C01D9
:104CE0008D8BC8010E94B00B9F8B4C018C8BC8012F
:104CF0000E94B00B988F5C018B8BB20161507040A9
:104D0000C7010E94048969837A838B839C83222450
:104D10003324CC24DD2435C0C701698D7A8D0E94EF
:104D200004899B01AC0183010C0D1D1D69817A81F1
:104D30008B819C810E9466CFF8016083718382839E
:104D40009383C701698D7A8D0E949E88F401EC0DD2
:104D5000FD1D6083718382839383C701698D7A8D82
:104D60000E94AB86F501EC0DFD1D905860837183A8
:104D7000828393830894211C311C24E030E0C20E0E
:104D8000D31E898D9A8D01979A8F898F24143504AB
:104D90001CF2C7010E947686C7010E947E86C70169
:104DA0000E94A786C701B2010E944E8900E010E070
:104DB000CC24DD2424C0F301EC0DFD1D4081518184
:104DC00062817381C7010E942889F401EC0DFD1DE9
:104DD0004081518162817381C7010E94C288F501BF
:104DE000EC0DFD1D4081518162817381C7010E94DC
:104DF00082860F5F1F4FE4E0F0E0CE0EDF1E041549
:104E00001505CCF28D899E890E945A0C8C899F8948
:104E10000E945A0C8B89988D0E945A0C2D813E81DC
:104E20002F5F3F4F3E832D832330310509F032CF72
:104E30006A960FB6F894DEBF0FBECDBFCF91DF915B
:104E40001F910F91FF90EF90DF90CF90BF90AF90A8
:104E50009F908F907F906F905F904F903F902F909A
:104E600008950F931F93CF93DF93EC018B018881FB
:104E700084FF0FC08981882321F089E793E10E9494
:104E80005BC58A81882329F08B819C81B8010E94AF
:104E90005BC5DF91CF911F910F910895EF92FF9223
:104EA0000F931F93E82E83EE9CE069ED72E10E9460
:104EB00031278091A1048823F1F083EE9CE06FEA12
:104EC00072E10E943127EE2021F08091D0108823DA
:104ED00071F58091A004813039F483EE9CE06CE799
:104EE00072E10E9431271AC083EE9CE062E572E114
:104EF0000E9431271CC0E090B803F090B90300E095
:104F000010E087EB96E00E94EEAEE616F706080783
:104F1000190798F08091D010882379F481E008C0B7
:104F20009091D010911191E081E0892701C080E03B
:104F30001F910F91FF90EF9008950E9411C07B0187
:104F40008C018091CC109091CD10A091CE10B09199
:104F5000CF10E81AF90A0A0B1B0B87EB96E00E94A8
:104F6000EEAE2091B8033091B90340E050E0621BEF
:104F7000730B840B950BE616F70608071907B8F2B2
:104F8000CFCF0F931F93DF93CF93CDB7DEB7279784
:104F90000FB6F894DEBF0FBECDBF8093E1048091C1
:104FA000E30C83FF16C08091E40C882331F089E77D
:104FB00093E165EA7EE00E941AC58091E50C8823A2
:104FC00041F08091E60C9091E70C65EA7EE00E944A
:104FD0001AC58E010F5F1F4FC8016091E1044AE0BE
:104FE0000E94F6C98091E30C83FF16C08091E40C07
:104FF000882329F089E793E1B8010E94AFC7809127
:10500000E50C882349F08091E60C9091E70CBE01F5
:105010006F5F7F4F0E94AFC7CE0101960E944ACAC0
:105020008091E1048823C9F08CEC96E040E050E0E8
:1050300060E070E00E94B89486EC98E040E050E0B8
:1050400060E070E00E94B89480EC9AE040E050E0AC
:1050500060E070E00E94B89403C080E00E940911F3
:1050600027960FB6F894DEBF0FBECDBFCF91DF916C
:105070001F910F9108950F931F93CF93DF93EC012E
:105080008B01888184FF0FC08981882321F089E703
:1050900093E10E94AFC78A81882329F08B819C818C
:1050A000B8010E94AFC7DF91CF911F910F91089572
:1050B0002F923F924F925F926F927F928F929F9228
:1050C000AF92BF92CF92DF92EF92FF920F931F9316
:1050D000DF93CF9300D000D00F92CDB7DEB7D82E9C
:1050E0006D838091A204882309F455C02D2D30E0F2
:1050F0008AEF91E0AC01249FC001259F900D349F61
:10510000900D11248453994F0E944F9F3B014C01F5
:1051100087EB96E00E9402AF7C0187EB96E00E944D
:105120000AAF1B012C0187EB96E00E9406AF5C01E1
:10513000C401B30120E030E04AEF55E40E94CFCF34
:1051400020E030E04AE754E40E941ED13B014C01CC
:1051500000E010E0CC24DD24EA0CFB1C0C1D1D1D1E
:10516000E20CF31C041D151DC801B7010E9468D094
:105170009B01AC01C401B3010E9466CF0E943CD0E8
:10518000AB01BC0187EB96E00E94E8AE5D81552340
:1051900009F0B4C0B5C00E944296882309F04DC002
:1051A00087EB96E00E94EEAE7B018C0187EB96E0E8
:1051B0000E9402AF3C0187EB96E00E940AAF1B0100
:1051C0002C0187EB96E00E9406AF5C012D2D30E0AC
:1051D0008AEF91E0FC012E9FC0012F9F900D3E9F12
:1051E000900D11248453994F0E944F9F69837A83B5
:1051F0008B839C8388249924E618F70808091909E9
:10520000E218F30804091509CC24DD24EA18FB0888
:105210000C091D09C801B7010E9468D020E030E0E8
:105220004AE754E40E94CFCF9B01AC0169817A81A7
:105230008B819C810E94CFCF14C00E94429688230C
:1052400091F08D2D90E02AEF31E0AC01429FC0013A
:10525000439F900D529F900D11248453994F0E94AB
:105260004F9F7B018C0183EE9CE06DE27FE00E940A
:10527000902583EE9CE0B801A7010E94E61CC801BE
:10528000B70120E030E04AE756E40E941AD18823B3
:1052900044F083EE9CE063E17FE00E94312780E0F0
:1052A00032C05D81552361F1C801B70120E030E0D3
:1052B0004AEF55E40E941AD1882364F0C801B7016F
:1052C00020E030E04AE756E40E94CBCF882314F474
:1052D00084E019C0C801B70120E030E04AEF55E48E
:1052E0000E94CBCF882374F4C801B70120E030E0DE
:1052F0004AE755E40E941AD1181624F488E003C046
:1053000081E001C080E10F900F900F900F900F90FF
:10531000CF91DF911F910F91FF90EF90DF90CF9091
:10532000BF90AF909F908F907F906F905F904F90C5
:105330003F902F9008950F931F93CF93DF93182FD3
:10534000062F83EE9CE065EF7EE00E9431270E94ED
:1053500011C08091C1048823B1F5212F30E08AEF7C
:1053600091E0289FE001299FD00D389FD00D112496
:10537000C453D94FCE010E944394882321F5812F35
:1053800061E00E945828182F002321F08823A9F0FB
:1053900011E013C0882311F41FEF0FC0CE01612F5D
:1053A0000E9421AB83EE9CE06EED7EE00E94902592
:1053B00083EE9CE0612F0E94B71F812FDF91CF9178
:1053C0001F910F91089583EE9CE060EB7EE00E94B8
:1053D000312710E0F2CF60E00E949B29089560E041
:1053E0000E9458280895EF92FF921F93CF93DF9366
:1053F00010E0C0E0D0E021E0E22EF12C8C2F0E94E2
:10540000EF29813041F4C7010C2E02C0880F991F8B
:105410000A94E2F7182B2196C330D10579F7812F32
:10542000DF91CF911F91FF90EF9008950F931F93FD
:10543000DF93CF930F92CDB7DEB76983082F10E0CB
:105440008AEF91E0AC01049FC001059F900D149F6D
:10545000900D11248453994F0E9421A1C801880FF7
:10546000991F800F911F33E0880F991F3A95E1F73C
:105470008396BE016F5F7F4F0E9435190F90CF91C9
:10548000DF911F910F9108952F923F924F925F925B
:105490006F927F928F929F92AF92BF92CF92DF9244
:1054A000EF92FF920F931F93DF93CF93CDB7DEB7A9
:1054B00068970FB6F894DEBF0FBECDBF80E090E0D6
:1054C00064EB73E00E94E91882E090E069EA73E01F
:1054D0004AE00E9481B58AE590E068E974E00E94A4
:1054E000ED188BE590E06AE974E00E94ED188CE518
:1054F00090E069E974E00E94ED1880919804823090
:1055000010F01092980480919A04823010F010925A
:105510009A0480919904823010F0109299041982B3
:105520001A821D821E821F82188619861A861B8681
:105530001C861D861E861F86188A198A1A8A1B8A4F
:105540001C8A80E090E0A0E0B0E08D8B9E8BAF8B5A
:10555000B88F1C821B82A9EAAA2EA4E0BA2ECC2402
:10556000DD24F2E2EF2EF12CE1E12E2E312C2C0E77
:105570003D1E75E1472E512C4C0E5D1E63E0662EDC
:10558000712C6C0E7D1E5AEF852E51E0952EC701B1
:10559000BE016F5F7F4F0E94ED18C7010196BE01EB
:1055A0006E5F7F4F0E94F118C7014097BE016B5F8D
:1055B0007F4F0E94F518C7010897BE01675F7F4FB4
:1055C0000E94F518C7010497BE01635F7F4F0E94D8
:1055D000F518C7010C97B1010E94F518C701049690
:1055E000B2010E94F918C7010296B3010E94FD188A
:1055F000C89C8001C99C100DD89C100D1124045327
:10560000194FC80169810E9421AB80E591E16C2DA1
:1056100049810E948516C8016A810E9421A14D8995
:105620005E896F89788DC8010E9401946B817C81AD
:10563000C8010E949C9480919804882339F04D8180
:105640005E816F817885C8010E942D9680919A04B1
:10565000882371F049855A856B857C85C8010E9435
:105660000D964D855E856F857889C8010E941D96CF
:1056700080919904882349F089899A89AB89BC89EA
:10568000F50180839183A283B3830894C11CD11C4C
:1056900088E190E0E80EF91EE4E0F0E0AE0EBF1EF7
:1056A000F3E0CF16D10409F072CF0AE510E0B8019B
:1056B000665D7E4EC8010E94E5180F5F1F4F0936D8
:1056C0001105A9F768960FB6F894DEBF0FBECDBFDF
:1056D000CF91DF911F910F91FF90EF90DF90CF90CE
:1056E000BF90AF909F908F907F906F905F904F9002
:1056F0003F902F9008958091CA06882331F08091C1
:10570000C611882391F01092C61180919E048730B3
:1057100041F080919F04873021F08AEB9CE062E0A9
:105720000AC08AEB9CE066E006C081E08093C61167
:105730008AEB9CE064E00E94A6AE0895843051F4A8
:1057400083EE9CE063ED74E10E9431278AEB9CE0DC
:1057500064E014C08230A9F483EE9CE06EEB74E147
:105760000E9431278091A3049091A4040196909304
:10577000A4048093A3048AEB9CE065E00E94A6AE9B
:105780000895863011F40E947B2B08958AEB9CE0EB
:1057900060E00E94A6AE87EB96E00E94C7AF089536
:1057A0008CEC96E00E944394882361F486EC98E0A8
:1057B0000E944394882331F480EC9AE00E94439441
:1057C0008823F9F08091A7048823D9F482E00E940D
:1057D0004C158CEC96E00E948994AC0160E070E07E
:1057E0008EEE91E10E94987F8EEE91E16CE372E380
:1057F0002FEF3FEF4FEF5FEF0E94AF7F81E080938D
:10580000A70408954F925F926F927F928F929F921A
:10581000AF92BF92CF92DF92EF92FF920F931F93BE
:10582000CF93DF93582E3A014B01422E222309F0E9
:1058300042C0282F30E08AEF91E0289F6001299F25
:10584000D00C389FD00C11248CEC96E0C80ED91ED9
:10585000C60164E00E9421ABC6010E94A893E82E15
:10586000C6010E94AD935C01C401B3010E946AD0DD
:105870003B014C01FF2400E010E0C801B7010E9489
:1058800068D07B018C01CC24B7FCC094DC2CC60111
:10589000B5010E946AD09B01AC01C801B7010E940A
:1058A000CFCF9B01AC01C401B3010E941ED10E9465
:1058B00037D03B014C0183EE9CE06CE57EE00E941A
:1058C000902583EE9CE0652D0E94352083EE9CE0C0
:1058D0006EE571E00E94AB2083EE9CE0B401A30171
:1058E0000E945C22252D30E08AEF91E0289FE001A4
:1058F000299FD00D389FD00D1124C453D94FCE010C
:105900000E945894A0E0B0E0BC01CD010E9468D094
:10591000AB01BC01CE010E94B894CE01B401A30139
:1059200021E00E94B7A783EE9CE06CE671E00E9444
:10593000AB20CE010E94ED93AB01BC0183EE9CE055
:105940000E94E61C83EE9CE064E771E00E94AB20BD
:10595000CE010E94FC93682F83EE9CE00E94B71F4B
:105960000E94D02B442021F4CE0161E00E94F7A0D8
:10597000DF91CF911F910F91FF90EF90DF90CF902B
:10598000BF90AF909F908F907F906F905F904F905F
:10599000089520E00E94022C08950F931F9390E039
:1059A0002AEF31E0829F8001839F100D929F100D9E
:1059B00011240453194FC80164E00E9421ABC801AF
:1059C0000E945894A0E0B0E0BC01CD010E9468D0D4
:1059D000AB01BC01C8010E94B894C8010E9403A891
:1059E0000E94D02BC80161E00E94F7A01F910F9187
:1059F00008958CEC96E00E9443948823A1F486ECF1
:105A000098E00E944394882371F480EC9AE00E940D
:105A10004394882341F40E94CD2C81E00E94CD2C38
:105A200082E00E94CD2C08956F927F928F929F9278
:105A3000AF92BF92CF92DF92EF92FF920F931F939C
:105A4000CF93DF9390E02AEF31E0829FE001839FC4
:105A5000D00D929FD00D1124C453D94FCE010E9476
:105A600025967B018C01CE010E9415965B016C018D
:105A7000CE010E9415963B014C01CE010E94359645
:105A800030E0EA18FB080C091D091E141F0410065B
:105A900011060CF431E020E0661A770A880A990AA8
:105AA00016141704180419040CF421E0321719F025
:105AB000CE0161E002C0CE0160E00E9470A0CE0184
:105AC00064E00E9421ABCE010E945894A0E0B0E0B7
:105AD000BC01CD010E9468D0AB01BC01CE010E9487
:105AE000B894CE010E9411A80E94D02BCE0161E093
:105AF0000E94F7A0DF91CF911F910F91FF90EF903F
:105B0000DF90CF90BF90AF909F908F907F906F90DD
:105B100008958CEC96E00E9443948823A1F486ECCF
:105B200098E00E944394882371F480EC9AE00E94EC
:105B30004394882341F40E94142D81E00E94142D87
:105B400082E00E94142D08952F923F924F925F920F
:105B50006F927F928F929F92AF92BF92CF92DF927D
:105B6000EF92FF920F931F93DF93CF9300D000D05B
:105B700000D0CDB7DEB749835A836B837C832AEF8D
:105B800031E0829FA001839F500D929F500D112400
:105B90004453594F5E834D83CA010E94E3937B01B6
:105BA0008C0169817A818B819C8120E030E040E02A
:105BB00050E00E941AD118162CF4A980BA80CB802C
:105BC000DC8008C0A980BA80CB80DC80D7FAD09472
:105BD000D7F8D0948D819E810E945894A0E0B0E0C7
:105BE000BC01CD010E9468D09B01AC01C601B5018A
:105BF0000E941AD118162CF0A980BA80CB80DC80C4
:105C000029C069817A818B819C8120E030E040E06D
:105C100050E00E94CBCF88238CF48D819E810E941E
:105C20005894A0E0B0E0BC01CD010E9468D05B01B7
:105C30006C01D7FAD094D7F8D0940CC08D819E8196
:105C40000E945894A0E0B0E0BC01CD010E9468D051
:105C50005B016C018D819E81B601A5010E94B89403
:105C6000C801B70120E030E040E050E00E941AD1C6
:105C700018165CF4C801B70120E030E040E85FE3AB
:105C80000E94CBCF87FD0BC03BC0C801B70120E00D
:105C900030E040E85FEB0E941AD1181604F5C60107
:105CA000B50120E030E040E050E00E941AD1181623
:105CB00064F4C601B50120E030E040E85FE30E94F3
:105CC0001AD118160CF47DC00AC0C601B50120E037
:105CD00030E040E85FEB0E94CBCF87FD5CC0C8019D
:105CE000B70120E030E040E050E00E941AD11816E1
:105CF0003CF01701280157FA509457F8509402C00D
:105D000017012801C601B50120E030E040E050E075
:105D10000E941AD118161CF43501460106C035013F
:105D2000460197FA909497F89094C801B701A201A0
:105D300091010E94CFCF7B018C01C601B501A40166
:105D400093010E94CFCF9B01AC01C801B7010E9413
:105D5000CBCF882309F44CC0C601B50120E030E068
:105D600040E050E00E941AD118165CF4C601B5015B
:105D700020E030E040E85FE30E941AD118160CF1F1
:105D800037C0C601B50120E030E040E85FEB0E947B
:105D9000CBCF88236CF5C601B50120E030E040E8A8
:105DA0005FE30E941AD1181664F0C601B50120E025
:105DB00030E040E85FE30E94CBCF88231CF410E082
:105DC00001C011E08D819E8161E00E94F7938D8179
:105DD0009E81612F20E030E040E050E00E9427A843
:105DE0000E94D02B83EE9CE06EE77EE00E94AD2502
:105DF00069817A818B819C8120E030E040E050E035
:105E00000E94CBCF882339F58CEC96E00E94E39377
:105E100020E030E040E050E00E94CBCF882311F535
:105E200086EC98E00E94E39320E030E040E050E010
:105E30000E94CBCF8823B1F480EC9AE00E94E393D8
:105E400020E030E040E050E00E94CBCF882351F4C6
:105E50001092DC0407C00E940E11882319F081E023
:105E60008093DC0426960FB6F894DEBF0FBECDBF3C
:105E7000CF91DF911F910F91FF90EF90DF90CF9026
:105E8000BF90AF909F908F907F906F905F904F905A
:105E90003F902F9008952F923F924F925F926F9272
:105EA0007F928F929F92AF92BF92CF92DF92EF92AA
:105EB000FF920F931F93CF93DF930E9411C07B013A
:105EC0008C0180916A0590916B05A0916C05B09151
:105ED0006D05E81AF90A0A0B1B0B0E946986AA27AE
:105EE00097FDA095BA2F8E159F05A007B10708F062
:105EF000E5C044245524BCE22B2E312C429CE00109
:105F0000439CD00D529CD00D1124CE51DB4FCE01BD
:105F10000E946E86BC0161507040CE010E940489CF
:105F20007B018C010E944296882371F487EB96E0F6
:105F30000E94EEAE0E9468D09B01AC01C801B7017F
:105F40000E941ED17B018C01CE010E946E86181624
:105F500019060CF082C060916E0570916F058091FA
:105F60007005909171050E9468D03B014C016091D1
:105F7000D2047091D3048091D4049091D5040E94EE
:105F800068D09B01AC01C801B7010E9467CF9B019B
:105F9000AC01C401B3010E941AD118160CF450C010
:105FA000CE0160E070E00E9404897B018C01609169
:105FB000D2047091D3048091D4049091D5040E94AE
:105FC00068D09B01AC01C801B7010E9467CF9B015B
:105FD000AC01C401B3010E94CBCF87FD31C06091F9
:105FE0006E0570916F0580917005909171050E940A
:105FF00068D05B016C01CE010E946E86BC016150CD
:106000007040CE010E9404897B018C016091D20412
:106010007091D3048091D4049091D5040E9468D0EB
:106020003B014C01C801B701A40193010E9467CF55
:106030009B01AC01C601B5010E941AD1181604F5E6
:10604000A0E050E040E060E0C2012A2F352FE42FAD
:10605000F62FA901BF010E94A42D0894411C511CD8
:1060600083E04816510409F049CF0E9411C06093A3
:106070006A0570936B0580936C0590936D051EC047
:1060800060916E0570916F0580917005909171051A
:106090000E9468D0A40193010E9466CFAB01BC01AD
:1060A000CE010E94568820E030E04AE754E40E9486
:1060B0001ED1A62F572F482F692FC6CFDF91CF9122
:1060C0001F910F91FF90EF90DF90CF90BF90AF9016
:1060D0009F908F907F906F905F904F903F902F9008
:1060E00008959F92AF92BF92CF92DF92EF92FF926C
:1060F0000F931F93CF93DF93982E10E0CC24DD24D1
:106100000AEFA02E01E0B02ECA9CE001CB9CD00D7E
:10611000DA9CD00D1124C453D94FCE010E9478A02F
:106120008130A9F5CE010E94C393892B81F1CE0164
:1061300064E00E9421ABCE010E945894A0E0B0E040
:10614000BC01CD010E9468D0AB01BC01CE010E9410
:10615000B894CE010E9425967B018C01CE010E944D
:10616000159620E0E61AF70A080B190B1E141F04F7
:10617000100611060CF421E0CE01622F21E030E080
:1061800040E050E00E9427A80E94D02B11E0089424
:10619000C11CD11C23E0C216D10409F0B5CF1123D4
:1061A00089F0992079F40E9411C07B018C010E9432
:1061B00011C06E197F09800B910B6C5271408040A9
:1061C0009040A8F3C0E0D0E01AEFE12E11E0F12EEC
:1061D000CE9D8001CF9D100DDE9D100D1124045326
:1061E000194FC8010E9482AC83EE9CE06BE67FE011
:1061F0000E949025C8010E94A893682F83EE9CE01E
:106200000E94B71F2196C330D10511F783EE9CE0A1
:1062100060E57FE00E943127DF91CF911F910F91C0
:10622000FF90EF90DF90CF90BF90AF909F90089538
:1062300080E00E94713008958F929F92BF92CF921A
:10624000DF92EF92FF920F931F93CF93DF9386EB32
:1062500096E00E94EF92B82E8CEC96E00E94D493C8
:10626000882309F06BC086EC98E00E94D4938823C1
:1062700009F064C080EC9AE00E94D493882309F06E
:106280005DC08AEB9CE06B2D0E94A6AE5EC0C89CF0
:10629000E001C99CD00DD89CD00D1124C453D94F16
:1062A000CE010E94D4938823F1F1CE010E9474960E
:1062B000611571058105910531F1E090A304F0901D
:1062C000A40400E010E0CE010E9474966E157F05D4
:1062D0008007910720F00E944296882321F10E94B6
:1062E0004296882381F0E090B504F090B6040091C6
:1062F000B7041091B804CE010E9474966E157F0504
:106300008007910780F4CE010E947CAA0E944296E9
:10631000882321F48AEB9CE063E003C08AEB9CE0D5
:106320006B2D0E94A6AE0894C11CD11C83E0C81638
:10633000D10409F0ACCF0E94D02B07C0CC24DD24BF
:106340008AEF882E81E0982EA2CFDF91CF911F9106
:106350000F91FF90EF90DF90CF90BF909F908F9024
:1063600008958F929F92AF92BF92CF92DF92EF9259
:10637000FF920F931F93DF93CF9300D000D0CDB740
:10638000DEB7EE24FF2422E1C22ED12C9AEF892E13
:1063900091E0992E5E010894A11CB11CE89C80013B
:1063A000E99C100DF89C100D11240453194FC801DD
:1063B0000E940495C8010E94359669837A838B8375
:1063C0009C83C601B5010E9439190894E11CF11C97
:1063D00088E190E0C80ED91E93E0E916F104F1F6C9
:1063E0001092A70481E00E944C158EEE91E10E946C
:1063F000A07F0F900F900F900F90CF91DF911F9182
:106400000F91FF90EF90DF90CF90BF90AF909F9053
:106410008F9008951F93CF93DF93EC0180E091E17B
:1064200064E00E949C15182F833031F40E9411C043
:106430006E8F7F8F88A399A30E945E19882311F421
:10644000188216C01130A1F40E9411C02E8D3F8D0C
:1064500048A159A1621B730B840B950B615D7740BA
:106460008040904028F01AA20E94B13183E08883D6
:10647000DF91CF911F910895AF92BF92CF92DF929B
:10648000EF92FF920F931F93CF93DF935EECE52E75
:1064900056E0F52E00E010E04AEFA42E41E0B42EC5
:1064A00031E0C32ED12C0A9DE0010B9DD00D1A9D29
:1064B000D00D1124C453D94FCE010E944394882398
:1064C000A9F0CE010E9456A0CE010E947EA388238F
:1064D00069F09601F701008002C0220F331F0A9471
:1064E000E2F78091A804822B8093A8040F5F1F4FCE
:1064F0008AEF91E0E80EF91E03301105A1F681B391
:106500009091A804892B81BB81E090E00E949EC0FD
:1065100091B38091A8048095892381BB1092A8042F
:106520008CEC96E00E944394882371F486EC98E00A
:106530000E944394882341F480EC9AE00E944394A3
:10654000882311F40E94B131DF91CF911F910F91F7
:10655000FF90EF90DF90CF90BF90AF9008958CECBC
:1065600096E00E944394882361F486EC98E00E94B0
:106570004394882331F480EC9AE00E94439488236A
:1065800011F00E94B1318CEC96E00E945C9586EC93
:1065900098E00E945C9580EC9AE00E945C950895DA
:1065A0000E947A7E80919E048650823048F460E09A
:1065B0008091C103882309F461E088E10E94A0C1B1
:1065C00080919F048650823048F460E08091C1033E
:1065D000882309F461E089E10E94A0C18091D01074
:1065E000863021F48AEB9CE061E003C08AEB9CE0FA
:1065F00062E00E94A6AE08958CE060E00E94A0C117
:106600001092DC0C08958CE061E00E94A0C181E052
:106610008093DC0C08958091DC0C882319F00E9493
:10662000FC3208950E94033308950E94E8108823E5
:1066300019F00E94033308950E94FC3208951F93BD
:10664000182F83EE9CE064E071E10E94902580E0C9
:1066500090E040E050E060E070E00E94A42D81E016
:1066600090E040E050E060E070E00E94A42D82E005
:1066700090E040E050E060E070E00E94A42D80E0F7
:106680000E94C12710928205109283051092D804AF
:106690001123A1F41092C8041092C9041092CA04E4
:1066A0001092CB041092CD041092CC040E94F614E8
:1066B000882321F00E94F3140E94CA250E9442966A
:1066C000823021F487EB96E00E94C7AF0E94153319
:1066D0001F91089580E00E941F330895CF93DF93A8
:1066E00083EE9CE068E271E10E949025C0E0D0E07A
:1066F00083EE9CE068E171E10E94902583EE9CE0CE
:106700006C2F0E94B71FCE0140E050E060E070E0C7
:106710000E94A42D2196C330D10551F781E08093CA
:1067200083051092760510927705109278051092E5
:1067300079050E9411C06093720570937305809370
:106740007405909375050E941533DF91CF910895DC
:10675000AF92BF92CF92DF92EF92FF920F931F936F
:106760008091D704882309F063C080918305882332
:1067700009F05EC00E94E810882359F40F2EFDEC4A
:10678000AF2EFCECBF2EFCECCF2EFDE3DF2EF02D68
:106790000AC00F2EF6E6AF2EF6E6BF2EF6E6CF2E97
:1067A000FFE3DF2EF02D0E9411C02091D111309116
:1067B000D2114091D3115091D411621B730B840BF1
:1067C000950B615D77408040904068F00E940333F4
:1067D0000E9411C06093D1117093D2118093D31194
:1067E0009093D41125C00E9411C07B018C0180912F
:1067F000D1119091D211A091D311B091D411E81A76
:10680000F90A0A0B1B0BC601B50120E030E04AEF84
:1068100054E40E941ED10E9437D0882777FD8095CE
:10682000982F6E157F058007910710F40E94FC32A7
:106830001F910F91FF90EF90DF90CF90BF90AF909E
:106840000895FC01EB5BFB4F90E0662309F491E0B7
:106850008081692F0E94A0C108954F925F926F922C
:106860007F928F929F92AF92BF92CF92DF92EF92E0
:10687000FF920F931F93CF93DF932C017A018B012B
:106880008FEF90E0489EF001499EF00D589EF00D6C
:106890001124E554F14FA080B180C280D380A416AA
:1068A000B506C606D7061CF0CFEFDFEF02C0C1E089
:1068B000D0E08FEF90E0489EF001499EF00D589E89
:1068C000F00D1124E753F14F608171818281938132
:1068D00020E030E040E050E00E94CBCF882321F060
:1068E000C2010E944F1195C0CE01880F991F3C0133
:1068F000882477FC8094982CA60CB71CC81CD91C43
:10690000C130D10531F4EA14FB040C051D055CF41B
:1069100008C0CF5FDF4F39F4AE14BF04C006D10604
:1069200014F4570168018FEF90E0489EF001499EF2
:10693000F00D589EF00D1124E85FF14F80E090E0DB
:1069400020E030E040E050E0F8972083318342833C
:106950005383F8962083318342835383248F358F6A
:10696000468F578F019634968730910569F78FEFE0
:1069700090E0489EF001499EF00D589EF00D1124C4
:10698000E253F24FEC51FF4F208331834283538314
:10699000E45EF0408AE097EDA3E2BCE38283938358
:1069A000A483B583E751FF4F80819181A281B38198
:1069B000E95EF040868F978FA0A3B1A3680E791E81
:1069C0008A1E9B1E62A273A284A295A2EE51FF4F63
:1069D000118210823B96A082B182C282D382A81615
:1069E000B906CA06DB06A9F081E090E0A0E0B0E0BD
:1069F000042C04C0880F991FAA1FBB1F0A94D2F74A
:106A00002091C90D282B2093C90DC20161E00E947D
:106A10002134DF91CF911F910F91FF90EF90DF9084
:106A2000CF90BF90AF909F908F907F906F905F902E
:106A30004F9008952F923F924F925F926F927F9264
:106A40008F929F92AF92BF92CF92DF92EF92FF927E
:106A50000F931F93DF93CF93CDB7DEB728970FB671
:106A6000F894DEBF0FBECDBF8091C70D882321F003
:106A70001092C70D0E94DC12F0EB6F2EFEE07F2E0D
:106A800018861F82D30158961C921E92579720E0B9
:106A900030E040E050E059962D933D934D935C9348
:106AA0005C971091C90D812F90E00F8002C09595E1
:106AB00087950A94E2F780FF69C1ED91FC91FA8312
:106AC000E9836F01CC0CDD1CCC0CDD1C2F813885DB
:106AD0004FEF50E0249FC001259F900D349F900DF3
:106AE0001124C80ED91E80ED9DE0C80ED91ED60116
:106AF0006D917D918D919C9120E030E040E050E0DF
:106B00000E94CBCF882341F581E090E0A0E0B0E087
:106B10000F8004C0880F991FAA1FBB1F0A94D2F7C9
:106B2000809581238093C90DEF81F8852AEF31E0AC
:106B3000E29FC001E39F900DF29F900D11248453BA
:106B4000994F0E94DE93882309F420C18F81988594
:106B500060E00E9421341AC1D30112968D919D915B
:106B60000D90BC91A02D8B839C83AD83BE83BC0113
:106B7000CD012DEC3CEC4CE45DE30E9467CF7B0142
:106B80008C01F3016283738384839583D601AD9076
:106B9000BD90CD90DC90A60195010E941AD187FF8F
:106BA00003C089819A8110C0C801B701A60195016F
:106BB0000E9466CFF3016283738384839583898106
:106BC0009A81019691838083D30112968D909D9036
:106BD000AD90BC9015978C01000F111F000F111F75
:106BE000EF81F8852FEF30E0E29FC001E39F900D29
:106BF000F29F900D1124080F191F0253124FD80154
:106C00005E966D917D918D919C9191970E946AD035
:106C10006B017C01C501B401F80122AD33AD44AD77
:106C200055AD0E941ED19B01AC01C701B6010E9467
:106C300067CF6B017C010A5A1F4FC501B401D8010F
:106C40002D913D914D915C910E941ED1A501940121
:106C50000E941ED19B01AC01C701B6010E9467CF03
:106C60000E9437D01B012C01F30187819085A185FB
:106C7000B28562015101A81AB90ACA0ADB0AD7FE15
:106C800008C0D094C094B094A094A11CB11CC11CA5
:106C9000D11CA114B104C104D10409F477C0882423
:106CA00082159305A405B50514F4882483942F81D7
:106CB00038854FEF50E0249FF001259FF00D349F61
:106CC000F00D1124EA54F14F8081881671F08B8108
:106CD0009C81AD81BE81F30182839383A483B583BC
:106CE00029813A813183208343C0C601B5010E94C6
:106CF0006AD023E333E343E852E40E941ED17B01D0
:106D00008C0120E03FEF4FE757E40E941AD118169C
:106D1000ACF0C801B70120E030E040E85FE30E943A
:106D2000CBCF8823ACF40F2EF0E0EF2EF0E0FF2E57
:106D3000F0E80F2FFFE31F2FF02D0AC00F2EF0E019
:106D4000EF2EFFEFFF2EFFE70F2FF7E41F2FF02DA1
:106D5000D3015996ED92FD920D931C935C97589632
:106D6000BC92AE925797F3012782308641865286B5
:106D70002F8138854FEF50E0249FF001259FF00DC3
:106D8000349FF00D1124EA54F14F80828F81988551
:106D9000019698878F83AFEFB0E06A0E7B1E039752
:106DA00009F070CE81E08093C30D28960FB6F89459
:106DB000DEBF0FBECDBFCF91DF911F910F91FF902E
:106DC000EF90DF90CF90BF90AF909F908F907F908B
:106DD0006F905F904F903F902F9008952F923F9229
:106DE0004F925F926F927F928F929F92AF92BF92DB
:106DF000CF92DF92EF92FF920F931F93CF93DF9387
:106E000090E08091CA0D882309F491E09093CA0D17
:106E1000992309F467C04091B70D5091B80D411501
:106E20005105D9F02091B10D3091B20D8091BD0D79
:106E30009091BE0D820F931F9093B20D8093B10D70
:106E40008217930750F4415050405093B80D40932F
:106E5000B70D8DE261E00E94A0C14091B90D509143
:106E6000BA0D41155105D9F02091B30D3091B40DF3
:106E70008091BF0D9091C00D820F931F9093B40D20
:106E80008093B30D8217930750F4415050405093B4
:106E9000BA0D4093B90D8EE261E00E94A0C140910D
:106EA000BB0D5091BC0D4115510509F4B1C02091A5
:106EB000B50D3091B60D8091C10D9091C20D820F2C
:106EC000931F9093B60D8093B50D8217930708F02A
:106ED0009FC0415050405093BC0D4093BB0D8FE27A
:106EE00061E094C08091C40D9091C50D019690937E
:106EF000C50D8093C40D885E934009F07DC010924B
:106F0000C50D1092C40D8091C60D882319F08150D3
:106F10008093C60D00EDC02E03E0D02E1AEC812E1A
:106F200013E0912EC7ECDEE0B4ECAB2EB3E0BB2E49
:106F3000EE24FF24A1E04A2E512C612C712C222436
:106F40002A94322CD601ED91FC9180819181892B7C
:106F5000D9F06A817B818C819D8120E030E040E026
:106F600050E00E94CBCF882379F4D301C2010E2CCC
:106F700004C0880F991FAA1FBB1F0A94D2F7209143
:106F8000C80D282B2093C80DD401ED91FD914D0122
:106F90008881998191838083F601019111916F011C
:106FA0006A817B818C819D810E943CD0D8016D9348
:106FB0007C938FEF90E0E89EF001E99EF00DF89E43
:106FC000F00D1124EA54F14F6081C85FD0408881F0
:106FD0000E94A0C1D501ED91FD915D013182208219
:106FE0000894E11CF11CC950DE4FB3E0EB16F1042C
:106FF00009F0A8CF1092C30D8DE260E00E94A0C1FD
:107000008EE260E00E94A0C18FE260E00E94A0C119
:10701000DF91CF911F910F91FF90EF90DF90CF9074
:10702000BF90AF909F908F907F906F905F904F90A8
:107030003F902F9008951F93CF93DF93182F8630A2
:1070400029F4C091BC03D091BD0304C0C091BE031C
:10705000D091BF0380919E04181711F090E006C0F4
:1070600088E16091C1030E94A0C191E080919F04DA
:10707000181731F489E16091C1030E94A0C102C0D8
:10708000992369F0BE0180E090E040ED52E30E9458
:107090001C7E0E94647E8AEB9CE060E009C0163092
:1070A00021F48AEB9CE061E003C08AEB9CE062E0A3
:1070B0000E94A6AEDF91CF911F9108958091B311E8
:1070C0008823A1F483EB91E10E94E2C4892B71F043
:1070D0000E9411C06093BB117093BC118093BD11CD
:1070E0009093BE1183EB91E10E94ECC480919E04C9
:1070F000873051F080919F04873031F08AEB9CE01B
:1071000062E00E94A6AE08958091D010882371F4A9
:1071100087E08093D0100E9411C06093BB117093E0
:10712000BC118093BD119093BE1108950E9411C0AF
:107130002091BB113091BC114091BD115091BE11F5
:10714000621B730B840B950B2091BA033091BB0328
:1071500040E050E0261737074807590728F41092F7
:10716000D01087E00E941B380895FF920F931F9361
:10717000F82E062FE82FF0E0E256FB4F608381E007
:10718000F816D9F1FF2019F482E00E9415BE18E12B
:10719000002329F4812F60E00E941DC133C00650F6
:1071A0000230E8F0812F60E00E941DC1812F61E074
:1071B0000E94A0C1FF2021F081E0F81619F506C059
:1071C0004091C00382E060E17CE605C04091C003CD
:1071D00083E06CE07CE650E00E9499BD13C0812FF3
:1071E00061E00E941DC160E08091C103882309F421
:1071F00061E0812F0E94A0C105C083E00E9415BEFE
:1072000019E1C6CF1F910F91FF90089580E0609122
:107210009E040E94B53881E060919F040E94B538B9
:1072200090E080919E04843009F491E080919F0465
:10723000843009F491E09093A1040895882399F093
:1072400080E00E943B1580E064E00E94B53881E058
:1072500064E00E94B5380E94063981E08093A20460
:107260000E940333089580E060E00E94B53881E019
:1072700060E00E94B5380E9406391092A2040E9474
:10728000FC320895EF92FF920F931F93CF93DF93F9
:10729000EC017A018B01888184FF14C089818823E5
:1072A00031F089E793E12AE030E00E9441C68A810B
:1072B000882341F08B819C81B801A7012AE030E04E
:1072C0000E9441C6DF91CF911F910F91FF90EF90E7
:1072D0000895EF92FF920F931F930E94429682307F
:1072E000F1F087EB96E00E941DAF7C0187EB96E002
:1072F0000E94EEAE9B01AC0100E010E0C801B701B6
:107300000E94E6D1F62E072F182FE92E80918205D4
:107310008823A9F483EE9CE060E97FE00EC00E9420
:107320004386F62E072F182FE92E80918205882399
:1073300031F483EE9CE068E77FE00E949025809125
:107340008205882371F483EE9CE04F2D502F612F2E
:107350007E2D0E94423983EE9CE061E871E00E943C
:10736000F51A6F2D702F812F9E2D1F910F91FF9079
:10737000EF9008958F929F92AF92BF92CF92DF923B
:10738000EF92FF920F931F930E9469394B015C01AA
:1073900087EBC82E86E0D82EC6010E9406AF7C017E
:1073A000C6010E940AAF00E010E0E80CF91C0A1DBB
:1073B0001B1DE60EF71E081F191FB701C8011F91FC
:1073C0000F91FF90EF90DF90CF90BF90AF909F9084
:1073D0008F900895EF92FF920F931F930E94429611
:1073E000823079F460916E0570916F05809170051F
:1073F000909171050E9468D07B018C010E946939CF
:107400000EC060916E0570916F058091700590912E
:1074100071050E9468D07B018C010E94BA399B01E2
:10742000AC016091D2047091D3048091D404909106
:10743000D504620F731F841F951F0E9468D09B01A3
:10744000AC01C801B7010E94CFCF20E030E048EC8A
:1074500052E40E941ED10E9437D0CB011F910F91A0
:10746000FF90EF9008950E944296823019F40E9496
:10747000693902C00E94BA399B01AC018091D204E3
:107480009091D304A091D404B091D504280F391F52
:107490004A1F5B1FB901CA0108952F923F924F9274
:1074A0005F926F927F928F929F92AF92BF92CF9294
:1074B000DF92EF92FF920F931F93DF93CF9300D051
:1074C00000D0CDB7DEB70E945C15882309F494C1C3
:1074D0000091A3041091A40487EB96E00E941DAFD5
:1074E0000817190709F088C18DC18091A00488236D
:1074F00059F48091DB10882339F483EE9CE06FE12E
:1075000070E10E9431277EC180919E04863039F05F
:1075100080919F04863019F080E090E004C0809153
:10752000B8039091B9039C01442737FD4095542F2F
:1075300029833A834B835C8387EB96E00E94EEAE0F
:107540007B018C01A0906E05B0906F05C090700516
:10755000D090710560907E0570907F0580908005C9
:107560009090810587EB96E00E94EEAE29813A81EA
:107570004B815C812E153F054007510768F4A61822
:10758000B708C808D908621B730B840B950BA616A5
:10759000B706C806D90620F08091D010882321F0C4
:1075A0008091A004882329F180916E0590916F0548
:1075B000A0917005B091710580937E0590937F0531
:1075C000A0938005B09381051092D5101092D6102B
:1075D0001092D7101092D8101092D9101092DA1081
:1075E0008091A004882329F081E08093DB10109221
:1075F000A00480919E04863021F080919F04863003
:10760000E9F581E00E944E278823C1F18091D610D0
:107610008823A1F58091D510882379F486E08093A2
:10762000D0100E941B3883EE9CE067EE7FE00E9442
:10763000312781E08093D510E5C080917E0590913F
:107640007F05A0918005B091810529813A814B8108
:107650005C81820F931FA41FB51F20916E0530918E
:107660006F054091700550917105281739074A0739
:107670005B0708F4C7C081E08093D6101092D01049
:107680001092A0048091D810882309F049C08091FD
:10769000D7108823D1F483EE9CE067ED7FE00E9451
:1076A000902540916E0550916F0560917005709125
:1076B000710583EE9CE00E94832287EB96E00E9496
:1076C0007CAF81E08093D7109DC0E0906E05F09074
:1076D0006F050091700510917105A0907E05B09026
:1076E0007F05C0908005D090810587EB96E00E94D1
:1076F00006AF29813A814B815C81A20EB31EC41E64
:10770000D51EA0E0B0E0A80EB91ECA1EDB1EEA140A
:10771000FB040C051D0508F475C081E08093D810AA
:107720008091DA10882309F06DC08091D9108823E8
:10773000C9F483EE9CE064EC7FE00E9490254091C8
:107740006E0550916F05609170057091710583EE23
:107750009CE00E94832287EB96E00E94C7AF81E005
:107760008093D91020906E0530906F054090700581
:107770005090710560907E0570907F058090800527
:107780009090810587EB96E00E9406AF7C0187EB25
:1077900096E00E940AAF5B016C0187EB96E00E94C5
:1077A00002AF29813A814B815C81260D371D481D2E
:1077B000591D2A0D3B1D4C1D5D1D00E010E02E0DD6
:1077C0003F1D401F511FA0E0B0E0280F391F4A1F86
:1077D0005B1F2216330644065506A0F011E01093F5
:1077E000DA101092DB1083EE9CE067EA7FE00E94E3
:1077F00031271093D21006C08091A104882309F08C
:1078000074CE82CE0F900F900F900F90CF91DF919A
:107810001F910F91FF90EF90DF90CF90BF90AF90AE
:107820009F908F907F906F905F904F903F902F90A0
:107830000895AF92BF92CF92DF92EF92FF920F9393
:107840001F93CF93DF938091D210882309F4C3C094
:10785000E0906E05F0906F05009170051091710534
:107860000E9469392091D2043091D3044091D4040C
:107870005091D504260F371F481F591F2E153F055D
:107880004007510708F4A7C078C0CA9CE001CB9C10
:10789000D00DDA9CD00D1124CE51DB4FCE010E94C9
:1078A0006E8602970CF455C06091D3107091D4107D
:1078B0006F5F7F4F882777FD8095982F0E946AD051
:1078C0007B018C01CE010E946E86BC01615070402C
:1078D000CE010E9404899B01AC01C801B7010E943E
:1078E0001AD11816B4F155C0EB0121968091E40C21
:1078F000882339F089E793E1BE014AE050E00E9415
:10790000A4C68091E50C882349F08091E60C909103
:10791000E70CBE014AE050E00E94A4C683EE9CE062
:107920006EE570E10E94902583EE9CE0B801A7010E
:107930000E94E61C83EE9CE06DE571E00E94F51A62
:10794000C801B7010E9437D0AB01BC018C2D0E9449
:10795000C92C0894C11CD11C83E0C816D10409F0BD
:1079600094CF8091D3109091D41001969093D4101D
:107970008093D3101092D2102EC083EE9CE068E862
:1079800070E10E943127CC24DD249CE2A92EB12C89
:107990007CCF6091D3107091D4106F5F7F4F882798
:1079A00077FD8095982F0E946AD0AB01BC01CE0173
:1079B0000E947A887B018C0183EE9CE06AE670E18C
:1079C0000E9490256091D3107091D4108091E30CA7
:1079D00084FD8ACFA3CFDF91CF911F910F91FF90AC
:1079E000EF90DF90CF90BF90AF9008950F931F93CB
:1079F000CF93DF93EC018B01888184FF13C08981D1
:107A0000882331F089E793E14AE050E00E9491C673
:107A10008A81882339F08B819C81B8014AE050E04B
:107A20000E9491C6DF91CF911F910F910895EF921F
:107A3000FF920F931F93CF93DF93182F80918305AD
:107A40008823E9F080917A0590917B05A0917C05CF
:107A5000B0917D05209176053091770540917805AC
:107A600050917905820F931FA41FB51F80937A054B
:107A700090937B05A0937C05B0937D05C3C083EEF6
:107A80009CE067E471E10E9490250E944296682F75
:107A900083EE9CE070E00E94F63C83EE9CE06BE39A
:107AA00071E10E9431271092DA041092D2101092E4
:107AB000D4101092D31010927A0510927B05109278
:107AC0007C0510927D051092830510927E05109220
:107AD0007F0510928005109281051092D5101092AA
:107AE000D6101092D7101092D8101092D910109270
:107AF000DA101092DB101092A4041092A304112348
:107B000061F41092CD041092CC041092C40410922F
:107B1000C5041092C6041092C7040E9469390E94DD
:107B2000BA39112311F40E94E3140E94429688236B
:107B300061F487EB96E00E94EEAE0E9469390E94E4
:107B4000BA3980E00E94C12741C081E00E94C1276C
:107B500000E010E02CE2E22EF12C0E9DE0010F9DE2
:107B6000D00D1E9DD00D1124CE51DB4FCE010E94B1
:107B70006E86181619062CF5CE0160E070E00E94A2
:107B8000048920E030E040E050E00E94CBCF882321
:107B900089F4CE0140E050E060E070E00E94568839
:107BA00020E030E04AE754E40E941ED1AB01BC0162
:107BB000C80105C0C80140E050E060E070E00E94EC
:107BC000A42D0F5F1F4F0330110539F610926E057B
:107BD00010926F0510927005109271050E9411C0ED
:107BE00060936605709367058093680590936905B7
:107BF0000E9411C060936A0570936B0580936C05B9
:107C000090936D0581E080938205109283058093A7
:107C1000C303DF91CF911F910F91FF90EF900895D3
:107C2000AF92BF92CF92DF92EF92FF920F931F938A
:107C30000E9411C05B016C0180916E0590916F05EF
:107C4000A0917005B09171050097A105B10541F4AF
:107C5000A092AF11B092B011C092B111D092B211F6
:107C600080918305882349F10E9411C020917205FB
:107C7000309173054091740550917505621B730B2B
:107C8000840B950B60937605709377058093780548
:107C90009093790583EE9CE065EF70E10E9490255A
:107CA000409176055091770560917805709179053E
:107CB00083EE9CE00E94832239C10E9411C0209172
:107CC0006605309167054091680550916905621B12
:107CD000730B840B950B20917A0530917B054091B5
:107CE0007C0550917D05621B730B840B950B609393
:107CF0006E0570936F0580937005909371050E94D7
:107D00001FC07B018C010E941FC06E197F09800B70
:107D1000910B645F714080409040A8F320916E0504
:107D200030916F0540917005509171058091D2049A
:107D30009091D304A091D404B091D50428173907A9
:107D40004A075B0740F58091D904882321F581E03B
:107D50008093D6048091AF119091B011A091B11190
:107D6000B091B211A6019501281B390B4A0B5B0B90
:107D7000DA01C901855F9140A040B04008F4D6C047
:107D80000E940B33A092AF11B092B011C092B1110A
:107D9000D092B211CBC08091A204882319F00E9426
:107DA000033302C00E94FC321092D6048091C303B8
:107DB000882351F00E944296823021F487EB96E0AE
:107DC0000E94C7AF1092C3030E944296882331F0ED
:107DD0008091D804882311F40E944B2F0E94429670
:107DE000823011F00E944D3A0E944296882331F46D
:107DF0008091D804882311F40E94193C0E94BA395A
:107E00009B01AC018091D904882361F48091D20454
:107E10009091D304A091D404B091D504280F391FB8
:107E20004A1F5B1F80916E0590916F05A0917005B0
:107E3000B0917105281739074A075B0708F076C02B
:107E40008091A604882329F183EE9CE06BED70E11C
:107E50000E94AD2581E08093D80480E090E040E06E
:107E600050E060E070E00E94A42D81E090E040E0EE
:107E700050E060E070E00E94A42D82E090E040E0DD
:107E800050E060E070E00E94A42D80E00E94C127D5
:107E90004DC083EE9CE067EC70E10E94AD250E942E
:107EA0005C158823F1F18091C8049091C904A091D8
:107EB000CA04B091CB0420916E0530916F054091BA
:107EC000700550917105820F931FA41FB51F8093F9
:107ED000C8049093C904A093CA04B093CB048091C2
:107EE000CC049091CD042091A3043091A404820F7E
:107EF000931F9093CD048093CC0481E00E941F33A4
:107F000081E08093D9040E94EC140E94CA2583EE7C
:107F10009CE068EA70E10E94AD2581E00E94173D77
:107F200005C00E946A3381E08093DA041F910F91AB
:107F3000FF90EF90DF90CF90BF90AF90089580E0DA
:107F40000E94173D0895CF92DF92EF92FF920F9318
:107F50001F93CF93DF9389E793E16DE172E10E9474
:107F60001AC589E793E16DE571E00E9468C789E76A
:107F700093E16BE072E10E941AC50E94BA39AB012D
:107F8000BC0189E793E12AE030E00E947DC689E7E1
:107F900093E16BEF71E10E941AC50E946939AB0150
:107FA000BC0189E793E12AE030E00E947DC689E7C1
:107FB00093E16EEE71E10E941AC50E941015BC019A
:107FC00089E793E14AE050E00E94A4C689E793E183
:107FD0006BED71E10E941AC50E942415AB01BC0132
:107FE00089E793E12AE030E00E947DC689E793E1CA
:107FF00068EC71E10E941AC50E94EA39BC0189E768
:1080000093E14AE050E00E94A4C689E793E169EB5E
:1080100071E10E941AC50E944296682F89E793E198
:108020004AE050E00E942DC689E793E166EA71E1DB
:108030000E941AC50E944386AB01BC0189E793E107
:108040002AE030E00E947DC6EE243CE2C32ED12C13
:1080500092C089E793E169E971E10E941AC589E755
:1080600093E16E2D4AE050E00E941BC689E793E140
:1080700061E971E10E945BC589E793E16DE571E01B
:108080000E9468C789E793E16FE771E10E945BC5D1
:10809000CC9D8001CD9D100DDC9D100D11240E5145
:1080A0001B4FFF240DC0C801BE010E940489AB0113
:1080B000BC0189E793E122E030E00E9454C7F394C9
:1080C000CF2DD0E0C8010E946E86C817D9075CF397
:1080D00089E793E16DE571E00E9468C789E793E164
:1080E0006DE671E10E945BC5FF240DC0C801BE01B1
:1080F0000E949E88AB01BC0189E793E122E030E059
:108100000E9454C7F394CF2DD0E0C8010E946E8620
:10811000C817D9075CF389E793E16DE571E00E9428
:1081200068C789E793E16AE571E10E945BC5FF24B6
:108130000DC0C801BE010E94AB86AB01BC0189E73E
:1081400093E122E030E00E9454C7F394CF2DD0E0B9
:10815000C8010E946E86C817D9075CF389E793E1CE
:108160006DE571E00E9468C789E793E16DE571E014
:108170000E9468C7E394CE2DD0E00E945F86C817A6
:10818000D9070CF466CFDF91CF911F910F91FF902B
:10819000EF90DF90CF9008958F929F92AF92BF9211
:1081A000CF92DF92EF92FF920F931F93CF93DF93C3
:1081B000843609F4F9C1853670F5803109F458C167
:1081C000813198F48C3009F4A9C08D3038F48A30AC
:1081D00009F452C08B3009F0F0C36CC08E3009F442
:1081E000F9C08F3008F028C1C7C0853109F4B5C186
:1081F000863138F4813109F494C1843109F0DDC34A
:10820000A4C1873109F4BDC1873108F4B0C18336F8
:1082100009F0D3C3C3C18B3609F4E5C28C3698F498
:10822000873609F436C2883638F4853609F4DCC15D
:10823000863609F0C2C3EEC1893609F490C28A3687
:1082400008F0ACC259C28B3709F411C38C3750F413
:10825000893709F4EEC28A3708F0FBC2883709F083
:10826000ACC3D1C2833809F440C3843809F466C36F
:10827000823809F0A2C315C384E596E00E9496B047
:108280007C01B701882777FD8095982F0E946AD0DE
:108290008B019C0185E06AE070E04AEC53E00E94AB
:1082A0000C2324E0E216F10408F0B1C1C7010E94DA
:1082B0005586ADC184E596E00E9496B0EC0197FD2D
:1082C0002AC00E945A862CE230E0829F8001839F60
:1082D000100D929F100D11240E511B4FC8010E94CA
:1082E0007686C8010E947E86C8010E94A786C801C2
:1082F000BE010E944E89BE01882777FD8095982F88
:108300000E946AD08B019C0185E06BE070E040EB3D
:1083100053E00E940C2381E0BE01C0C284E596E0D8
:108320000E94F2B06B017C010E945A862CE230E080
:10833000829F8001839F100D929F100D11240E517A
:108340001B4FC8010E9472865C01C801B701A601DB
:108350000E942889C801B5010E9404896B017C0133
:10836000C801B5010E9404898B019C0185E06CE085
:1083700070E04DE953E05BC084E596E00E94F2B006
:108380006B017C010E945A862CE230E0829F8001C2
:10839000839F100D929F100D11240E511B4FC80189
:1083A0000E947A865C01C801B701A6010E94C288BA
:1083B000C801B5010E949E886B017C01C801B5010E
:1083C0000E949E888B019C0185E06DE070E04AE888
:1083D00053E02DC084E596E00E94F2B06B017C0171
:1083E0000E945A862CE230E0829F8001839F100D0C
:1083F000929F100D11240E511B4FC8010E94A3869D
:108400005C01C801B701A6010E948286C801B501BE
:108410000E94AB866B017C01C801B5010E94AB864E
:108420008B019C0185E06EE070E047E753E00E941D
:108430000C23C701B60124C184E596E00E949EB0DA
:108440000E9464860E9469867C01BC0180E090E005
:108450000E9468D08B019C0185E06FE070E041E6EE
:1084600053E00E940C2381E0B7010E947E1CA5C24C
:108470000E945A867C018CE290E0E89EE001E99E31
:10848000D00DF89ED00D1124CE51DB4FCE010E94AD
:108490006E8602971CF1CE0160E070E00E949E881B
:1084A0002AEF31E0E29E8001E39E100DF29E100D56
:1084B00011240453194F0E9437D0AB01BC01C801ED
:1084C0000E940D96CE010E946E86BC0161507040E4
:1084D000CE010E949E880E9437D016C08AEF91E09C
:1084E000E89E8001E99E100DF89E100D11240453A2
:1084F000194FC8010E943596AB01BC01C8010E940A
:108500000D96C8010E943596AB01BC01C8010E94BE
:108510001D9685E060E170E04AE453E00E94BF24CC
:1085200039C084E596E00E94C2B00E943A860E945B
:1085300043866B017C010E946AD08B019C0185E01F
:1085400061E170E04BE253E0F3C10E949F3F85E0A0
:1085500064E170E04FE053E0E1CF85E065E170E079
:108560004CEF52E00E94BF240E946E3313C085E09E
:1085700066E170E048EE52E00E94BF240E946A3338
:1085800009C085E067E170E045ED52E00E94BF243C
:108590000E94183181E00E94B21C0FC281E00E944B
:1085A000B21C0E94A33F09C20E945A862CE230E00E
:1085B000AC01429FC001439F900D529F900D11242A
:1085C0008E519B4F0E946E867C01B701882777FDF4
:1085D0008095982F0E946AD08B019C0185E064E60B
:1085E00070E043EC52E011C00E9469867C01B70143
:1085F000882777FD8095982F0E946AD08B019C0177
:1086000085E065E670E046EA52E00E940C2381E0D6
:10861000B70144C184E596E00E94F2B07B018C0171
:108620000E945A866CE2C62ED12C9C012C9DC00162
:108630002D9D900D3C9D900D11248E519B4FB801A6
:10864000A7010E947A884B015C010E945A86AC0106
:108650004C9DC0014D9D900D5C9D900D11248E513F
:108660009B4FB801A7010E947A888B019C0185E08D
:1086700066E670E041E952E00E940C23C501B401B6
:1086800020E030E048EC52E40E941ED10E9437D036
:108690008FC184E596E00E94F2B06B017C010E94DC
:1086A0005A865CE2A52EB12C9C012A9DC0012B9D0F
:1086B000900D3A9D900D11248E519B4FB701A6014C
:1086C0000E9456888B019C0185E067E670E041E8D6
:1086D00052E00E940C230E945A86AC014A9DC001C0
:1086E0004B9D900D5A9D900D11248E519B4FB701BB
:1086F000A6010E945688C4CF84E596E00E94F2B09D
:108700006B017C010E945A864CE2A42EB12C9C0184
:108710002A9DC0012B9D900D3A9D900D11248E51E4
:108720009B4FB701A6010E9432888B019C0185E016
:1087300068E670E04FE652E00E940C230E945A86E1
:10874000AC014A9DC0014B9D900D5A9D900D112486
:108750008E519B4FB701A6010E94328891CF0E9493
:108760005A862CE230E0AC01429FC001439F900D3D
:10877000529F900D11248E519B4F0E94BB87F82E63
:10878000682F70E080E090E00E9468D08B019C012F
:1087900085E069E670E043E652E01EC00E945A861A
:1087A0002CE230E0AC01429FC001439F900D529FEC
:1087B000900D11248E519B4F0E944487F82E682FF4
:1087C00070E080E090E00E9468D08B019C0185E021
:1087D0006AE670E045E552E00E940C2381E06F2DCF
:1087E0000E94981CEAC00E9443860E946AD08B01B6
:1087F0009C0185E06BE670E040E452E00E940C23AF
:108800000E944386D5C00E941015AA2797FDA09507
:10881000BA2FBC01CD010E946AD08B019C0185E07A
:1088200068E770E044E352E00E940C230E941015B8
:1088300033C00E9424150E946AD08B019C0185E000
:1088400069E770E04EE152E00E940C230E9424157B
:10885000AFC00E94333A6B017C010E946AD08B0149
:108860009C0185E06AE770E047EF51E061C00E943B
:10887000EA39AA2797FDA095BA2FBC01CD010E9425
:108880006AD08B019C0185E06BE770E044EE51E01B
:108890000E940C230E94EA39BC0181E00E94641C02
:1088A0008CC084E596E00E9496B08C010E945A86A6
:1088B0002CE230E0AC01429FC001439F900D529FDB
:1088C000900D11248E519B4FB8010E9404890E9483
:1088D00037D06B017C010E946AD08B019C0185E03E
:1088E00062E870E04DEC51E023C084E596E00E9420
:1088F00096B08C010E945A862CE230E0AC01429F77
:10890000C001439F900D529F900D11248E519B4F9B
:10891000B8010E949E880E9437D06B017C010E94A2
:108920006AD08B019C0185E063E870E047EB51E081
:108930000E940C2381E0B701A6013DC084E596E0CA
:108940000E9496B05C010E945A860CE210E09C01E5
:10895000209FC001219F900D309F900D11248E51BA
:108960009B4FB5010E94AB866B017C010E945A8629
:10897000AC01409FC001419F900D509F900D11246C
:108980008E519B4FB5010E94AB868B019C0185E007
:1089900064E870E041EA51E00E940C23C701B6018F
:1089A0000E9437D024E630E040E050E00E94E6D15B
:1089B000AB01BC0181E00E942E1CDF91CF911F9181
:1089C0000F91FF90EF90DF90CF90BF90AF909F906E
:1089D0008F9008952F923F924F925F926F927F9265
:1089E0008F929F92AF92BF92CF92DF92EF92FF92BF
:1089F0000F931F93DF93CF93CDB7DEB762970FB678
:108A0000F894DEBF0FBECDBF87E090E00E9403B6B2
:108A100080E090E064EB73E00E94261982E090E031
:108A200069EA73E04AE00E94D8B519821A821B8273
:108A30001C821D821E821F82188619861A861B863A
:108A40001C861D861E861F86188A198A1A8A19EAAC
:108A5000A12E14E0B12ECC24DD24B2E2EB2EF12CB9
:108A6000A3E02A2E312C2C0E3D1EF7E04F2E512C68
:108A70004C0E5D1EEBE06E2E712C6C0E7D1E7FE0A9
:108A8000872E912C8C0E9D1E8AEF91E0C89E80014E
:108A9000C99E100DD89E100D11240453194FC80102
:108AA0000E94A8938983C8010E94DE931A828823BA
:108AB00011F091E09A83C8010E9435966B837C8304
:108AC0008D839E83C8010E9415966F83788789875E
:108AD0009A87C8010E9425966B877C878D879E8721
:108AE000F50181919191A191B1915F018F87988B4F
:108AF000A98BBA8B80E591E16C2D49810E94851686
:108B0000C701BE016F5F7F4F0E942219C701019606
:108B1000BE016E5F7F4F0E943519C7014097B101BA
:108B20000E943919C7010897B2010E943919C7017B
:108B30000497B3010E943919C7010C97B4010E9430
:108B400039190894C11CD11C88E190E0E80EF91E87
:108B500093E0C916D10409F097CF0AE510E0B801F7
:108B6000665D7E4EC8010E9401190F5F1F4F0936D6
:108B70001105A9F70E94591F0E94741962960FB639
:108B8000F894DEBF0FBECDBFCF91DF911F910F9143
:108B9000FF90EF90DF90CF90BF90AF909F908F901D
:108BA0007F906F905F904F903F902F9008950E941C
:108BB000C3B5882339F00E94A9B5079719F40E941C
:108BC000442A08950E94EA4408954F925F926F925A
:108BD0007F929F92AF92BF92CF92DF92EF92FF92DD
:108BE0000F931F93DF93CF9300D00F92CDB7DEB7D3
:108BF00000E010E03AEFE32E31E0F32E0E9DC001CD
:108C00000F9D900D1E9D900D11248453994F0E942D
:108C10004394882309F0B2C08091C104882309F0ED
:108C2000ADC0C2C0EE24FF242AEFA22E21E0B22E56
:108C30006E010894C11CD11C99249394EA9C800174
:108C4000EB9C100DFA9C100D11240453194FC80110
:108C50000E94DE93F601EE0DFF1D108281119082BD
:108C6000C80161E00E9421A10894E11CF11C83E08D
:108C7000E816F10419F79924EE24FF249AEF492EFF
:108C800091E0592E81E0682E712CE49C8001E59CD6
:108C9000100DF49C100D11240453194FC80160E00D
:108CA0000E9421A164E670E080E090E00E9445C04F
:108CB00089E20E94EEC0AA2797FDA095BA2FBC01B9
:108CC000CD010E946AD020E030EC4FE754E40E94CE
:108CD000CFCF20E030E040EA50E40E941ED15B019B
:108CE0006C010E949F1F9B01AC0166E676E686EE52
:108CF0009FE30E94CFCF9B01AC01C601B5010E944A
:108D00001AD1181644F4C3010E2C02C0880F991F03
:108D10000A94E2F7982AC80161E00E9421A183EE3B
:108D20009CE064E871E00E94AB2083EE9CE0B70118
:108D30000E94F63C83EE9CE06BE871E00E94AB2061
:108D400083EE9CE0B601A5010E94E61C0894E11C9C
:108D5000F11C83E0E816F10409F097CF8CEC96E063
:108D600069810E9421A186EC98E06A810E9421A17C
:108D700080EC9AE06B810E9421A102C008E0902E55
:108D8000892D0F900F900F90CF91DF911F910F9130
:108D9000FF90EF90DF90CF90BF90AF909F907F902B
:108DA0006F905F904F9008950F5F1F4F0330110534
:108DB00009F024CF37CFCF92DF92EF92FF920F933B
:108DC0001F93CF93DF9387EB96E00E94C7AF68EEC7
:108DD00073E080E090E00E9445C087EB96E00E943F
:108DE000C7AF68EE73E080E090E00E9445C0C0E04D
:108DF000D0E06AEFE62E61E0F62ECE9D8001CF9D99
:108E0000100DDE9D100D11240453194FC80161E0AF
:108E10000E94CF93C80161E00E9421A12196C33036
:108E2000D10559F70E94E545182F6AEF70E080E000
:108E300090E00E9445C0C0E0D0E0E12EFF245AEF50
:108E4000C52E51E0D52EC7010C2E02C095958795F1
:108E50000A94E2F780FF1CC0CC9D8001CD9D100DCF
:108E6000DC9D100D11240453194FC80160E00E94CD
:108E700021A16AEF70E080E090E00E9445C0C80147
:108E800061E00E9421A16AEF70E080E090E004C000
:108E900068EE73E080E090E00E9445C02196C33008
:108EA000D10589F68CEC96E060E00E9421A186EC69
:108EB00098E060E00E9421A180EC9AE060E00E94CE
:108EC00021A10E9411C0C0E0D0E04AEFE42E41E0B1
:108ED000F42ECE9D8001CF9D100DDE9D100D11242E
:108EE0000453194FC80140E050E06AE775E40E945E
:108EF000B894C80160E00E94F793C80160E020EEDA
:108F00003EE240E050E00E9427A82196C330D10500
:108F100001F70E94D02B8CEC96E00E9443948823AA
:108F2000D1F786EC98E00E9443948823A1F780EC67
:108F30009AE00E944394882371F78CEC96E061E0FC
:108F400020EE3EE240E050E00E9427A886EC98E048
:108F500061E020EE3EE240E050E00E9427A880EC75
:108F60009AE061E020EE3EE240E050E00E9427A857
:108F70000E94D02BDF91CF911F910F91FF90EF9026
:108F8000DF90CF9008954F925F926F927F928F9271
:108F90009F92AF92BF92CF92DF92EF92FF920F9388
:108FA0001F93DF93CF9300D00F92CDB7DEB7882EFB
:108FB000EE24FF24FAEFAF2EF1E0BF2E6E010894ED
:108FC000C11CD11C99249394EA9C8001EB9C100D48
:108FD000FA9C100D11240453194FC8010E94DE930E
:108FE000F601EE0DFF1D108281119082C80161E033
:108FF0000E9421A10894E11CF11C83E0E816F10411
:1090000019F783E0889E300111249924EAEF4E2E4F
:10901000E1E05E2E28C0E49C8001E59C100DF49CEC
:10902000100D11240453194FC80160E00E9421A1C2
:109030006BE470E080E090E00E9445C0C80161E010
:109040000E9421A1EA0CFB1C83E0E816F10421F444
:10905000B094A194B108B3940894C11CD11CC61457
:10906000D704CCF29394981440F471E0A72EB12C5D
:10907000CC24DD24EE24FF24F2CF8CEC96E0698131
:109080000E9421A186EC98E06A810E9421A180ECD7
:109090009AE06B810E9421A10F900F900F90CF91C9
:1090A000DF911F910F91FF90EF90DF90CF90BF90D5
:1090B000AF909F908F907F906F905F904F900895AA
:1090C000FF920F931F93CF93DF93F82E8B01C0E095
:1090D000D0E015C08F2D61E00E94A0C164E670E071
:1090E00080E090E00E9445C08F2D60E00E94A0C10A
:1090F00064E670E080E090E00E9445C02196C017D1
:10910000D10744F3DF91CF911F910F91FF90089504
:10911000FF920F931F93082F83EE9CE00E94A710ED
:10912000482F90E0202F30E082239323892B21F0D9
:10913000F02EF094F42202C0F42EF02A83EE9CE08C
:109140006F2D0E94B2100F2D10E0C801B4E096956B
:109150008795BA95E1F781700E9416AF169507952D
:1091600016950795802F81700E947DA08F2D1F91ED
:109170000F91FF900895CF92DF92EF92FF920F939D
:109180001F93CF93DF9386EB96E00E942693EE2405
:10919000FF2400E010E08AEFC82E81E0D82E0C9D5D
:1091A000E0010D9DD00D1C9DD00D1124C453D94F4D
:1091B000CE010E94D4938823B9F0E114F10469F040
:1091C000CE010E9474969701442737FD4095542F95
:1091D000621773078407950718F00115110521F42C
:1091E000CE010E9474967B010F5F1F4F0330110563
:1091F000B1F61E141F043CF58091A3049091A404C1
:10920000E816F90620F00E9442968230B1F40E94DE
:1092100042968230C1F49701442737FD4095542F80
:109220008091B5049091B604A091B704B091B804B0
:10923000281739074A075B0730F08AEB9CE061E0AA
:109240000E94A6AE02C00E941C31DF91CF911F91F7
:109250000F91FF90EF90DF90CF900895EF92FF92E3
:109260000F931F93CF93DF93EC017A018B018881D9
:1092700084FF14C08981882331F089E793E12AE0D3
:1092800030E00E94E7C58A81882341F08B819C8170
:10929000B801A7012AE030E00E94E7C5DF91CF9135
:1092A0001F910F91FF90EF9008950F931F930AEB7A
:1092B0001CE0C80161E047E758E70E94BDAEC80165
:1092C00062E04BEB58E40E94BDAEC80163E04BE3A3
:1092D00058E70E94BDAEC80164E046EC5BE20E9424
:1092E000BDAEC80165E040E859E40E94BDAEC801CA
:1092F00066E04EE558E30E94BDAE1F910F910895C0
:109300008AEB9CE060E00E94A6AE87EB96E00E94AC
:1093100044AF08952F923F924F925F926F927F9247
:109320008F929F92AF92BF92CF92DF92EF92FF9275
:109330000F931F93DF93CF93CDB7DEB7A2970FB6EE
:10934000F894DEBF0FBECDBF1C01498F5A8F6B8FC3
:109350007C8F8FEF90E0289E9001299E300D389EE3
:10936000300D1124285F314F3A832983F90180E0C1
:1093700090E020E030E040E050E0F8972083318337
:1093800042835383F8962083318342835383248F0F
:10939000358F468F578F019634968730910569F740
:1093A0008FEF90E0289EB001299E700D389E700DC1
:1093B00011246253724F6C517F4FDB012D933D930B
:1093C0004D935C9313976B5F7F4FDB012D913D9124
:1093D0004D915C912D8B3E8B4F8B588F695E704009
:1093E000FB01268F378F40A351A36F507F4FDB01C6
:1093F000ED90FD900D911D918D919D910D90BC91E1
:10940000A02D898B9A8BAB8BBC8BC801B7012989A6
:109410003A894B895C890E94CFCF6D877E878F8781
:10942000988BC801B7012D853E854F8558890E94CC
:109430001ED169877A878B879C87698D7A8D8B8D02
:109440009C8D2D893E894F89588D621B730B840B2F
:10945000950B97FF07C090958095709561957F4F0C
:109460008F4F9F4F0E946AD06D837E838F83988732
:10947000898D9A8DAB8DBC8D2D893E894F89588DF4
:10948000281739074A075B072CF04FEF5FEF5C8323
:109490004B8304C081E090E09C838B838FEF90E04E
:1094A000289E8001299E100D389E100D1124025314
:1094B000124F05501F4FD8018D909D90AD90BC90DC
:1094C0000B5F1040C501B40120E030E040EA50E4F9
:1094D0000E941AD118160CF027C1F801E851FF4F6D
:1094E0008081882329F460E070E080EA91EC04C078
:1094F00060E070E080EA91E4A50194010E941ED131
:109500002FE632E143E852E40E94CFCF6B017C01A9
:1095100029893A894B895C890E94CFCF2B013C0174
:10952000E89477F869897A898B899C8920E030E012
:1095300040E05FE30E941ED1A30192010E941ED170
:10954000A30192010E941ED16D8F7E8F8F8F98A3F1
:10955000EB81FC81BF01882777FD8095982F0E94C1
:109560006AD04B015C01C701B601A50194010E94BC
:109570001ED120E030E040E050E00E94CBCF8823B5
:10958000BCF58FEF90E0289E8001299E100D389E3B
:10959000100D11240253124FD80112964D925D9274
:1095A0006D927C9215970B501F4FC501B401F801C5
:1095B00020813181428153810E941ED10F59104078
:1095C000D8016D937D938D939C931397065510400E
:1095D000F801C2AED3AEE4AEF5AE6D817E818F816F
:1095E00098852D8D3E8D4F8D58A10E9467CF50C01C
:1095F0006D817E818F8198852D8D3E8D4F8D58A1F7
:109600000E94CBCF88230CF04BC08FEF90E0289EB8
:109610008001299E100D389E100D11240253124F07
:10962000D80112964D925D926D927C921597EB81C6
:10963000FC81F095E195FF4FFC83EB83BF01882708
:1096400077FD8095982F0E946AD00B501F4FD8014C
:109650002D913D914D915C910E941ED10F5910406A
:10966000F801608371838283938306551040D8018B
:10967000DA96CD92DD92ED92FC92DD976D8D7E8D26
:109680008F8D98A12D813E814F8158850E9466CF94
:109690006D837E838F839887B1E06B2E712C46C0DB
:1096A0006D817E818F8198852D8D3E8D4F8D58A146
:1096B0000E9467CF6D837E838F8398878FEF90E0C2
:1096C000289E6001299ED00C389ED00C1124EEEC0F
:1096D000FDE0CE0EDF1E6D897E898F89988D0E94F8
:1096E0006AD07B018C01C501B4012D8D3E8D4F8D5B
:1096F00058A10E941ED19B01AC01C801B7010E9474
:1097000066CF0E9437D0D6015E966D937D938D9380
:109710009C939197E4EEF0E0CE0EDF1ED6014D92C1
:109720005D926D927C921397662477246D817E8181
:109730008F81988529853A854B855C850E94CBCFA2
:1097400018163CF4BD85B9A3EE85EAA34F8458886A
:109750001AC08FEF90E0289EF001299EF00D389EF0
:10976000F00D1124ED53F14F6D817E818F8198852D
:1097700020813181428153810E94CFCF0E9485D1C7
:1097800069A37AA32C01F301EE0FFF1FEE0FFF1F59
:109790008FEF90E0289E7001299EF00C389EF00C0F
:1097A0001124EE0DFF1DE053F24F29A13AA1C9018A
:1097B000D20180839183A283B3832B813C81B90141
:1097C000882777FD8095982F0E946AD04B015C0115
:1097D0008301000F111F000F111F0E0D1F1D0C5DC7
:1097E000114FEEECCE2EEDE0DE2ECE0CDF1CF6019E
:1097F000EB50FF4F20813181428153810E941ED165
:10980000D8016D937D938D939C9313976D817E8189
:109810008F81988529853A854B855C850E941AD170
:109820001816ACF50894611C711C8301000F111F00
:10983000000F111F0E0D1F1D0053124F6D817E81F1
:109840008F81988529853A854B855C850E9466CFF6
:10985000F601EF50FF4F20813181428153810E94F8
:10986000CFCFF8016083718382839383F301EE0F7E
:10987000FF1FEE0FFF1FEE0DFF1DEC5DF14F80E0AF
:1098800090E0A0E0B0E080839183A283B38308944A
:10989000611C711CF301EE0FFF1FEE0FFF1F8FEF16
:1098A00090E0289E7001299EF00C389EF00C112447
:1098B000EE0DFF1DE053F24F29A13AA1C901D201DB
:1098C00080839183A283B3838301000F111F000F54
:1098D000111F0E0D1F1D0C5D114FF701ED53F14FC0
:1098E00020813181428153815058C501B4010E94C9
:1098F0001ED1D8016D937D938D939C93139730ED7A
:10990000432E3DE0532E4E0C5F1C21E0822E912C05
:10991000F201A080B180C280D380648D758D868D68
:10992000978D0E946AD07B018C01C601B501A98187
:10993000BA812D913D914D915C910E941ED19B0168
:10994000AC01C801B7010E9467CF7B018C01E9819E
:10995000FA81648D758D868D978D20E030E040E032
:109960005FE30E941ED1A60195010E941ED1A601AF
:1099700095010E941ED19B01AC01C801B7010E9454
:1099800067CF0E9437D0D20190966D937D938D93CF
:109990009C939397C601B501E981FA81248D358D99
:1099A000468D578D0E941ED19B01AC01A981BA81C1
:1099B0006D917D918D919C910E9467CFE981FA8193
:1099C00064837583868397830894811C911C24E0AB
:1099D00030E0420E531E3496FA83E983681479040A
:1099E0000CF096CFF3013196EE0FFF1FEE0FFF1F25
:1099F0008FEF90E0AC01249EC001259E900D349E17
:109A0000900D1124E80FF91FE253F24F298D3A8D82
:109A10004B8D5C8D268F378F40A351A38C010C5D3D
:109A2000114FEE24FF24D8016D917D918D919C9171
:109A300020E030E040E05FE30E941ED1F801619336
:109A40007193819391938F010894E11CF11C6E1422
:109A50007F044CF78FEF90E0289EF001299EF00DD7
:109A6000389EF00D1124E055F14F11821082A2961C
:109A70000FB6F894DEBF0FBECDBFCF91DF911F911F
:109A80000F91FF90EF90DF90CF90BF90AF909F909D
:109A90008F907F906F905F904F903F902F900895A0
:109AA000CF93DF93EC018FEF90E0C89FF001C99F47
:109AB000F00DD89FF00D1124E253F24FE351FF4F08
:109AC0004083518362837383B291A2919291829178
:109AD000481759076A077B07C1F0CE010E948A49DF
:109AE00081E090E0A0E0B0E00C2E04C0880F991F48
:109AF000AA1FBB1F0A94D2F72091C90D282B2093CF
:109B0000C90DCE0161E00E942134DF91CF9108950B
:109B10002F923F924F925F926F927F928F929F927D
:109B2000AF92BF92CF92DF92EF92FF920F931F936B
:109B3000DF93CF93CDB7DEB760970FB6F894DEBF53
:109B40000FBECDBF9A8789877C876B872801390133
:109B5000CD86DE86EF86F88A662757FD6095762FDC
:109B6000CB01BA010E946AD020E030E04AE754E419
:109B70000E94CFCF7B018C016D857E858F85988972
:109B80000E946AD06D837E838F8398872D853E8562
:109B90004F855889421A530A640A750AC301B201F3
:109BA0000E946AD09B01AC01C801B7010E941ED17E
:109BB0009B01AC016D817E818F8198850E9467CF6A
:109BC0000E9437D01B012C018D859E85AF85B889F9
:109BD000881A990AAA0ABB0AC501B4010E946AD070
:109BE0009B01AC01C801B7010E941ED19B01AC01D1
:109BF0006D817E818F8198850E9467CF0E9437D0CA
:109C000069837A838B839C838FEF90E0A985BA85E3
:109C1000A89FF001A99FF00DB89FF00D1124E858FE
:109C2000F14F20E030E080E090E0A0E0B0E0F89775
:109C300080839183A283B383F89680839183A283E8
:109C4000B383848F958FA68FB78F2F5F3F4F349646
:109C50002730310561F78FEF90E0E985FA85E89FBD
:109C60008001E99F100DF89F100D11240253124F2F
:109C70000E561F4FD8012D923D924D925C92139734
:109C8000EB85FC85BF01882777FD8095982F0E9482
:109C90006AD020E030E04AE754E40E94CFCF20E0D1
:109CA00030E040E05FE30E941ED16B017C010C516B
:109CB0001040D8016D937D938D939C931397065715
:109CC00010408EEA682E712C600E711E6D857E85A7
:109CD0008F85988962197309840995090E946AD051
:109CE000A70196010E94CFCFF30160837183828325
:109CF00093830A561F4F2D853E854F855889D8017D
:109D00002D933D934D935C9313970C511040F801A4
:109D1000C082D182E282F382085C1F4F69817A811E
:109D20008B819C81621B730B840B950B0E946AD004
:109D3000A70196010E94CFCF4B015C01D8016D9322
:109D40007D938D939C931397F30160817181828140
:109D5000938120E030E040E05FE30E941ED16B0180
:109D60007C01C201B1010E946AD0A70196010E9444
:109D700066CF0E9437D02B013C0104521040D8011D
:109D80006D937D938D939C9313970C51104080E0BD
:109D900090E0A0E8BFE3F80180839183A283B383BE
:109DA0000C5A1F4FF801C082D182E282F3820C521A
:109DB000104029813A814B815C81F80120833183F5
:109DC000428353830C511040F80180839183A28316
:109DD000B383085C1F4FD8018D929D92AD92BC92C7
:109DE0001397045E1F4FC501B40120E030E040E04E
:109DF0005FEB0E941ED1F80160837183828393839D
:109E00000453104069817A818B819C810E946AD0C1
:109E10006B017C01C501B40120E030E040E05FE36C
:109E20000E941ED19B01AC01C701B6010E9467CF01
:109E30000E9437D0D8016D937D938D939C93139797
:109E400089859A85B301A2010E94504D60960FB694
:109E5000F894DEBF0FBECDBFCF91DF911F910F9160
:109E6000FF90EF90DF90CF90BF90AF909F908F903A
:109E70007F906F905F904F903F902F9008950F9339
:109E80001F93CF93DF93062F853009F4BBC0863034
:109E900080F4823009F449C0833020F4813009F025
:109EA0001DC11AC0833009F462C0843009F016C1A4
:109EB0008AC08A3009F4E1C08B3038F4863009F466
:109EC000D2C0873009F00AC1D3C08C3009F4EBC08E
:109ED0008D3009F003C1ECC089E793E16BE971E0D3
:109EE0000E94B8C689E793E161E070E04AE050E083
:109EF0000E9491C689E793E16FE971E00E94B8C6BC
:109F000089E793E163E070E04AE050E00E9491C687
:109F100089E793E16FE971E00E94B8C689E793E1B0
:109F200061EA71E00E94B8C6D3C089E793E16AEAAA
:109F300071E00E94B8C610E0B8016F5F7F4F89E7FB
:109F400093E14AE050E00E9491C689E793E16FE90E
:109F500071E00E94B8C68FEF90E0089FF001099F62
:109F6000F00D189FF00D1124E554F14F21C089E741
:109F700093E16EEA71E00E94B8C610E0B8016F5F2D
:109F80007F4F89E793E14AE050E00E9491C689E75C
:109F900093E16FE971E00E94B8C68FEF90E0089FEF
:109FA000F001099FF00D189FF00D1124E954F14FB5
:109FB000408151816281738189E793E12AE030E039
:109FC0000E9441C685C089E793E162EB71E00E947F
:109FD000B8C6C0E0D0E08091C90D90E00C2E02C060
:109FE000959587950A94E2F780FD02C060E301C071
:109FF00061E389E793E10E943DC52196C330D10515
:10A0000051F766C089E793E166EB71E00E94B8C63C
:10A0100010E0B8016F5F7F4F89E793E14AE050E0BD
:10A020000E9491C689E793E16FE971E00E94B8C68A
:10A030008FEF90E0089FF001099FF00D189FF00D41
:10A040001124E154F14F60817181828193810E94DA
:10A050003CD09B01AC0189E793E1B9014AE050E0B3
:10A060000E940AC635C089E793E16AEB71E024C01B
:10A0700089E793E16EEB71E02FC089E793E163EC30
:10A0800071E00E94B8C66091CC0D7091CD0D89E74A
:10A0900093E14AE050E00E9491C689E793E167EAC4
:10A0A00071E00E94B8C689E793E167EC71E004C0F3
:10A0B00089E793E16BEC71E00E94B8C6602F70E015
:10A0C0006F5F7F4F89E793E14AE050E00E9491C6BD
:10A0D00089E793E167EA71E00E94B8C6DF91CF910A
:10A0E0001F910F910895CF93DF93EC018FEF90E0D4
:10A0F000C89FF001C99FF00DD89FF00D1124E954BD
:10A10000F14F80819181A281B38184179507A607C1
:10A11000B70729F0CE010E94504D82E001C083E0D4
:10A120006C2F0E943F4FDF91CF9108956F927F92E5
:10A130008F929F92AF92BF92CF92DF92EF92FF9257
:10A140000F931F93CF93DF931092CB0D10920A0DB4
:10A1500010920C0D10920B0D1092C50D1092C40DA3
:10A160008AE08093C60D1092C30D1092C70D8CE04B
:10A1700061E00E941DC1C0E0D0E08CE061E00E947F
:10A18000A0C162E370E080E090E00E9445C08CE0F6
:10A1900060E00E94A0C162E370E080E090E00E9475
:10A1A00045C02196CC30D10541F7E8EEFCE0119294
:10A1B0008DE0E830F807D9F7B097F093090DE093F8
:10A1C000080D81E063E171E141E050E00E9499BD3A
:10A1D0000EEC1DE027EBE22E2EE0F22E6801C0E02F
:10A1E000D0E09FEF692E712C0F2EF0E08F2EF0E063
:10A1F0009F2EF0E0AF2EF0E0BF2EF02DFE01E85BC9
:10A20000FB4F8081F6018083FE01E55BFB4F80817F
:10A21000F6018183FE01EB5BFB4F808161E00E94D0
:10A220001DC1CE0160E00E942134C69DF001C79D92
:10A23000F00DD69DF00D1124EA54F14F81E080839A
:10A24000F701108211821282138214821582168203
:10A250001782118A108A828A938AA48AB58ACE01CB
:10A2600068E873E10E94171121968FEF90E0C80E05
:10A27000D91EE80EF91EC330D10509F0BFCFF80191
:10A28000808161E00E941DC1F801818161E00E942E
:10A290001DC1F80180818A3029F4809180008A7F75
:10A2A0008093800001501F4FF0E10B3C1F0739F7EE
:10A2B0008091B60E60E0811161E08091CF0D0E9427
:10A2C000A0C18091B50F60E0811161E08091CE0E58
:10A2D0000E94A0C18091B41060E0811161E0809182
:10A2E000CD0F0E94A0C181E060E00E943F4F8EEE42
:10A2F00091E149E150E060E070E00E94987F8EEECD
:10A3000091E16EEE76E32FEF3FEF4FEF5FEF0E94AC
:10A31000AF7FDF91CF911F910F91FF90EF90DF9072
:10A32000CF90BF90AF909F908F907F906F90089547
:10A330002F923F924F925F926F927F928F929F9255
:10A34000AF92BF92CF92DF92EF92FF920F931F9343
:10A35000DF93CF93CDB7DEB72A970FB6F894DEBF61
:10A360000FBECDBF89E793E10E945CC81E821D82AB
:10A37000282F30E03A87298722242394A3C289E733
:10A3800093E10E9416C80E94C820882309F495C250
:10A39000F090110DFA948B3209F4A8C08C32A8F415
:10A3A0008F3109F47EC0803230F48A3019F18E3159
:10A3B00009F07DC2A7C0893209F4CBC08A3208F007
:10A3C000A8C0883209F073C253C08C3309F4D7C0D7
:10A3D0008D3330F48C3281F0823309F068C2AFC023
:10A3E000863409F4FCC1873409F449C28D3309F07D
:10A3F0005EC246C181E0ABC08091100D813009F092
:10A4000056C20F2D10E0C8010E94E912882309F4FA
:10A410004EC28FEF90E0089FF001099FF00D189F4A
:10A42000F00D1124E954F14F10821182128213822F
:10A43000C80140E050E060E070E00E94504DC8016B
:10A4400040E050E060E070E00E94735081E090E0F6
:10A45000A0E0B0E00F2C04C0880F991FAA1FBB1FFB
:10A460000A94D2F72091C80D282B2093C80D25C23D
:10A470008091100D823009F01AC28F2D90E00E9459
:10A48000E912882309F413C24091150D5091160D5D
:10A490006091170D7091180D8F2D90E00E947350F0
:10A4A0000CC28091100D823009F001C20F2D10E016
:10A4B000C8010E94E912882309F4F9C1AFEFB0E0A6
:10A4C0000A9FF0010B9FF00D1A9FF00D1124E95423
:10A4D000F14F8091150D9091160DA091170DB0912F
:10A4E000180D80839183A283B38327C08091100DC0
:10A4F000813009F0DCC18F2D90E00E94E9128823A1
:10A50000E1F4D5C18091100D882309F0D0C184E019
:10A510001EC08091100D813009F0C9C18F2D90E0CF
:10A520000E94E912882309F4C2C18F2D90E00E9495
:10A530004F1186E06F2D0E943F4F83E09CC18091B8
:10A54000100D882309F0B3C10E94DC1287E060E09F
:10A5500093C18091100D823009F0A9C18F2D90E038
:10A560000E94E912882309F4A2C16091150D70912F
:10A57000160D8F2D90E00E94171185E07CC180910F
:10A58000C90D882309F093C18091100D853008F41E
:10A590008EC1282F30E022503040C9018370907066
:10A5A000892B09F084C1E4EFF1E0F093CD0DE09345
:10A5B000CC0DC90164E070E00E9419D22B0180E04B
:10A5C00090E0A0E0B0E08093400E9093410EA09305
:10A5D000420EB093430E80933F0F9093400FA09391
:10A5E000410FB093420F80933E1090933F10A09381
:10A5F0004010B093411039E1632E3DE0732E188670
:10A600001F822EC0D3013C903A94832D90E00E948B
:10A61000E912882311F411E029C06091110D7091A5
:10A62000120D4091150D5091160DF3010481158105
:10A6300026813781C084D184E284F3848484958424
:10A64000A684B784832D90E00E94884D2F813885A1
:10A650002F5F3F4F38872F8380E190E0680E791E8F
:10A66000AF81B885A415B5056CF210E02092CB0D32
:10A670008AE060E00E943F4F112309F41EC117C118
:10A680008091C90D882309F012C18091100D882393
:10A6900009F00DC18091CB0D882309F408C100EBAE
:10A6A0001EE0CC24DD24F801E057F0406081718188
:10A6B0008281938120E030E040E050E00E94CBCFE7
:10A6C000882309F477C0EFEFF0E0CE9EC001CF9E63
:10A6D000900DDE9E900D1124BC01605C714FAC01A9
:10A6E0004053524F9C012858314FFC01E85FF14F15
:10A6F000EE24FF24DB018D909D90AD90BC90DA019B
:10A700008D929D92AD92BC921397DB015C968D90D9
:10A710009D90AD90BC905F97DA015C968D929D9272
:10A72000AD92BC925F97D9018D909D90AD90BC90F9
:10A73000139780829182A282B3825C968D909D90C5
:10A74000AD90BC905F97848E958EA68EB78E089440
:10A75000E11CF11C6C5F7F4F4C5F5F4F2C5F3F4FE4
:10A760003496B7E0EB16F10429F604541040F801D2
:10A7700080819181A281B3810C5B1F4FF801838797
:10A780009487A587B6871182108281E090E0A0E0CF
:10A79000B0E00C2C04C0880F991FAA1FBB1F0A949D
:10A7A000D2F72091C90D282B2093C90DC60161E075
:10A7B0000E9421340894C11CD11C01501F4FF3E0AA
:10A7C000CF16D10409F06FCF0E941A35F89427EE06
:10A7D00033E03093C50D2093C40D78946EC0809102
:10A7E000100D823009F063C00F2D10E0C8010E94E7
:10A7F000E912882309F45BC019821A821B821C8229
:10A800004091150D5091160D6091170D7091180D16
:10A81000C8019E012F5F3F4F0E94EF12882351F124
:10A820008091C90D90E00F2C02C0959587950A94F0
:10A83000E2F780FF18C08FEF90E0089FF001099FBA
:10A84000F00D189FF00D1124E554F14F29813A8144
:10A850004B815C8180819181A281B3812817390766
:10A860004A075B0739F049815A816B817C81C801B5
:10A870000E94504D8CE06F2D0E943F4F1EC0809172
:10A88000100D8230A1F48F2D90E00E94E9128823F0
:10A8900071F04091150D5091160D6091170D70914A
:10A8A000180D8F2D90E00E942D348DE0E4CF89E7C4
:10A8B00093E16FEC71E00E94B8C6AD81BE81119644
:10A8C000BE83AD83ED81FE8129853A85E217F307CA
:10A8D0000CF455CD2A960FB6F894DEBF0FBECDBF4F
:10A8E000CF91DF911F910F91FF90EF90DF90CF906C
:10A8F000BF90AF909F908F907F906F905F904F90A0
:10A900003F902F900895AF92BF92CF92DF92EF9237
:10A91000FF920F931F93DF93CF930F92CDB7DEB7C4
:10A9200000E010E063E2E62EF12C5E010894A11C29
:10A93000B11C5AEFC52E51E0D52E1982C701B501C1
:10A940000E94F1180C9DC0010D9D900D1C9D900D55
:10A9500011248453994F69810E9421A10F5F1F4FD9
:10A9600088E190E0E80EF91E0330110531F744E16B
:10A97000F42E8091C30D882311F40E941A350E9491
:10A9800098518091C60D8823A1F7F092C60D00E082
:10A9900010E0602F8091C90D90E0002E02C09595C7
:10A9A00087950A94E2F780FD0BC08091C80D90E076
:10A9B000002E02C0959587950A94E2F780FF03C0A8
:10A9C00083E00E943F4F0F5F1F4F0330110509F7CF
:10A9D0001092C80DCECF0F931F9309E713E1C80162
:10A9E0000E9463C864E670E080E090E00E9445C089
:10A9F000C80140E05BE460E070E00E9466C864E685
:10AA000070E080E090E00E9445C01F910F91089592
:10AA1000EF92FF920F931F93CF93DF930E9411C089
:10AA20006093BD047093BE048093BF049093C004F0
:10AA300081E08093C10400E010E0EAEFEE2EE1E057
:10AA4000FE2E0E9DE0010F9DD00D1E9DD00D1124F8
:10AA5000C453D94FCE010E94D493882321F0CE0154
:10AA600060E00E948F960F5F1F4F0330110549F77A
:10AA70008091C204813031F48CE060E00E94A0C17A
:10AA80001092C20486EB96E00E94EF92882329F090
:10AA90008AEB9CE061E00E94A6AEDF91CF911F910E
:10AAA0000F91FF90EF9008956F927F928F929F92F7
:10AAB000AF92BF92CF92DF92EF92FF920F931F93CC
:10AAC000DF93CF930F92CDB7DEB7682E7A0170E097
:10AAD000FB013297EB37F10510F00C949D5FE45BBE
:10AAE000FF4FEE0FFF1F0590F491E02D0994182FF2
:10AAF000115060E0FA018081811161E0812F0E9494
:10AB0000162A812F0E940D1D90E0A0E0B0E0BC014C
:10AB1000CD010E9468D08B019C01862D62E070E01F
:10AB20004CED59E023C090E001972AEF31E0829F7D
:10AB30008001839F100D929F100D11240453194F13
:10AB4000C801FA0160810E94CF93C8010E94D4938A
:10AB500090E0A0E0B0E0BC01CD010E9468D08B0184
:10AB60009C01862D63E070E04BEC59E00E940C23C1
:10AB700081E00E94B21C0C949D5F64E070E04CEB9D
:10AB800059E00E94BF24862D90E001972AEF31E022
:10AB9000AC01429FC001439F900D529F900D112424
:10ABA0008453994F0E940495109282050E94FC32B2
:10ABB000DFCF84E596E0BA010E949EB07C01862D2D
:10ABC00090E001972AEF31E0FC01E29FC001E39F92
:10ABD000900DF29F900D11248453994FB7010E945C
:10ABE000C99300E010E0C801B7010E9468D08B0152
:10ABF0009C01862D65E070E049EA59E0B7CFFA0183
:10AC000060816983082F10E0015010408AEF91E0C5
:10AC1000089F6001099FD00C189FD00C11240F5F72
:10AC20001F4F2CEC36E0C20ED31EC6010E9421AB92
:10AC3000C801880F991F800F911F23E0880F991F6B
:10AC40002A95E1F70A96BE016F5F7F4F0E94221995
:10AC5000043011053CF4662D615080E591E1498195
:10AC60000E948516698170E080E090E00E9468D0C3
:10AC70008B019C01862D66E070E044E959E00E945A
:10AC80000C2381E00E94B21C8981853018F4C60132
:10AC900060E005C0C6010E94DE93682FC6010E94D5
:10ACA000D8A00C949D5F84E596E0BA010E949EB006
:10ACB000BC01862D90E001972AEF31E0AC01429F64
:10ACC000C001439F900D529F900D11248453994FC2
:10ACD0000E949C94A0E0B0E0BC01CD010E9468D02D
:10ACE0008B019C01862D67E070E044E859E00E94EA
:10ACF0000C230E9474193CCFFA01F0806F2D70E094
:10AD000080E090E00E9468D08B019C01862D68E075
:10AD100070E040E759E00E940C23862D90E00197F7
:10AD20002AEF31E0AC01429FC001439F900D529F3A
:10AD3000900D11248453994F6F2D0E942BA118CF91
:10AD400069E070E04EE559E00E94BF24862D90E056
:10AD500001972AEF31E0FC01E29FC001E39F900DD3
:10AD6000F29F900D11248453994F0E94B39500CF08
:10AD7000E82EFF240894E108F1088AEF91E0E89EAC
:10AD80006001E99ED00CF89ED00C11242CEC36E02A
:10AD9000C20ED31EC6010E9435960E946AD08B0156
:10ADA0009C01862D6AE070E04BE459E00E940C2380
:10ADB000C6010E943596EE0CFF1CEE0CFF1C49EA02
:10ADC00054E0E40EF51EF701608371838283938360
:10ADD000CFCE6BE070E04BE359E00E94BF24862D9C
:10ADE00090E001972AEF31E0829F8001839F100D50
:10ADF000929F100D11240453194FC8010E945894BA
:10AE0000A0E0B0E0BC01CD010E9468D0AB01BC0164
:10AE1000C8010E94B894C80164E00E9421ABC80137
:10AE20000E941FA80E94D02BC80161E00E94F7A0D9
:10AE30009FCE6CE070E04CE259E00E94BF24862D6A
:10AE400090E001972AEF31E0829F8001839F100DEF
:10AE5000929F100D11240453194FC8010E94589459
:10AE6000A0E0B0E0BC01CD010E9468D0AB01BC0104
:10AE7000C8010E94B894C8010E94F0A7FAC084E5F6
:10AE800096E0BA010E94F2B06B017C018091E1046E
:10AE9000882331F40E94FC10882311F40C94725F13
:10AEA000C701B6010E9437D0882777FD8095982F7B
:10AEB0000E946AD08B019C01862D6DE070E043E119
:10AEC00059E00E940C23862D90E00197B701A6015E
:10AED0000E94A42D23C0C8010E945894A0E0B0E0B5
:10AEE000BC01CD010E9468D06B017C01C801B70193
:10AEF000A6010E94B894C701B6010E9437D08827E6
:10AF000077FD8095982F0E946AD08B019C01862D39
:10AF10006DE070E04DEF58E00E940C238091E10459
:10AF2000882311F00C949D5F0E94FC10882311F07F
:10AF30000C949D5F1DCE84E596E0BA010E94F2B0AC
:10AF4000AB01BC01862D90E001972AEF31E0FC01B6
:10AF5000E29FC001E39F900DF29F900D1124845356
:10AF6000994F0E9401948B019C01862D6EE070E048
:10AF700046EE58E00E940C230E94591FF9CDFA01B9
:10AF8000B0808091E1048823A1F1862D90E00197A3
:10AF90002AEF31E0829F8001839F100D929F100D58
:10AFA00011240453194FC8010E94E39320E030E0BC
:10AFB00040E85FE30E94CBCF8823DCF4C8010E9405
:10AFC000E39320E030E040E85FEB0E941AD11816CE
:10AFD00084F4F1E0BF1631F4C80140E050E060E2D3
:10AFE00071E405C0C80140E050E060E271EC0E94ED
:10AFF000B8940894E11CF11C84E596E0B7010E9426
:10B00000A6B06B017C010E9468D08B019C01862D4B
:10B010006FE070E044ED58E00E940C23C114D104AD
:10B02000E104F10491F4862D90E001972AEF31E0DC
:10B03000AC01429FC001439F900D529F900D11247F
:10B040008453994F61E00E94F793862D90E0019719
:10B050002AEF31E0FC01E29FC001E39F900DF29FD7
:10B06000900D11248453994F6B2DA70196010E94D6
:10B0700027A80E94D02B7CCD84E596E0BA010E94DF
:10B08000C2B07B018C01862D90E001972AEF31E060
:10B09000AC01429FC001439F900D529F900D11241F
:10B0A0008453994FB801A7010E940D96C801B701BA
:10B0B0000E946AD08B019C01862D60E170E044EC17
:10B0C00058E054CD84E596E0BA010E94C2B07B01FD
:10B0D0008C01862D90E001972AEF31E0FC01E29F80
:10B0E000C001E39F900DF29F900D11248453994F5E
:10B0F000B801A7010E941D96C801B7010E946AD03D
:10B100008B019C01862D61E170E045EB58E02ECD6E
:10B11000FA014081413081F490E001972AEF31E05B
:10B12000AC01429FC001439F900D529F900D11248E
:10B130008453994F61E011C0423091F490E001973F
:10B140002AEF31E0FC01E29FC001E39F900DF29FE6
:10B15000900D11248453994F62E00E94239515C0ED
:10B16000433081F490E001972AEF31E0AC01429F37
:10B17000C001439F900D529F900D11248453994F0D
:10B1800063E0EBCF80E00E94B21C862D90E0019737
:10B190002AEF31E0FC01E29FC001E39F900DF29F96
:10B1A000900D11248453994F0E94579590E0A0E090
:10B1B000B0E0BC01CD010E9468D08B019C01862DBE
:10B1C00062E170E04FE958E0D1CC90E001972AEFBE
:10B1D00031E0829F6001839FD00C929FD00C11249C
:10B1E0002CEC36E0C20ED31E84E596E0BA010E9434
:10B1F000A6B09B01AC01C601B9010E946996C601C7
:10B200000E9474960E9468D08B019C01862D63E198
:10B2100070E04DE858E00E940C2380919B04882345
:10B2200059F5C60160E070E00E947C9625C090E070
:10B2300001972AEF31E0829F8001839F100D929F3A
:10B24000100D11240453194F84E596E0BA010E94B1
:10B25000A6B0AB01BC01C8010E944596C8010E947E
:10B260004B960E9468D08B019C01862D64E170E0B2
:10B2700045E758E00E940C230E947F1D79CC90E0A6
:10B2800001972AEF31E0829F8001839F100D929FEA
:10B29000100D11240453194F84E596E0BA010E9461
:10B2A000A6B0AB01BC01C8010E945196C8010E9422
:10B2B00057960E9468D08B019C01862D65E170E055
:10B2C0004EE558E053CC90E001972AEF31E0829FA1
:10B2D0008001839F100D929F100D11240453194F6C
:10B2E00084E596E0BA010E94A6B0AB01BC01C8019A
:10B2F0000E945D96C8010E9463960E9468D08B01EF
:10B300009C01862D66E170E047E458E02FCC67E1B0
:10B3100070E046E358E00E94BF24862D81500E94D1
:10B32000142D26CC68E170E045E258E00E94BF246D
:10B33000862D81500E94CD2C1BCC90E001972AEFE6
:10B3400031E0829F8001839F100D929F100D112488
:10B350000453194F84E596E0BA010E94A6B09B0100
:10B36000AC01C801B9010E947C960E947F1DC801F2
:10B370000E9487960E9468D08B019C01862D69E10E
:10B3800070E042E158E0F2CB6BE170E04CEE57E048
:10B390000E94BF24062D10E0015010408AEF91E07A
:10B3A000089F7001099FF00C189FF00C11244CECC1
:10B3B00056E0E40EF51EC7010E94B395C70140E0B8
:10B3C00050E060E070E00E940596000F111F000F32
:10B3D000111F07551B4FF801108211821282138230
:10B3E000C70140E050E060E070E00E940D96C701A8
:10B3F00040E050E060E070E049C081500E94EB29DD
:10B40000F82E682F70E080E090E00E9468D08B01F9
:10B410009C01862D6CE170E043ED57E05CC56DE169
:10B4200070E040EC57E00E94BF24862D90E0019729
:10B430002AEF31E0829F8001839F100D929F100DB3
:10B4400011240453194FC8010E943596AB01BC0169
:10B45000C8010E940D968CCB6EE170E04EEA57E079
:10B460000E94BF24862D90E001972AEF31E0829F51
:10B470008001839F100D929F100D11240453194FCA
:10B48000C8010E943596AB01BC01C8010E941D96FF
:10B490006FCB84E596E0BA010E94C2B06B017C01DB
:10B4A0000E946AD08B019C01862D6FE170E041EA19
:10B4B00057E00E940C23862D8150B701A6010E94FF
:10B4C000C92C56CB84E596E0BA010E94C2B06B014C
:10B4D0007C010E946AD08B019C01862D60E270E0A5
:10B4E00043E857E00E940C23862D90E001972AEF55
:10B4F00031E0AC01429FC001439F900D529F900DDF
:10B5000011248453994FB701A6010E942D9630CB88
:10B5100084E596E0BA010E94C2B06B017C010E94F2
:10B520006AD08B019C01862D61E270E049E657E00C
:10B530000E940C23E62DF0E0EE0FFF1FEE0FFF1F21
:10B54000EB55FB4FC082D182E282F38211CB84E5BE
:10B5500096E0BA010E9496B07C01B701882777FD7A
:10B560008095982F0E946AD08B019C01862D68E2FD
:10B5700070E049E557E00E940C23862D90E001978A
:10B580002AEF31E0FC01E29FC001E39F900DF29FA2
:10B59000900D11248453994FB7010E94A4A031C487
:10B5A00084E596E0BA010E94F2B06B017C01862D21
:10B5B00069E270E041E457E0970186010E940C23A4
:10B5C000862D90E001972AEF31E0AC01429FC00147
:10B5D000439F900D529F900D11248453994FB701B2
:10B5E000A6010E9480A045C484E596E0BA010E94AD
:10B5F000F2B06B017C01862D6AE270E048E257E010
:10B60000970186010E940C23862D90E001972AEF76
:10B6100031E0FC01E29FC001E39F900DF29F900D8D
:10B6200011248453994FB701A6010E9492A021C40E
:10B63000FA01F0806F2D70E080E090E00E9468D009
:10B640008B019C01862D62E370E04DE057E00E9483
:10B650000C23F092E606F092E008F092DA0A6DC44C
:10B6600090E001972AEF31E0829F6001839FD00C28
:10B67000929FD00C11242CEC36E0C20ED31EF601A2
:10B68000828D882309F475CA0E9411C07B018C0148
:10B6900087EB96E00E94EEAEE61AF70A080B190B4C
:10B6A000E092CC10F092CD100093CE101093CF10FA
:10B6B00081E0F60184830E9408555ACA90E0019700
:10B6C0002AEF31E0829F6001839FD00C929FD00CC3
:10B6D00011242CEC36E0C20ED31EF601828D882395
:10B6E00009F447CAC6010E94749661157105810567
:10B6F000910509F41AC4E090A304F090A40400E0BA
:10B7000010E0C6010E947496E616F70608071907AE
:10B7100008F00BC40AC001979093A4048093A3047B
:10B72000C6010E9485A80E94D02B87EB96E00E945C
:10B73000EEAE3B014C0187EB96E00E940AAF5B0145
:10B740006C0187EB96E00E9406AF7C0187EB96E0E8
:10B750000E9402AF00E010E0A0E0B0E0E80EF91EA9
:10B760000A1F1B1FEA0CFB1C0C1D1D1DE614F70411
:10B770000805190538F487EB96E00E94EEAE8B01C0
:10B780009C011BC087EB96E00E940AAF6B017C0115
:10B7900087EB96E00E9406AF8C0187EB96E00E9453
:10B7A00002AF20E030E0A0E0B0E0080F191F2A1F30
:10B7B0003B1F0C0D1D1D2E1D3F1D8091B50490914A
:10B7C000B604A091B704B091B80480179107A207FE
:10B7D000B30768F0801B910BA20BB30B8093B504E9
:10B7E0009093B604A093B704B093B804C1C9109263
:10B7F000B5041092B6041092B7041092B804B8C9F8
:10B8000090E001972AEF31E0829F7001839FF00C56
:10B81000929FF00C11242CEC36E0E20EF31EC701CF
:10B820000E94D49390E0A0E0B0E0BC01CD010E9462
:10B8300068D08B019C01862D64E670E043E057E000
:10B840000E940C23C7010E94D4936CC290E0019720
:10B850002AEF31E0829F7001839FF00C929FF00CE1
:10B8600011244CEC56E0E40EF51EC7010E94C39370
:10B87000A0E0B0E0BC01CD010E9468D08B019C012A
:10B88000862D65E670E048EF56E00E940C23C70164
:10B890000E94C39370C090E001972AEF31E0829F2D
:10B8A0007001839FF00C929FF00C11248CEC96E0B9
:10B8B000E80EF91EC7010E94A89390E0A0E0B0E056
:10B8C000BC01CD010E9468D08B019C01862D66E6EB
:10B8D00070E04BEE56E00E940C23C7010E94A89333
:10B8E00021C290E001972AEF31E0829F7001839F8F
:10B8F000F00C929FF00C1124ECECF6E0EE0EFF1E23
:10B90000C7010E94B39390E0A0E0B0E0BC01CD017C
:10B910000E9468D08B019C01862D67E670E04FED98
:10B9200056E00E940C23C7010E94B393FBC190E034
:10B9300001972AEF31E0829F7001839FF00C929F64
:10B94000F00C11242CEC36E0E20EF31EC7010E942D
:10B950005894A0E0B0E0BC01CD010E9468D08B01FA
:10B960009C01862D68E670E043ED56E00E940C23B2
:10B97000C7010E945894BC0181E00E947E1CDDC278
:10B98000E82EFF24EE0CFF1CEE0CFF1C45EA54E0F1
:10B99000E40EF51EF70160817181828193810E941E
:10B9A0006AD08B019C01862D69E670E049EC56E077
:10B9B0000E940C23F701408151816281738112C181
:10B9C00090E001972AEF31E0829F7001839FF00C95
:10B9D000929FF00C11242CEC36E0E20EF31EC7010E
:10B9E0000E9435965B016C01C7010E94B0A08823BC
:10B9F000B9F0C7010E94AD938C01C7010E94A893C2
:10BA0000682FC80170E00E9419D29B01442737FDBE
:10BA10004095542FC601B5010E94E6D15B016C012F
:10BA2000C601B5010E946AD08B019C01862D6AE691
:10BA300070E04BEB56E00E940C2381E0B601A501BB
:10BA4000D2C090E001972AEF31E0829F7001839F7E
:10BA5000F00C929FF00C11244CEC56E0E40EF51E15
:10BA6000C7010E94439490E0A0E0B0E0BC01CD018A
:10BA70000E9468D08B019C01862D6BE670E04FEA36
:10BA800056E00E940C23C7010E9443944BC190E0F2
:10BA900001972AEF31E0829F7001839FF00C929F03
:10BAA000F00C11248CEC96E0E80EF91EC7010E9400
:10BAB000ED938B019C01862D6CE670E047EA56E021
:10BAC0000E940C23C7010E94ED931EC090E00197D5
:10BAD0002AEF31E0829F7001839FF00C929FF00C5F
:10BAE0001124ECECF6E0EE0EFF1EC7010E94359427
:10BAF0008B019C01862D6DE670E04FE956E00E94B7
:10BB00000C23C7010E94359420E030E048EC52E459
:10BB1000B6C190E001972AEF31E0829F7001839FC8
:10BB2000F00C929FF00C11242CEC36E0E20EF31E88
:10BB3000C7010E94579590E0A0E0B0E0BC01CD01A4
:10BB40000E9468D08B019C01862D6EE670E046E96C
:10BB500056E00E940C23C7010E945795E3C090E075
:10BB600001972AEF31E0829F7001839FF00C929F32
:10BB7000F00C11244CEC56E0E40EF51EC7010E94B7
:10BB800015960E946AD08B019C01862D6FE670E0AD
:10BB90004AE856E00E940C23C7010E94159620C077
:10BBA00090E001972AEF31E0829F7001839FF00CB3
:10BBB000929FF00C11248CEC96E0E80EF91EC70160
:10BBC0000E9425960E946AD08B019C01862D60E719
:10BBD00070E04FE756E00E940C23C7010E942596B3
:10BBE000AB01BC0181E00E942E1CA7C190E001972F
:10BBF0002AEF31E0829F7001839FF00C929FF00C3E
:10BC00001124ECECF6E0EE0EFF1EC7010E944B96ED
:10BC10000E9468D08B019C01862D61E770E04FE6A1
:10BC200056E00E940C23C7010E944B962CC190E065
:10BC300001972AEF31E0829F7001839FF00C929F61
:10BC4000F00C11242CEC36E0E20EF31EC7010E942A
:10BC500074960E9468D08B019C01862D62E770E08B
:10BC600045E656E00E940C23C7010E9474960BC162
:10BC700090E001972AEF31E0829F7001839FF00CE2
:10BC8000929FF00C11244CEC56E0E40EF51EC70117
:10BC90000E9457960E9468D08B019C01862D63E715
:10BCA00070E04EE456E00E940C23C7010E945796B4
:10BCB000EAC090E001972AEF31E0829F7001839FF4
:10BCC000F00C929FF00C11248CEC96E0E80EF91E1B
:10BCD000C7010E9463960E9468D08B019C01862D4B
:10BCE00064E770E047E356E00E940C23C7010E941E
:10BCF0006396C9C0F82EFA948F2D0E940D1D90E016
:10BD0000A0E0B0E0BC01CD010E9468D08B019C0195
:10BD1000862D65E770E04FE256E00E940C238F2DE0
:10BD20000E940D1D682F81E0DAC0815060E00E9402
:10BD30005828F82E882311F0FF24F3946F2D70E01B
:10BD400080E090E00E9468D08B019C01862D66E720
:10BD500070E04AE156E0BFC090E001972AEF31E081
:10BD6000829F7001839FF00C929FF00C1124ECECE9
:10BD7000F6E0EE0EFF1EC7010E9487960E9468D073
:10BD80008B019C01862D67E770E04FE056E00E9432
:10BD90000C23C7010E94879676C0815061E00E9403
:10BDA0009B29F82E682F70E080E090E00E9468D018
:10BDB0008B019C01862D68E770E042EF55E08BC057
:10BDC00090E001972AEF31E0AC01429FC001439F10
:10BDD000900D529F900D11248453994F0E94AAA058
:10BDE0007C01B701882777FD8095982F0E946AD043
:10BDF0008B019C01862D69E770E046EE55E00E94BC
:10BE00000C2381E0B7010E94641C97C090E0019769
:10BE10002AEF31E0FC01E29FC001E39F900DF29F09
:10BE2000900D11248453994F0E9488A06B017C01CE
:10BE3000862D6AE770E046ED55E017C090E0019767
:10BE40002AEF31E0AC01429FC001439F900D529F09
:10BE5000900D11248453994F0E949AA06B017C018C
:10BE6000862D6BE770E045EC55E0970186010E9456
:10BE70000C23C701B60120E034E244E759E40E94F4
:10BE80001ED10E943CD0AB01BC0181E00E94491C44
:10BE900054C090E001972AEF31E0FC01E29FC0011D
:10BEA000E39F900DF29F900D11248453994F0E94AF
:10BEB000B0A0F82E882311F0FF24F3946F2D70E0CA
:10BEC00080E090E00E9468D08B019C01862D6CE799
:10BED00070E047EB55E00E940C2381E06F2D0E943B
:10BEE000981C2BC0862D90E001972AEF31E0829FAD
:10BEF0008001839F100D929F100D11240453194F40
:10BF0000C8010E945894A0E0B0E0BC01CD010E949D
:10BF100068D09B01AC01C701B6010E941AD1181666
:10BF200014F00C9476570C946B578091A304909165
:10BF3000A404009709F0EFCBF3CB0F90CF91DF91E2
:10BF40001F910F91FF90EF90DF90CF90BF90AF9037
:10BF50009F908F907F906F9008953F924F925F9245
:10BF60006F927F928F929F92AF92BF92CF92DF9209
:10BF7000EF92FF920F931F93DF93CF93CDB7DEB76E
:10BF8000CD54D0400FB6F894DEBF0FBECDBF309079
:10BF9000D7041092D7048091C104882309F0DBC034
:10BFA000332009F0D8C00E94E3141092DA041092F2
:10BFB000C4041092C5041092C6041092C7040E94D3
:10BFC000183100E010E02AEFE22E21E0F22E0E946C
:10BFD000FC10882319F4802F0E94EB2983EE9CE04B
:10BFE00063E47FE00E9490250E9DC0010F9D900D9F
:10BFF0001E9D900D11248453994F0E94A893682F81
:10C0000083EE9CE00E94B71F0F5F1F4F03301105A6
:10C01000F1F60E944296882309F081C087EB96E0F2
:10C020000E94EEAE7B018C0187EB96E00E940AAF86
:10C030003B014C0187EB96E00E9402AF5C0187EB6D
:10C0400096E00E9406AFE618F70808091909CC2403
:10C05000DD24EA18FB080C091D09A0E0B0E0E81A8D
:10C06000F90A0A0B1B0BC801B7010E9468D020E037
:10C0700030E04AE754E40E94CFCF5B016C0120E03E
:10C0800030E040E05FE30E941AD1181654F40F2EFE
:10C09000F0E0AF2EF0E0BF2EF0E0CF2EFFE3DF2E7A
:10C0A000F02D662477249AEF492E91E0592E649C56
:10C0B0004001659C900C749C900C11248CEC96E0D3
:10C0C000880E991EC4010E944F9F0E9437D09B0189
:10C0D00091E0243F3907E4F4B901882777FD809582
:10C0E000982F0E946AD07B018C01C601B50120E027
:10C0F00030E040E05FE30E941ED19B01AC01C8012B
:10C10000B7010E94CFCFAB01BC01C4010E94B8941B
:10C110000894611C711C83E06816710441F60E944A
:10C1200042968230C1F487EB96E00E94C7AF0E942E
:10C1300011C07B018C010E9411C06E197F09800B18
:10C14000910B0E9468D020E030E84BEB54E40E9451
:10C15000CBCF87FDF0CF8091C104882309F074C153
:10C160008E010F5F1F4FC80164E871E00E9446C94D
:10C1700088E0E82EF12CEC0EFD1EC701B8010E94EC
:10C180003FCAC7016DED71E00E94F3C8BC018E018A
:10C19000015F1F4FC8010E943FCA83EE9CE0B801B7
:10C1A0000E943B28C8010E9450CAC7010E9450CA81
:10C1B000AA24BB240AEF802E01E0902EA89C6001E7
:10C1C000A99CD00CB89CD00C11248CEC96E0C80E25
:10C1D000D91EC6010E9425967B018C01C6010E94D2
:10C1E0003596E61AF70A080B190B83EE9CE0B801A6
:10C1F000A7010E945C220894A11CB11C93E0A9161F
:10C20000B104E1F616E1E12EF12CEC0EFD1EC701A2
:10C21000BE016F5F7F4F0E943FCAC70164EE71E0AD
:10C220000E94F3C8BC018E01035E1F4FC8010E942B
:10C230003FCA83EE9CE0B8010E943B28C8010E94DF
:10C2400050CAC7010E9450CA00E010E0BAEFEB2EBE
:10C25000B1E0FB2E0E9DC0010F9D900D1E9D900D17
:10C2600011248453994F0E941596AB01BC0183EEB3
:10C270009CE00E945C220F5F1F4F0330110551F7B5
:10C28000A4E2EA2EF12CEC0EFD1EC701BE016F5F89
:10C290007F4F0E943FCAC7016BEE71E00E94F3C856
:10C2A000BC018E01055D1F4FC8010E943FCA83EE8D
:10C2B0009CE0B8010E943B28C8010E9450CAC701F7
:10C2C0000E9450CA00E010E0FAEFEF2EF1E0FF2EDE
:10C2D0000E9DC0010F9D900D1E9D900D1124845345
:10C2E000994F0E942596AB01BC0183EE9CE00E9411
:10C2F0005C220F5F1F4F0330110551F7E2E3EE2E72
:10C30000F12CEC0EFD1EC701BE016F5F7F4F0E9436
:10C310003FCAC70161EF71E00E94F3C8BC018E0102
:10C32000075C1F4FC8010E943FCA83EE9CE0B80122
:10C330000E943B28C8010E9450CAC7010E9450CAEF
:10C3400000E010E07AEFE72E71E0F72E0E9DC001BD
:10C350000F9D900D1E9D900D11248453994F0E94A6
:10C360003596AB01BC0183EE9CE00E945C220F5F1E
:10C370001F4F0330110551F760E4E62EF12CEC0E4F
:10C38000FD1EC701BE016F5F7F4F0E943FCAC701FC
:10C390006AEF71E00E94F3C8BC018E01095B1F4F78
:10C3A000C8010E943FCA83EE9CE0B8010E943B286E
:10C3B000C8010E9450CAC7010E9450CA00E010E0A4
:10C3C0005AEFE52E51E0F52E0E9DC0010F9D900D08
:10C3D0001E9D900D11248453994F0E944B96AB01E2
:10C3E000BC0183EE9CE00E9483220F5F1F4F03304D
:10C3F000110551F7332011F10E9442968823F1F084
:10C40000EE24FF244AEFC42E41E0D42EEC9C8001A0
:10C41000ED9C100DFC9C100D11240453194FC80104
:10C420000E94D493882319F0C8010E942DA8089473
:10C43000E11CF11C83E0E816F10441F70E94085565
:10C44000CE0101960E944ACAC35BDF4F0FB6F89433
:10C45000DEBF0FBECDBFCF91DF911F910F91FF9037
:10C46000EF90DF90CF90BF90AF909F908F907F9094
:10C470006F905F904F903F9008952F923F924F9210
:10C480005F926F927F928F929F92AF92BF92CF9264
:10C49000DF92EF92FF920F931F93DF93CF93CDB76D
:10C4A000DEB72A970FB6F894DEBF0FBECDBF9A87CE
:10C4B0008987DC01DB963C90DB97DD968C90DD97DD
:10C4C000AF5BBF4F9C90A154B040DA96AC90DA9726
:10C4D000DC96DC90DC97AE5BBF4F2C9012976C9192
:10C4E000A054B040BA87A98770E080E090E024E6CD
:10C4F00030E040E050E00E94E6D12B013C01E985AC
:10C50000FA8561AD70E080E090E028EE33E040E035
:10C5100050E00E94E6D1460E571E681E791EA9857E
:10C52000BA85D7968C91D797282F30E0D8968C91E2
:10C53000F901E80FF11DE536F1056CF080E090E0BF
:10C54000A0E0B0E08D839E83AF83B88789839A8310
:10C55000AB83BC8315C0B901882777FD8095982FE0
:10C560000E946AD020E030E048EC52E40E94CFCF35
:10C570006D837E838F83988769837A838B839C8383
:10C58000A985BA85D6966C9170E080E090E020E1B4
:10C590003EE040E050E00E94E6D17B018C01E9855D
:10C5A000FA8565A970E080E090E02CE330E040E09F
:10C5B00050E00E94E6D1E60EF71E081F191FC801C1
:10C5C000B70128EE33E040E050E00E94E6D1A985B3
:10C5D000BA8552966D937D938D939C935597DE9675
:10C5E0006C9170E080E090E020E63AEE40E050E0B0
:10C5F0000E94E6D1E985FA85668B778B808F918FD3
:10C6000067AD70E080E090E00E94E6D1A985BA8530
:10C610005A966D937D938D939C935D9780E00E94D5
:10C62000571587EB96E0B301A2010E94E8AE6A2D90
:10C6300070E080E090E024E630E040E050E00E94CE
:10C64000E6D17B018C01692D70E080E090E028EE5E
:10C6500033E040E050E00E94E6D1E60EF71E081FEE
:10C66000191F87EB96E0B7010E94F4AE682D70E0C9
:10C6700080E090E024E630E040E050E00E94E6D127
:10C680007B018C01632D70E080E090E028EE33E0C8
:10C6900040E050E00E94E6D1E60EF71E081F191F89
:10C6A00087EB96E0B801A7010E94F8AE622D70E01A
:10C6B00080E090E024E630E040E050E00E94E6D1E7
:10C6C0007B018C016D2D70E080E090E028EE33E07E
:10C6D00040E050E00E94E6D1E60EF71E081F191F49
:10C6E00087EB96E0B7010E94FEAE22243324EAEFE6
:10C6F000F1E02E9E40012F9E900C3E9E900C112446
:10C700004CEC56E0840E951EC4010E945C95C40159
:10C7100062E00E942395A985BA85D4968C910E94E7
:10C720003F96E985FA8566897789808D918DA30189
:10C7300092010E942CD2C401B9010E946996A98578
:10C74000BA855A966D917D918D919C915D97A301CB
:10C7500092010E942CD2C401B9010E947C96E98505
:10C76000FA8584A9882361F562897389848995890A
:10C77000A30192010E942CD279018A01C801B7015C
:10C780000E9468D09B01AC016D817E818F8198856C
:10C790000E941ED10E943CD05B016C01C401B60115
:10C7A000A5010E945196C401B601A5010E945D96A3
:10C7B000C401B801A7010E9445960E947F1D3BC09D
:10C7C000A985BA8552966D917D918D919C915597D1
:10C7D0000E9468D09B01AC016D817E818F8198851C
:10C7E0000E941ED10E943CD0AB01BC01C4010E943A
:10C7F0005196E985FA8562897389848995890E94B1
:10C8000068D09B01AC0169817A818B819C810E94F7
:10C810001ED10E943CD0AB01BC01C4010E945D96B8
:10C82000A985BA8552964D915D916D917C915597F0
:10C83000C4010E944596C4010E94F3A80894211CDB
:10C84000311CB3E02B16310409F051CF0E9411C006
:10C85000E985FA8566877787808B918B81E0828373
:10C860000E94AD5F2A960FB6F894DEBF0FBECDBF13
:10C87000CF91DF911F910F91FF90EF90DF90CF90BC
:10C88000BF90AF909F908F907F906F905F904F90F0
:10C890003F902F9008954F925F926F927F928F9268
:10C8A0009F92AF92BF92CF92DF92EF92FF920F933F
:10C8B0001F93DF93CF93CDB7DEB729970FB6F894C8
:10C8C000DEBF0FBECDBF4C01DC0119968C918823D1
:10C8D00029F40E945415813009F4CEC40E946215D7
:10C8E000882309F0C9C493C480E091E10E9428160E
:10C8F00090E0A0E0B0E0BC01CD010E9468D0AB01A7
:10C90000BC01C4010E943C166E837F83888799878F
:10C9100080E091E10E942D1690E0A0E0B0E0BC0123
:10C92000CD010E9468D0AB01BC01C4010E943C163D
:10C930006A837B838C839D8380E091E10E94321621
:10C9400090E0A0E0B0E0BC01CD010E9468D0AB0156
:10C95000BC01C4010E943C162B013C016E817F8109
:10C960008885998520E030E040E053E40E941AD1A8
:10C97000181624F4F401838187FF11C06E817F8132
:10C980008885998520E030E040E053E40E94CBCFD9
:10C99000882344F4D40113968C91813818F083E0F5
:10C9A000F4018683D40116968C911697882359F04A
:10C9B000815016968C9380E090E0A0E0B3E48E83E3
:10C9C0009F83A887B9876A817B818C819D8120E0C4
:10C9D00030E040E053E40E941AD118162CF4D40140
:10C9E00014968C9187FF10C06A817B818C819D8118
:10C9F00020E030E040E053E40E94CBCF882344F4B1
:10CA0000F4018481813820F083E0D40117968C935F
:10CA1000F4018781882351F08150878380E090E082
:10CA2000A0E0B3E48A839B83AC83BD83C301B201DE
:10CA300020E030E040E053E40E941AD118162CF4B4
:10CA4000D40115968C9187FF0EC0C301B20120E07E
:10CA500030E040E053E40E94CBCF882344F4F4015B
:10CA60008581813820F083E0D40118968C93F401FD
:10CA70008085882361F0815080870F2EF0E04F2E53
:10CA8000F0E05F2EF0E06F2EF3E47F2EF02D6E814C
:10CA90007F818885998520E030E040E053E40E9462
:10CAA000CBCF8823B1F46A817B818C819D8120E08A
:10CAB00030E040E053E40E94CBCF882351F4C3011F
:10CAC000B20120E030E040E053E40E94CBCF882365
:10CAD00059F0D40119968C911997882329F481E093
:10CAE00019968C930E94C127F401638170E0882716
:10CAF00077FD8095982F0E946AD09B01AC016E81D2
:10CB00007F81888599850E94CBCF882399F1D401B4
:10CB100092961C9292978CEC96E01B966C910E94D8
:10CB200021AB8CEC96E00E9458947C016E817F8151
:10CB30008885998520E030E040E053E40E9466CF8C
:10CB400020E030E040E05CE30E941ED15B016C011C
:10CB500000E010E0C801B7010E9468D09B01AC0161
:10CB6000C601B5010E941ED1AB01BC0180E090E07E
:10CB70000E94A42DF401648170E0882777FD8095E0
:10CB8000982F0E946AD09B01AC016A817B818C81C5
:10CB90009D810E94CBCF8823C1F1D4011A968C913C
:10CBA0001A97823090F592961C92929786EC98E0B4
:10CBB0001C966C910E9421AB86EC98E00E945894E0
:10CBC0007C016A817B818C819D8120E030E040E0A6
:10CBD00053E40E9466CF20E030E040E05CEB0E942E
:10CBE0001ED15B016C0100E010E0C801B7010E949A
:10CBF00068D09B01AC01C601B5010E941ED1AB01FA
:10CC0000BC0181E090E00E94A42DF401658170E0F8
:10CC1000882777FD8095982F0E946AD09B01AC01F0
:10CC2000C301B2010E94CBCF8823A9F1D4011A9687
:10CC30008C91823011F0882371F5F40112A280ECFE
:10CC40009AE065850E9421AB80EC9AE00E9458949E
:10CC50007C01C301B20120E030E040E053E40E94D7
:10CC600066CF20E030E040E05CEB0E941ED15B012B
:10CC70006C0100E010E0C801B7010E9468D09B0180
:10CC8000AC01C601B5010E941ED1AB01BC0182E01E
:10CC900090E00E94A42D6E817F81888599850E94F5
:10CCA0003CD0D40113966C936A817B818C819D81E9
:10CCB0000E943CD0F4016483C301B2010E943CD0C5
:10CCC000D40115966C9380E091E161E00E949C157F
:10CCD000A82E80E091E161E00E94FA15882309F412
:10CCE0009DC280E091E168E00E94FA15833009F06E
:10CCF00095C282E0F40180830E94892D81E0D401F5
:10CD000092968C93B9C28981882339F5C40160E970
:10CD100071E04AE050E021E00E948A16EE24FF24F0
:10CD20007AEFC72E71E0D72EEC9C8001ED9C100DA0
:10CD3000FC9C100D11240453194FC8010E94359614
:10CD4000AB01BC01C8010E940D960894E11CF11CC6
:10CD5000B3E0EB16F10441F703C08150F40186AF54
:10CD600080E091E161E00E94FA15882309F46AC22B
:10CD700080E091E166E00E94FA15833009F062C21A
:10CD800082E0D4018C930E94F92C76C28981882399
:10CD900039F5C40160E971E04AE050E021E00E9409
:10CDA0008A16EE24FF246AEFC62E61E0D62EEC9C94
:10CDB0008001ED9C100DFC9C100D11240453194FA3
:10CDC000C8010E943596AB01BC01C8010E941D96A6
:10CDD0000894E11CF11CB3E0EB16F10441F703C029
:10CDE0008150F40187AFD4011A960C91C4016A2DC9
:10CDF00043E09E012F5F3F4F10E054EFE52E51E0DE
:10CE0000F52ECC24C3940E94F6168823B9F099819C
:10CE10009130A1F4F4018285813049F0813018F01D
:10CE2000823061F408C0D4011A969C9307C082E056
:10CE3000F401828703C0D4011A961C92F40105A95B
:10CE4000C4016A2D4CE09E012F5F3F4F10E0B4EF0C
:10CE5000EB2EB1E0FB2ECC24CA940E94F616882358
:10CE600021F08981D401D5968C93F40106A9C401DF
:10CE70006A2D4AE09E012F5F3F4F10E0A4EFEA2E9B
:10CE8000A1E0FA2ECC24CA940E94F616882321F041
:10CE90008981D401D6968C93F40107A9C4016A2D27
:10CEA0004BE09E012F5F3F4F10E0F4EFEF2EF1E0DB
:10CEB000FF2EE4E6CE2E0E94F616882321F089810B
:10CEC000D401D7968C93F40100ADC4016A2D49E0DA
:10CED0009E012F5F3F4F10E074EFE72E71E0F72EB9
:10CEE00054E6C52E0E94F616882321F08981D401CC
:10CEF000D8968C93F40101ADC4016A2D4FE09E01D8
:10CF00002F5F3F4F10E0B4EFEB2EB1E0FB2ECC24AF
:10CF1000CA940E94F616882321F08981D401D996FB
:10CF20008C93F40102ADC4016A2D4EE09E012F5F87
:10CF30003F4F10E0A4EFEA2EA1E0FA2EFAE0CF2E48
:10CF40000E94F616882321F08981D401DA968C9309
:10CF5000F40103ADC4016A2D40E19E012F5F3F4FF4
:10CF600010E0E4EFEE2EE1E0FE2ECC24CA940E9405
:10CF7000F616882321F08981D401DB968C93F40185
:10CF800005ADC4016A2D4DE09E012F5F3F4F10E0BB
:10CF900074EFE72E71E0F72E5AE0C52E0E94F616C8
:10CFA000882321F08981D401DD968C93C4016A2DF8
:10CFB00047E09E012F5F3F4F00E010E0B8EEEB2E00
:10CFC000B3E0FB2EA3E0CA2E0E94F616882339F0A8
:10CFD00069816150633018F4C4010E940519C401CD
:10CFE0006A2D45E09E012F5F3F4F00E010E0F8EE14
:10CFF000EF2EF3E0FF2EE3E0CE2E0E94F6168823FC
:10D0000039F069816150633018F4C4010E94831AB9
:10D0100080E091E161E10E949C15833091F490E001
:10D02000F40184A9882309F491E0D401D4969C9357
:10D0300040E0992309F441E080E091E162E00E9440
:10D04000601A80E091E161E10E949C15833091F4C7
:10D0500090E0F40184A9882309F491E0D401D496E6
:10D060009C9340E0992309F441E080E091E162E083
:10D070000E94601A8CEC96E00E9435967B018C0130
:10D080008CEC96E00E941596E616F706080719073D
:10D09000F1F486EC98E00E9435967B018C0186ECD9
:10D0A00098E00E941596E616F7060807190779F426
:10D0B00080EC9AE00E9435967B018C0180EC9AE02E
:10D0C0000E941596E616F7060807190711F0F401F5
:10D0D00012A280E091E164E00E949C158330D9F5B2
:10D0E00080E091E161E00E949C15833041F080E096
:10D0F00091E161E00E949C15813009F0B7C0C40144
:10D100000E94B01AC40160E00E940519C4010E9487
:10D11000A71621C0D40192961C920E9411C0F4015E
:10D12000668F778F80A391A31083C4010E943D6214
:10D13000A3C0112381F481E0D40192968C930E94C4
:10D1400011C0F401668F778F80A391A382E0808362
:10D150000E94892D91C06E817F818885998520E00C
:10D1600030E040E053E40E94CBCF8823D9F46A81B9
:10D170007B818C819D8120E030E040E053E40E947F
:10D18000CBCF882379F4C301B20120E030E040E046
:10D1900053E40E94CBCF882329F4D40119968C91B3
:10D1A000813039F080E091E10E948C15882309F0EC
:10D1B00063C0F401118627C0D40113968C91139794
:10D1C000803859F080E813968C9380E090E040E03E
:10D1D00050E060E070E00E94A42DF401848180386A
:10D1E00051F080E8848381E090E040E050E060E02E
:10D1F00070E00E94A42DD40119968C91199781306A
:10D20000D9F519961C9280E00E94C12735C080E0B4
:10D2100091E10E948C15813079F666CBC4016A2DAC
:10D2200048E09E012F5F3F4F00E010E074EFE72ED3
:10D2300071E0F72ECC24CA940E94F616882309F0D8
:10D2400062CD8ECDC4016A2D46E09E012F5F3F4F17
:10D2500000E010E054EFE52E51E0F52ECC24CA9406
:10D260000E94F616882309F091CDBDCDF40112A1DC
:10D27000113009F05ECF4ECF29960FB6F894DEBF7D
:10D280000FBECDBFCF91DF911F910F91FF90EF9017
:10D29000DF90CF90BF90AF909F908F907F906F90D6
:10D2A0005F904F9008951F93182F0E94B1311092F4
:10D2B000B5041092B6041092B7041092B8041092FC
:10D2C000A4041092A3048CEC96E00E94959686EC40
:10D2D00098E00E94959680EC9AE00E9495961092B4
:10D2E000C1041092D8040E94AF320E94CFAF0E94B6
:10D2F0001533112341F40E94F614882321F00E9473
:10D30000F3140E94CA251F9108950F931F938C0157
:10D3100081E00E945369F80112821F910F910895D4
:10D320002F923F924F925F926F927F928F929F9235
:10D33000AF92BF92CF92DF92EF92FF920F931F9323
:10D34000CF93DF93EC0180919C118823A1F48CE9A9
:10D3500091E10E94E2C4892B71F00E9411C0609398
:10D36000A6117093A7118093A8119093A9118CE92D
:10D3700091E10E94ECC4CE010E94CB18882309F4ED
:10D3800080C08A81882329F08091C104882309F014
:10D3900078C01092A5111092A41180E091E164E090
:10D3A00040E00E94601A80E091E163E04091A411A6
:10D3B0000E94601A18820BC10E9411C06E8F7F8F6D
:10D3C00088A399A367C0813009F064C00E9411C08E
:10D3D0002E8D3F8D48A159A1621B730B840B950BB9
:10D3E000615D77408040904008F454C01092A511D0
:10D3F0001092A41180E091E164E040E00E94601A84
:10D4000080E091E163E04091A4110E94601A83E002
:10D410008883CE010E948569DAC040E08091A51121
:10D42000882309F441E04093A51180E091E164E094
:10D430000E94601A0E9411C06093A6117093A711F8
:10D440008093A8119093A9110E94E0AE9091A4112D
:10D45000882359F0992309F0BAC081E08093A41180
:10D4600080E091E163E041E009C0992309F4AFC095
:10D470001092A41180E091E163E040E00E94601A04
:10D48000A6C080E091E164E00E949C15833009F021
:10D490009ACF92CF2A883B884C885D88EE88FF8897
:10D4A000088D198DAA8CBB8CCC8CDD8C6E847F840E
:10D4B000888899880E9411C0E20CF31C041D151D78
:10D4C000EA0CFB1C0C1D1D1DE60CF71C081D191D8C
:10D4D000E61AF70A080B190BC801B70120E83EEE5F
:10D4E00046E350E00E942CD2D22EC801B70120E6BC
:10D4F0003AEE40E050E00E942CD28CE3D89EC0016E
:10D500001124281BCE016CE0422F50E024EF31E0C3
:10D510000E94AF16CE016AE04D2D50E024EF31E0BD
:10D520000E94AF164FA9CE016BE050E024EF31E02E
:10D530000E94AF1648ADCE0169E050E024EF31E023
:10D540000E94AF1649ADCE016FE050E024EF31E00C
:10D550000E94AF164AADCE016EE050E024EF31E0FC
:10D560000E94AF164BADCE0160E150E024EF31E0F8
:10D570000E94AF164DADCE016DE050E024EF31E0DA
:10D580000E94AF164EADCE0168E050E024EF31E0CE
:10D590000E94AF164FADCE0166E050E024EF31E0BF
:10D5A0000E94AF160E9411C02091A6113091A711C0
:10D5B0004091A8115091A911621B730B840B950B1C
:10D5C000645F71408040904008F43ECF26CFDF91E9
:10D5D000CF911F910F91FF90EF90DF90CF90BF9070
:10D5E000AF909F908F907F906F905F904F903F9003
:10D5F0002F900895CF93DF93EC010E9411C02091EA
:10D60000AA113091AB114091AC115091AD11621B38
:10D61000730B840B950B6A3071058105910508F435
:10D6200050C00E9411C06093AA117093AB118093F7
:10D63000AC119093AD1180E091E10E945B1B0E94C0
:10D640003BBD80E091E10E948C158130D1F489814D
:10D650008823B9F480E091E161E041E00E94601A22
:10D6600040E08CA9882309F441E080E091E162E088
:10D670000E94601A1E821F82188680E88B838C832A
:10D680008D8380E091E10E948C15898388818823B5
:10D6900021F4CE010E944B6411C0813021F4CE01EF
:10D6A0000E9490690BC0823021F4CE010E940A32A0
:10D6B00005C0833019F4CE010E944519CE010E94A5
:10D6C000F619DF91CF9108951F93182F0E9411C072
:10D6D0002091DC103091DD104091DE105091DF1070
:10D6E000621B730B840B950B6E5E72408040904002
:10D6F00008F490C00E9411C06093DC107093DD109C
:10D700008093DE109093DF10E12FF0E0E256FB4FA4
:10D7100080818130B1F0883041F48091C104813042
:10D7200009F078C00E94B13175C0823031F0833089
:10D7300059F48091C104882321F080E00E9453694C
:10D7400069C00E94085566C0843051F483EE9CE0A5
:10D7500062E072E00E94121B81E08093A0045AC034
:10D76000853029F58CEC96E00E94B39360E0882325
:10D7700009F461E08CEC96E00E942BA186EC98E025
:10D780000E94B39360E0882309F461E086EC98E09E
:10D790000E942BA180EC9AE00E94B39360E0882362
:10D7A00009F461E080EC9AE00E942BA133C089303B
:10D7B00079F40E94B1318CEC96E00E94B39586EC2E
:10D7C00098E00E94B39580EC9AE00E94B39522C045
:10D7D0008A3001F50E94B1318CEC96E00E943596BA
:10D7E000AB01BC018CEC96E00E94489486EC98E07A
:10D7F0000E943596AB01BC0186EC98E00E944894EB
:10D8000080EC9AE00E943596AB01BC0180EC9AE076
:10D810000E9448941F91089581E00E94646B0895CE
:10D8200080E00E94646B0895EF92FF920F931F9324
:10D83000CF93DF93982F8091A504891709F468C0CE
:10D8400081E08093CB069093A5049923E1F10E9497
:10D8500042968093CB1080E00E943F96C0E0D0E0DB
:10D86000EAEFEE2EE1E0FE2ECE9D8001CF9D100D61
:10D87000DE9D100D11240453194FC8010E94D4934A
:10D88000FE01ED53FE4E8083C80160E00E94CF93FD
:10D890002196C330D10541F787EB96E00E941DAF7A
:10D8A000A0E0B0E08093BF119093C011A093C1118C
:10D8B000B093C21187EB96E060E177E20E9419AF66
:10D8C0000E94085525C080E00E9453698CEC96E0C8
:10D8D0006091C3110E94CF9386EC98E06091C411CF
:10D8E0000E94CF9380EC9AE06091C5110E94CF9383
:10D8F0006091BF117091C01187EB96E00E9419AF43
:10D900001092A4041092A3048091CB100E943F9621
:10D91000DF91CF911F910F91FF90EF9008959F920B
:10D92000AF92BF92CF92DF92EF92FF920F931F932D
:10D93000982EFA01643609F46EC1653670F56730C9
:10D9400009F4CEC0683098F4643009F476C06530CC
:10D9500038F4623009F44FC0633009F0C3C25EC0CE
:10D96000653009F485C0663009F0BCC29DC06A30DC
:10D9700009F400C16B3038F4683009F4CDC0693067
:10D9800009F0B0C2E4C06C3009F421C16C3008F475
:10D990000AC16D3009F0A6C22AC16B3609F4DDC197
:10D9A0006C3698F4673609F473C1683638F4653616
:10D9B00009F445C1663609F095C256C1693609F4C5
:10D9C00097C16A3608F0B0C17BC16E3609F40DC24A
:10D9D0006F3638F46C3609F4D7C16D3609F082C25F
:10D9E000ECC1603709F42AC2603708F413C261370A
:10D9F00009F078C23CC24081411141E04093CB061E
:10DA0000642F70E080E090E00E9468D08B019C0160
:10DA1000892D62E070E049EA55E027C087EB96E087
:10DA20000E94C7AF892D63E070E04BE955E00E948A
:10DA3000BF2481E00E94B21C55C284E596E0BA0181
:10DA40000E94A6B0AB01BC0187EB96E00E94F8AE45
:10DA500087EB96E00E940AAF0E9468D08B019C0180
:10DA6000892D64E070E044E855E00E940C23E1CF8A
:10DA700084E596E0BA010E949EB0BC0187EB96E077
:10DA80000E94F4AE87EB96E00E9406AFA0E0B0E003
:10DA9000BC01CD010E9468D08B019C01892D65E0FD
:10DAA00070E04FE655E0E1CF84E596E0BA010E94D0
:10DAB0009EB0BC0187EB96E00E9419AF87EB96E021
:10DAC0000E941DAFA0E0B0E0BC01CD010E9468D073
:10DAD0008B019C01892D66E070E04BE555E0C5CFD8
:10DAE00084E596E0BA010E949EB0BC0187EB96E007
:10DAF0000E94FEAE87EB96E00E9402AFA0E0B0E08D
:10DB0000BC01CD010E9468D08B019C01892D67E08A
:10DB100070E046E455E0A9CF60E08081811161E0CA
:10DB200087EB96E00E9410AF87EB96E00E9413AF60
:10DB300090E0A0E0B0E0BC01CD010E9468D08B0174
:10DB40009C01892D68E070E04AE255E08ECF40816B
:10DB5000411141E04093CA06642F70E080E090E0FC
:10DB60000E9468D08B019C01892D69E070E042E140
:10DB700055E07BCF84E596E0BA010E94A6B0AB01E8
:10DB8000BC0187EB96E00E94E8AE87EB96E00E942E
:10DB9000EEAE0E9468D08B019C01892D6AE070E096
:10DBA0004AEF54E062CF80810E94146C0E94C91435
:10DBB00090E0A0E0B0E0BC01CD010E9468D08B01F4
:10DBC0009C01892D6BE070E046EE54E04ECF608101
:10DBD0006093A60470E080E090E00E9468D08B0122
:10DBE0009C01892D6CE070E041ED54E03ECF8081D6
:10DBF0000E941E390E94E81090E0A0E0B0E0BC0155
:10DC0000CD010E9468D08B019C01892D6DE070E0F0
:10DC100043EB54E02ACF6091CB0670E080E090E0C7
:10DC20000E9468D08B019C01892D64E670E047EA70
:10DC300054E00E940C2381E06091CB0615C10E9444
:10DC4000E0AE90E0A0E0B0E0BC01CD010E9468D061
:10DC50008B019C01892D65E670E045E954E00E9446
:10DC60000C230E94E0AEFEC087EB96E00E940AAF54
:10DC70000E9468D08B019C01892D66E670E046E821
:10DC800054E00E940C2387EB96E00E940AAF8FC0FD
:10DC900087EB96E00E9406AFA0E0B0E0BC01CD01AA
:10DCA0000E9468D08B019C01892D67E670E049E7EE
:10DCB00054E00E940C2387EB96E00E9406AF2FC031
:10DCC00087EB96E00E941DAFA0E0B0E0BC01CD0163
:10DCD0000E9468D08B019C01892D68E670E04DE6BA
:10DCE00054E00E940C2387EB96E00E941DAF17C002
:10DCF00087EB96E00E9402AFA0E0B0E0BC01CD014E
:10DD00000E9468D08B019C01892D69E670E040E695
:10DD100054E00E940C2387EB96E00E9402AFBC0106
:10DD200081E00E947E1CDEC087EB96E00E9413AF6C
:10DD300090E0A0E0B0E0BC01CD010E9468D08B0172
:10DD40009C01892D6AE670E04BE454E00E940C23AC
:10DD500087EB96E00E9413AF85C06091CA0670E021
:10DD600080E090E00E9468D08B019C01892D6BE6D9
:10DD700070E04DE354E00E940C236091CA0681E0FC
:10DD800070E00E94641CAEC087EB96E00E94EEAE8D
:10DD90000E9468D08B019C01892D6CE670E04DE2F9
:10DDA00054E00E940C2387EB96E00E94EEAEAB019C
:10DDB000BC0181E00E94491C95C00E94CC14BC01AA
:10DDC00081E00E947E1C0E94CC14A0E0B0E0BC0167
:10DDD000CD010E9468D08B019C01892D6DE670E019
:10DDE0004FE154E00E940C237DC00E94C91490E0D2
:10DDF000A0E0B0E0BC01CD010E9468D08B019C0185
:10DE0000892D6EE670E041E154E00E940C230E94EF
:10DE1000C91428C06091A60470E080E090E00E94E0
:10DE200068D08B019C01892D6FE670E042E054E0E0
:10DE30000E940C2381E06091A60416C00E94E810A5
:10DE400090E0A0E0B0E0BC01CD010E9468D08B0161
:10DE50009C01892D60E770E04AEE53E00E940C239C
:10DE60000E94E810682F81E00E94981C3BC08091BE
:10DE70008205882399F10E944296882379F587EBE1
:10DE800096E00E9406AF6C0187EB96E00E940AAF15
:10DE90007B018C0187EB96E00E9402AF5601CC24F7
:10DEA000DD24A0E0B0E0A80EB91ECA1EDB1EAE0C39
:10DEB000BF1CC01ED11EC601B5010E946AD08B01D5
:10DEC0009C01892D61E770E04BED53E00E940C232B
:10DED00081E0B601A5010E942E1C04C0AA24BB2427
:10DEE0006501E9CF1F910F91FF90EF90DF90CF90E8
:10DEF000BF90AF909F900895EF92FF920F931F9362
:10DF00000E9411C07B018C018091C9119091CA11AE
:10DF1000A091CB11B091CC11A8019701281B390B0E
:10DF20004A0B5B0B273931054105510508F466C0E2
:10DF30008091C104882339F08091A504811180E08B
:10DF40000E9453695BC080918205882319F00E946A
:10DF50006A3361C08CEC96E00E944394882309F0F8
:10DF60005AC086EC98E00E944394882309F053C07D
:10DF700080EC9AE00E944394882309F04CC0809181
:10DF8000C9119091CA11A091CB11B091CC11A801E7
:10DF90009701281B390B4A0B5B0BDA01C901885E1C
:10DFA0009340A040B04020F48091C8118F5F01C021
:10DFB00081E08093C81183EE9CE06CE172E00E94E6
:10DFC000AB2083EE9CE06091C8110E94B71F809146
:10DFD000C811833098F08091A204882311F481E065
:10DFE00001C080E00E941E391092C81164E670E002
:10DFF00080E090E00E9445C00E94EB54E092C9117D
:10E00000F092CA110093CB111093CC111F910F9174
:10E01000FF90EF9008950E94B131F0CF0E94CFAFF2
:10E020000E94B1311092C1040E9415330895CF921D
:10E03000DF92EF92FF920F931F93CF93DF93EB0149
:10E04000873609F43DC4883608F082C0843109F46B
:10E0500061C28531E8F58A3009F4AFC18B30E0F454
:10E06000853009F42AC1863050F4833009F400C1A8
:10E07000843008F012C1823009F0BBC6EFC087308F
:10E0800009F43AC1873008F42EC1883009F453C12D
:10E09000893009F0AEC682C18F3009F408C28031E0
:10E0A00050F48D3009F4D4C18E3008F0E8C18C30C2
:10E0B00009F09FC6B8C1813109F40DC2813108F45D
:10E0C000FFC1823109F410C2833109F092C615C232
:10E0D0008D3109F401C38E31C8F4883109F464C26A
:10E0E000893138F4863109F438C2873108F049C2E1
:10E0F0001EC28A3109F46DC28A3108F460C28B31C4
:10E1000009F49DC28C3109F074C6D6C2823309F479
:10E1100045C3833368F48F3109F400C38F3108F4A9
:10E12000E5C2803209F412C3813209F062C626C307
:10E13000843609F468C3853620F4833309F059C660
:10E1400045C3853609F465C3863609F052C686C3D1
:10E150008B3709F4B5C48C3708F040C0813709F417
:10E1600022C48237E0F48C3609F4C3C38D3650F4F0
:10E17000893609F4ACC3893608F4A5C38B3609F097
:10E1800038C6ADC38E3609F4F5C38E3608F4DEC347
:10E190008F3609F4F6C3803709F02BC6FFC38637E4
:10E1A00009F433C4873768F4833709F406C4833726
:10E1B00008F4FEC3843709F408C4853709F019C68A
:10E1C00008C4883709F439C4883708F433C4893758
:10E1D00009F447C48A3709F00CC658C4843809F4D6
:10E1E00060C58538C8F48F3709F4E2C4803838F444
:10E1F0008D3709F4B3C48E3708F0C5C495C481388F
:10E2000009F411C5813808F4E7C4823809F420C53F
:10E21000833809F0EEC531C5883C09F4A9C5893CAD
:10E2200068F4863809F465C5863808F44EC58C381C
:10E2300009F474C5863909F0DCC585C58D3F09F43C
:10E24000B6C58E3F20F48C3F09F0D3C5A7C58E3FDD
:10E2500009F4BBC58F3F09F0CCC5BFC580E062E0C3
:10E2600070E04CEC5DE00E94BF240E94AD5F21C0D5
:10E2700080E063E070E04CEB5DE00E94BF248091A1
:10E28000C1048823B1F081E08093D7040E944296B4
:10E29000882379F00E940E700CC080E064E070E08A
:10E2A0004BEA5DE00E94BF2480E00E945369109217
:10E2B000D70481E00E94B21C9CC580E065E070E05C
:10E2C00048E95DE00E94BF248091AE11882331F4BB
:10E2D0000E94FC3281E08093AE11EBCF0E940333A9
:10E2E0001092AE11E6CF60E08881811161E086EB8B
:10E2F00096E00E949D93DDCF8AE0E9EAF3E0DF013A
:10E300001D928A95E9F780E090E0FE01E80FF91F81
:10E310002081222321F0FC01E755FC4F2083019648
:10E320008B30910591F782E090E069EA73E04AE072
:10E330000E94D8B5BECF6881623010F480E018C06A
:10E340006093B4031092B50384E596E070E00E94F8
:10E3500079B06091B4037091B50380E995E00E94B3
:10E3600079B080E090E064EB73E00E94261981E0D0
:10E370000E94B21C6091B4037091B503882777FDA9
:10E380008095982F0E946AD08B019C0180E068E004
:10E3900070E046E85DE00E940C232BC58881833045
:10E3A00020F080E00E94B21C84CF882319F40E94E0
:10E3B00039937FCF0E9465937CCF80E06AE070E064
:10E3C0004EE65DE00E94BF24C0E0D0E08AEFE82E78
:10E3D00081E0F82ECE9D8001CF9D100DDE9D100DA9
:10E3E00011240453194FC8010E945894A0E0B0E0D2
:10E3F000BC01CD010E9468D0AB01BC01C8010E94E4
:10E40000B894C80164E00E9421ABC8010E941FA813
:10E41000C80161E00E94F7A02196C330D105D1F672
:10E420000E94D02B46CFE8808E2D0E943B150E9483
:10E430000639FF2400E010E0C801B7010E9468D04F
:10E440008B019C0180E06CE070E04DE45DE0D8C1A0
:10E450001881098180E0612F0E94B53881E0602F2A
:10E460000E94B5380E940639143011F0043021F4AE
:10E4700081E08093A2041DCF1092A2041ACF90E0F5
:10E480008881811191E0892F0E9409110E940E114B
:10E4900090E0A0E0B0E0BC01CD010E9468D08B010B
:10E4A0009C0180E06EE070E045E35DE0A9C184E599
:10E4B00096E00E949EB09093B9038093B80308C081
:10E4C00084E596E00E949EB09093BB038093BA03CC
:10E4D0000E940639EECE84E596E00E949EB09093AD
:10E4E000BD038093BC03F4CF84E596E00E949EB008
:10E4F0009093BF038093BE03EBCF1881113019F4C2
:10E500001093C103D6CE112319F41092C103D1CEBA
:10E5100080E0D0CE84E596E00E94A6B06093CE0461
:10E520007093CF048093D0049093D104C2CE84E53D
:10E5300096E00E94A6B06093D2047093D3048093B7
:10E54000D4049093D5040E9468D08B019C0180E094
:10E5500065E170E04FE15DE053C188810E943F9624
:10E560000E94429690E0A0E0B0E0BC01CD010E9484
:10E5700068D08B019C0180E066E170E048E05DE0DE
:10E580003FC1E8808E2D0E94C127FF2400E010E0EB
:10E59000C801B7010E9468D08B019C0180E067E14F
:10E5A00070E041EF5CE02CC188810E94571580E04B
:10E5B00068E170E049ED5CE00E94BF247ACE80E023
:10E5C00069E170E048EB5CE00E94BF240E94892D65
:10E5D00070CEC0E0D0E00AEFE02E01E0F02ECE9D3C
:10E5E0008001CF9D100DDE9D100D11240453194F95
:10E5F000C8010E943596AB01BC01C8010E940D966E
:10E6000083EE9CE064E372E00E94542083EE9CE081
:10E610006C2F0E94D61F83EE9CE06CE372E00E9498
:10E620005420C8010E941596AB01BC0183EE9CE00A
:10E630000E9435222196C330D10589F63ACEC0E03A
:10E64000D0E01AEFE12E11E0F12ECE9D8001CF9D9A
:10E65000100DDE9D100D11240453194FC8010E94A6
:10E660003596AB01BC01C8010E941D9680E06BE1AC
:10E6700070E040E95CE00E94BF2483EE9CE065E42A
:10E6800072E00E94542083EE9CE06C2F0E94D61F03
:10E6900083EE9CE06CE472E00E945420C8010E946A
:10E6A0002596AB01BC0183EE9CE00E9435222196A9
:10E6B000C330D10551F6FDCD68816093C20370E08F
:10E6C00080E090E00E9468D08B019C0180E06CE1CA
:10E6D00070E04DE75CE094C080E06DE170E041E601
:10E6E0005CE00E94BF240E94CA25E3CD888180930C
:10E6F00098048AE590E068E974E00E94221960912C
:10E70000980470E080E090E00E9468D08B019C014A
:10E7100080E06EE170E047E45CE0BDC288818093F8
:10E720009A048BE590E06AE974E00E9422196091F6
:10E730009A0470E080E090E00E9468D08B019C0118
:10E7400080E06FE170E046E25CE0B9C288818093CE
:10E7500099048CE590E069E974E00E9422196091C7
:10E76000990470E080E090E00E9468D08B019C01E9
:10E7700080E060E270E04CE05CE0B5C268816093EC
:10E78000B70370E080E090E00E9468D08B019C01AC
:10E7900080E061E270E041EF5BE0BAC290E0888126
:10E7A000811191E0892F0E94F5100E94FC1090E0E9
:10E7B000A0E0B0E0BC01CD010E9468D08B019C01BB
:10E7C00080E062E370E04AED5BE01AC080E00E9406
:10E7D000F51090E08881811191E0892F0E94FF104F
:10E7E0000E94061190E0A0E0B0E0BC01CD010E94C3
:10E7F00068D08B019C0180E063E370E047EC5BE054
:10E800000E940C2356CD81E046E650E060E070E0C7
:10E81000B7C18091D804882319F0B4E0FB2E10C052
:10E820008091D604882319F0A3E0FA2E09C08091C4
:10E83000C104882319F0F2E0FF2E02C0F090D70443
:10E840006F2D70E080E090E00E9468D08B019C0109
:10E8500080E065E670E04AEB5BE070C20E94F9146C
:10E860000E9468D08B019C0180E066E670E047EA78
:10E870005BE00E940C230E94F9147B018C018091C3
:10E88000E30C83FF1AC08091E40C882341F089E7F0
:10E8900093E1B801A7012AE030E00E94F6C580911B
:10E8A000E50C882351F08091E60C9091E70CB801BB
:10E8B000A7012AE030E00E94F6C50E94F9145DC16C
:10E8C0000E94E0AE85C281E06091B60383C281E020
:10E8D00069EA73E04AE050E00E94111C8AC20E947B
:10E8E0009F1F6B017C0180E06BE670E046E95BE016
:10E8F0001EC089E20E94EEC0AA2797FDA095BA2FFC
:10E90000BC01CD010E946AD020E030EC4FE754E416
:10E910000E94CFCF20E030E040EA50E40E941ED1B8
:10E920006B017C0180E06CE670E045E85BE09701FC
:10E9300086010E940C23C701B60120E030E048ECBC
:10E9400052E40E941ED10E943CD017C16091C003C6
:10E9500070E080E090E00E9468D08B019C0180E034
:10E960006DE670E04AE65BE00E940C2381E0609176
:10E97000C00330C270919E0460E080919F0490E0DB
:10E9800009C088E10E94D3C1182F89E10E94D3C138
:10E99000712F60E0682B792B81E014C26091B8037D
:10E9A0007091B9030EC06091BA037091BB0309C0A6
:10E9B0006091BC037091BD0304C06091BE0370916F
:10E9C000BF0381E00E947E1C14C281E06091C103FC
:10E9D00001C26091D2047091D3048091D4049091CB
:10E9E000D5040E9468D08B019C0180E065E770E04F
:10E9F0004CE55BE00E940C234091D2045091D3047B
:10EA00006091D4047091D504BAC00E94429690E0FF
:10EA1000A0E0B0E0BC01CD010E9468D08B019C0158
:10EA200080E066E770E040E55BE00E940C230E9416
:10EA30004296CEC10E94F010CBC16091E10470E01B
:10EA400080E090E00E9468D08B019C0180E068E744
:10EA500070E040E45BE00E940C2381E06091E104FF
:10EA6000B9C10E945C1590E0A0E0B0E0BC01CD010E
:10EA70000E9468D08B019C0180E069E770E040E370
:10EA80005BE00E940C230E945C15A2C10E940E1143
:10EA900090E0A0E0B0E0BC01CD010E9468D08B0105
:10EAA0009C0180E06AE770E04EE15BE00E940C238D
:10EAB0008091E104882309F09CC10E940E117FC15E
:10EAC0000E947D1E90E0A0E0B0E0BC01CD010E945C
:10EAD00068D08B019C0180E06BE770E041E15BE076
:10EAE0000E940C230E947D1E182F8091E30C83FF4F
:10EAF00018C08091E40C882339F089E793E1612FF5
:10EB00004AE050E00E942DC68091E50C882349F030
:10EB10008091E60C9091E70C612F4AE050E00E9452
:10EB20002DC60E947D1E54C10E94E545182F80E02D
:10EB30006CE770E04CEF5AE00E94BF2483EE9CE04B
:10EB40000E94A710882339F089E793E1612F42E002
:10EB500050E00E942DC681E0612F3CC10E94D41D6F
:10EB60000E9468D08B019C0180E06DE770E047EE69
:10EB70005AE00E940C230E94D41DAB01BC0181E02D
:10EB80000E94491C36C10E94EB10F82E882311F018
:10EB9000FF24F3946F2D70E080E090E00E9468D035
:10EBA0008B019C0180E06EE770E040ED5AE0C6C04A
:10EBB0006091C20370E080E090E00E9468D08B0119
:10EBC0009C0180E06FE770E045EC5AE00E940C2366
:10EBD00081E06091C203FEC08CEC96E00E944394F9
:10EBE000682F811161E0F62E86EC98E00E94439434
:10EBF000882311F0FF24F39480EC9AE00E94439460
:10EC0000882311F0FF24F3946091C20370E080E048
:10EC100090E00E9468D08B019C0180E060E870E089
:10EC20004FEA5AE08BC00E94F329F82E882311F096
:10EC3000FF24F3946F2D70E080E090E00E9468D094
:10EC40008B019C0180E061E870E04EE95AE076C0FB
:10EC50000E941D1D90E0A0E0B0E0BC01CD010E942B
:10EC600068D08B019C0180E062E870E045E85AE0E2
:10EC70000E940C230E941D1DABC06091980470E09F
:10EC800080E090E00E9468D08B019C0180E063E806
:10EC900070E043E75AE00E940C2381E06091980401
:10ECA00099C060919A0470E080E090E00E9468D082
:10ECB0008B019C0180E064E870E04AE55AE00E9424
:10ECC0000C2381E060919A0485C06091990470E002
:10ECD00080E090E00E9468D08B019C0180E065E8B4
:10ECE00070E048E45AE00E940C2381E060919904AE
:10ECF00071C068816093B70370E080E090E00E948B
:10ED000068D08B019C0180E066E870E045E35AE042
:10ED10000E940C2381E06091B7035CC00E946215E1
:10ED2000F82E682F70E080E090E00E9468D08B01A0
:10ED30009C0180E06CE870E040E25AE00E940C2305
:10ED400081E06F2D47C00E94FC1090E0A0E0B0E091
:10ED5000BC01CD010E9468D08B019C0180E066E976
:10ED600070E041E15AE00E940C230E94FC1027C091
:10ED70000E945C827C01B701882777FD8095982FDF
:10ED80000E946AD08B019C0180E068EC70E043E057
:10ED90005AE00E940C2381E0B70114C060E0888132
:10EDA000811161E083EE9CE00E94AE1008C060E03B
:10EDB0008881811161E083EE9CE00E94AA10682F97
:10EDC00081E070E00E94641C14C088810E94884821
:10EDD000682F81E00E94981C0CC080E06FEF70E00B
:10EDE0004CEE59E00E94BF2481E00E94B21C0E94B8
:10EDF000DB46DF91CF911F910F91FF90EF90DF9055
:10EE0000CF9008950F931F93CF93DF93082F162F62
:10EE1000EA010E9411C06093DD047093DE048093C8
:10EE2000DF049093E004043018F40130E8F405C0E6
:10EE3000043091F10530D9F535C00E94FC108823CB
:10EE400071F48091E104813051F4143640F41E30A5
:10EE500031F0173121F0123311F0133341F5812FC6
:10EE6000BE010E94177026C00E94FC10882371F416
:10EE70008091E104813051F4143640F4812F8350A5
:10EE8000823020F0163011F01D3089F4802F612F70
:10EE9000AE010E9454550EC084E0612FAE010E9465
:10EEA0008F6C08C0812FBE010E94CC4003C080E05F
:10EEB0000E94B21CDF91CF911F910F91089593E0B2
:10EEC0009093A8030E9402770895EF92FF920F9308
:10EED0001F93F82EE62E8A0182E08093A8030E94F9
:10EEE00011C06093DD047093DE048093DF0490937F
:10EEF000E00483EE9CE06DEF7DE00E9471208F2D99
:10EF00006E2DA8010E94CA248F2D6E2DA8010E948B
:10EF100002771F910F91FF90EF900895EF92FF926B
:10EF20000F931F93F82EE62E8A0181E08093A803A9
:10EF30000E9411C06093DD047093DE048093DF04AF
:10EF40009093E00483EE9CE068E07EE00E947120F4
:10EF50008F2D6E2DA8010E94CA248F2D6E2DA80121
:10EF60000E9402771F910F91FF90EF900895CF9329
:10EF7000DF93EA01653009F45BC0663070F46230FB
:10EF8000F9F0633020F4613009F072C016C06330CC
:10EF9000D9F0643009F06CC01AC0683009F45AC066
:10EFA000693020F4673009F063C051C0693009F45A
:10EFB00054C06A3009F05CC053C00E94085558C064
:10EFC00080E00E94536954C00E940E7051C083EECD
:10EFD0009CE068EE7DE00E94121B4881423008F4FC
:10EFE00047C04093B4031092B50380E090E064EB17
:10EFF00073E00E9426196091B4037091B50384E513
:10F0000096E00E9479B06091B4037091B50380E9F5
:10F0100095E00E9479B00E94FC10882319F081E0ED
:10F020000E94B21C8CE065E070E00E94604820C045
:10F0300083E08093A80383EE9CE064E572E00E9485
:10F04000542081E00E94F51081E00E94B21C0E94D1
:10F050009F3F0EC00E946A330BC00E946E3308C0EF
:10F0600084E596E00E9473B0BC0181E00E947E1CA2
:10F07000DF91CF9108950E944296882391F48CEC01
:10F0800096E00E944394813089F186EC98E00E94DA
:10F090004394813059F180EC9AE00E94439481308E
:10F0A00029F186EB96E00E94EF928823D1F08AEB5B
:10F0B0009CE061E00E94A6AE8091D006813041F0D4
:10F0C0008091CA08813021F08091C40A813071F4A6
:10F0D00083EE9CE062E472E10E9431270E940E7090
:10F0E00008958AEB9CE060E00E94A6AE0895EF923E
:10F0F000FF920F931F93CF93DF9383EE9CE068EA18
:10F1000074E10E9431278091D704882341F083EE77
:10F110009CE060E974E10E9431270E940E700E9419
:10F120004296882399F487EB96E00E941DAF892BC5
:10F1300041F10091A3041091A40487EB96E00E9492
:10F140001DAF80179107E8F491E01CC00E94429621
:10F150008823B9F08CEC96E00E949296811181E0B0
:10F16000082F86EC98E00E949296882309F400E02C
:10F1700080EC9AE00E949296882309F400E090E0E7
:10F1800002C090E000E08091A604882309F0B7C097
:10F19000992319F4002309F4B9C00E9442968823E8
:10F1A00009F4C1C10E94D41D2091B9043091BA0460
:10F1B0004091BB045091BC04621B730B840B950BF4
:10F1C00016161706180619060CF0ADC183EE9CE062
:10F1D0006CE674E10E9431270E94D41D2091B9048D
:10F1E0003091BA044091BB045091BC04621773077C
:10F1F0008407950709F47EC00E94D41DAB01BC01B1
:10F2000083EE9CE00E942E494091B9045091BA04CB
:10F210006091BB047091BC0483EE9CE00E942E4977
:10F2200083EE9CE061E574E10E9490250E94D41D6C
:10F23000AB01BC018091B9049091BA04A091BB04C8
:10F24000B091BC04481B590B6A0B7B0B83EE9CE00E
:10F250000E94423983EE9CE068E374E10E9431270A
:10F2600049C00E944296823021F487EB96E00E94CA
:10F27000C7AF0E945C158823B9F18091CC049091AE
:10F28000CD042091A3043091A404820F931F909386
:10F29000CD048093CC048091C4049091C504A091C6
:10F2A000C604B091C7042091B5043091B6044091D2
:10F2B000B7045091B804820F931FA41FB51F809309
:10F2C000C4049093C504A093C604B093C70481E01E
:10F2D0000E9453690E94EC140E94CA2581E0809329
:10F2E000D9040E94085506C080E00E94536981E05D
:10F2F0008093DA0483EE9CE063E074E1C8C0992354
:10F3000011F4002319F081E08093D8048091A104C6
:10F31000882349F08091A004882329F483EE9CE09F
:10F3200067EC73E1B4C080919E04863029F080912F
:10F330009F04863009F0FDC081E00E944E2788239B
:10F3400009F4F7C086E08093D0100E941B3883EE4A
:10F350009CE062E973E19BC00E9411C07B018C01BB
:10F360008091CC109091CD10A091CE10B091CF1083
:10F37000E81AF90A0A0B1B0B87EB96E00E94EEAE27
:10F38000E616F7060807190748F48091CB0688238C
:10F3900029F08091A204882309F4D3C083EE9CE075
:10F3A0006AE773E10E943127C091A304D091A404BD
:10F3B0008091E30C84FF18C08091E40C882339F01D
:10F3C00089E793E1BE014AE050E00E940AC68091BD
:10F3D000E50C882349F08091E60C9091E70CBE0182
:10F3E0004AE050E00E940AC683EE9CE06FE971E0BB
:10F3F0000E94AB20C0E0D0E00AEF11E083EE9CE079
:10F4000063E773E10E94902583EE9CE06C2F0E94DD
:10F41000352083EE9CE069E672E00E94AB20C09F3D
:10F42000C001C19F900DD09F900D11248453994F1E
:10F430000E943596AB01BC0183EE9CE00E944239EC
:10F4400083EE9CE06FE971E00E94AB202196C3300F
:10F45000D105A1F683EE9CE06DE571E00E94F51AFE
:10F460008091CB068823B1F48AEB9CE062E00E9495
:10F47000A6AE0E9411C06093CC107093CD10809303
:10F48000CE109093CF1083EE9CE06EE373E10E9468
:10F49000312757C083EE9CE060E273E10E94312780
:10F4A0000E94E0AE082F8091E30C84FF1AC0809187
:10F4B000E40C882341F089E793E1602F70E04AE093
:10F4C00050E00E94A4C68091E50C882351F0809101
:10F4D000E60C9091E70C602F70E04AE050E00E944B
:10F4E000A4C60E94E0AE882361F583EE9CE068EF3D
:10F4F00072E10E9431278AEB9CE060E00E94A6AE98
:10F500001092D0101092A0040E9411C06093CC10F1
:10F510007093CD108093CE109093CF1087EB96E030
:10F520000E947CAF0EC00E945C15882309F0A1CE1A
:10F5300098CE86EB96E00E94EF92882309F42ECFB6
:10F540000BCFDF91CF911F910F91FF90EF90089516
:10F55000AF92BF92CF92DF92EF92FF920F931F93E1
:10F560000E9411C07B018C012091B5043091B6043A
:10F570004091B7045091B80421153105410551055A
:10F5800041F46093CD117093CE118093CF1190937D
:10F59000D0118091BD049091BE04A091BF04B091A0
:10F5A000C00459016A01A81AB90ACA0ADB0AD601BD
:10F5B000C5018E0D9F1DA01FB11F8093B5049093B0
:10F5C000B604A093B704B093B804E092BD04F092DF
:10F5D000BE040093BF041093C0040097A105B105B9
:10F5E00041F08093B9049093BA04A093BB04B09304
:10F5F000BC048091C204813019F480E00E945369F8
:10F6000086EB96E00E94EF928823E9F02091CE04E9
:10F610003091CF044091D0045091D104211531058F
:10F620004105510581F08091B5049091B604A091F7
:10F63000B704B091B804281739074A075B0718F4D4
:10F6400080E00E94536986EB96E00E94EF92882347
:10F6500049F40E94F292882329F08AEB9CE061E051
:10F660000E94A6AE2091B5043091B6044091B70433
:10F670005091B8048091D2049091D304A091D40405
:10F68000B091D504281739074A075B0720F4809109
:10F69000D904882339F08AEB9CE00E94A9AE10922D
:10F6A000D60422C081E08093D6048091CD11909140
:10F6B000CE11A091CF11B091D011A8019701281BB4
:10F6C000390B4A0B5B0BDA01C901855F9140A04001
:10F6D000B04050F00E940B33E092CD11F092CE1169
:10F6E0000093CF111093D0111F910F91FF90EF90C5
:10F6F000DF90CF90BF90AF900895EF92FF920F935D
:10F700001F93CF93DF9384E596E00E94DDB480E9F8
:10F7100095E00E94DDB482EF95E00E94DDB40E9486
:10F7200011C02091D9113091DA114091DB11509123
:10F73000DC11621B730B840B950B6536710581051B
:10F74000910508F456C088E20E94D3C1019759F48C
:10F750000E9411C06093DD117093DE118093DF1160
:10F760009093E01133C080919D04882379F50E9425
:10F7700011C02091DD113091DE114091DF115091C7
:10F78000E011621B730B840B950B695B7B4080401F
:10F790009040E0F082E00E94C34783EE9CE06CE67C
:10F7A00072E00E94AB208CEC96E068E00E9421ABF6
:10F7B00086EC98E068E00E9421AB80EC9AE068E07B
:10F7C0000E9421AB81E080939D04B2C080919D0492
:10F7D000882329F00E9496500E948354A9C00E9459
:10F7E00011C06093D9117093DA118093DB1190935B
:10F7F000DC110E9411C02091D5113091D611409199
:10F80000D7115091D811621B730B840B950B655F58
:10F8100071408040904050F00E9411C06093D5111B
:10F820007093D6118093D7119093D8118091DC04F6
:10F83000882339F10E9411C02091DD043091DE044B
:10F840004091DF045091E004621B730B840B950B15
:10F85000695E734080409040A0F08CEC96E00E947E
:10F860004394882361F486EC98E00E9443948823B3
:10F8700031F480EC9AE00E944394882311F00E94B6
:10F88000B13100E010E02AEFE22E21E0F22E0E9DD1
:10F89000E0010F9DD00D1E9DD00D1124C453D94FF2
:10F8A000CE010E944394882319F0CE010E941EA32A
:10F8B0000F5F1F4F0330110551F78091C10488235A
:10F8C00059F00E94A8330E94A87A00E010E09AEF55
:10F8D000E92E91E0F92E09C0809182058823A9F3D1
:10F8E0000E94A8330E94103EF0CF0E9DE0010F9DB4
:10F8F000D00D1E9DD00D1124C453D94FCE010E94AE
:10F90000B0A0882361F0CE010E944394882339F48B
:10F91000CE0160E00E94F7A0CE010E9482AC0F5F92
:10F920001F4F0330110509F780E591E10E94FA6A43
:10F93000DF91CF911F910F91FF90EF900895EF927B
:10F94000FF920F931F93CF93DF9389E793E140E0FA
:10F950005BE460E070E00E9466C864E670E080E00E
:10F9600090E00E9445C063E876E080E090E00E946D
:10F97000028283EE9CE06DE772E00E94F51A8CE053
:10F9800061E00E941DC180E061E00E941DC180E035
:10F9900061E00E94A0C18AE260E00E941DC189E28C
:10F9A00060E00E941DC10E9455498AEB9CE060E026
:10F9B0000E94A6AE60E070E08AE795E40E94BD86F2
:10F9C00060E070E48CE996E40E94C68686EB96E0DF
:10F9D00061E00E949D9380E49DE10E94EA9287EBA2
:10F9E00096E048E750E060E070E00E94F8AE87EBF8
:10F9F00096E060E070E00E94FEAE87EB96E060E08B
:10FA000070E00E94F4AE87EB96E06EE97BE20E9424
:10FA1000E3AE87E593E140E051EE60E070E00E94E4
:10FA200079C26091B4037091B50384E596E00E94B9
:10FA300079B084E596E06EE877E70E9484B384E5C8
:10FA400096E066ED72E20E9490B384E596E067EB83
:10FA500077E70E948AB384E596E060E00E946EB08A
:10FA60006091B4037091B50380E995E00E9479B08C
:10FA700080E995E065E677E70E9484B380E995E048
:10FA800060EC72E20E9490B380E995E067EB77E763
:10FA90000E948AB380E995E061E00E946EB06091B7
:10FAA000B4037091B50382EF95E00E9479B082EFC4
:10FAB00095E06FE577E70E9484B382EF95E06AEA0C
:10FAC00072E20E9490B382EF95E067EB77E70E94C5
:10FAD0008AB382EF95E061E00E946EB084E596E023
:10FAE0006AE279E10E9488B080E995E06AE279E112
:10FAF0000E9488B082EF95E06AE279E10E9488B0C6
:10FB000000E010E03AEFE32E31E0F32E0E9DE0012D
:10FB10000F9DD00D1E9DD00D1124C453D94FCE0181
:10FB200061E00E94CF93CE0160E27EE40E945E9489
:10FB3000CE0160E27EE40E949C94CE0140E050E45D
:10FB40006CE976E40E94B894CE0140E050E66AE6A3
:10FB500076E40E940194CE0160E00E9421A1CE01D2
:10FB600060E070E00E94C993CE0165E00E94239599
:10FB7000CE0140E050E060E070E00E940D96CE01C2
:10FB800040E050E060E070E00E941D96CE0160E031
:10FB900070E00E94A4A0CE0140E050E060E87FE366
:10FBA0000E9480A0CE0140E050E060E87FE30E9428
:10FBB00092A00115110519F4CE0164E002C0CE0136
:10FBC00060E10E9421ABCE0160E00E9470A00F5F57
:10FBD0001F4F0330110509F099CF80E591E10E9494
:10FBE000D21A0E94D7458CE065E070E00E94604820
:10FBF00081E06CE77FE642E050E00E9499BD82EE32
:10FC000094E063E070E00E944C86DF91CF911F91F9
:10FC10000F91FF90EF900895FC011382128282E50C
:10FC200094E091838083758364830895FC018481CB
:10FC300095810E9435B10895611571058105910581
:10FC400069F481E090E0A0E0B0E08093E11190934E
:10FC5000E211A093E311B093E41108C06093E111A5
:10FC60007093E2118093E3119093E4115093E611A5
:10FC70004093E511809170008E7F80937000809199
:10FC8000B0008C7F8093B0008091B100877F80931B
:10FC9000B1008091B6008F7D8093B6008091700096
:10FCA0008D7F809370008091B10084608093B1005B
:10FCB0008091B1008C7F8093B10086E090E09093BA
:10FCC000ED118093EC1108951092E7111092E81154
:10FCD0001092E9111092EA111092EB118091EC113F
:10FCE0009091ED118093B200E0E7F0E080818160B7
:10FCF00080830895E0E7F0E080818E7F808308951F
:10FD00008091E7119091E811A091E911B091EA1169
:10FD10000196A11DB11D8093E7119093E811A09366
:10FD2000E911B093EA118091E7119091E811A09147
:10FD3000E911B091EA112091E1113091E211409165
:10FD4000E3115091E41182179307A407B50710F14E
:10FD50008091EB118823F1F481E08093EB11809185
:10FD6000E7119091E811A091E911B091EA11821B7D
:10FD7000930BA40BB50B8093E7119093E811A0931C
:10FD8000E911B093EA11E091E511F091E6110995BE
:10FD90001092EB1108951F920F920FB60F920BB6AF
:10FDA0000F9211242F933F934F935F936F937F9301
:10FDB0008F939F93AF93BF93EF93FF938091EC1139
:10FDC0009091ED118093B2000E94807EFF91EF919F
:10FDD000BF91AF919F918F917F916F915F914F9163
:10FDE0003F912F910F900BBE0F900FBE0F901F9061
:10FDF00018951F920F920FB60F920BB60F92112407
:10FE00002F933F934F935F936F937F938F939F9322
:10FE1000AF93BF93EF93FF93E091F211F091F31141
:10FE20000995FF91EF91BF91AF919F918F917F9134
:10FE30006F915F914F913F912F910F900BBE0F905B
:10FE40000FBE0F901F901895FC01A3E0440F551FA3
:10FE5000661F771FAA95D1F7403080E0580781E0F0
:10FE6000680780E0780714F481E010C033E07595EE
:10FE70006795579547953A95D1F7403080E05807F8
:10FE800081E0680780E078071CF482E0828339C053
:10FE900023E075956795579547952A95D1F740309A
:10FEA00080E0580781E0680780E0780714F483E079
:10FEB000EDCF92E075956795579547959A95D1F74F
:10FEC000403080E0580781E0680780E0780714F44C
:10FED00084E0DCCF82E075956795579547958A95C4
:10FEE000D1F7403080E0580781E0680780E078076C
:10FEF00014F485E0CBCF85E082834FEF5FEF60E0C5
:10FF000070E08FB78383F8945183408350938700C8
:10FF10004093860083818FBF80918100887F80938A
:10FF20008100809181009281892B809381000895C6
:10FF30001092800020E1209381000E94247F089588
:10FF4000EFE6F0E080818E7F80830895E1E8F0E0C5
:10FF50002081DC0112968C91282B208308950F9329
:10FF60001F93CF93DF93EC018B0112161306140637
:10FF7000150624F4BA01A9010E94247F1D830C8375
:10FF800081E080936F00CE010E94A67FDF91CF9128
:10FF90001F910F910895F999FECF72BD61BDF89A36
:10FFA00080B50895F999FECF1FBA72BD61BD40BDFD
:10FFB0000FB6F894FA9AF99A0FBE0895282F9091E7
:10FFC00053129F5F943408F090E080915412891787
:10FFD000E1F33FB7F89480915012882341F0E92F64
:10FFE000F0E0EB5AFD4E2083909353121DC081E048
:10FFF00080935012209351121092521282E088BBCB
:020000021000EC
:1000000080917100826080937100809190008F7365
:100010008068809390008091940090919500409624
:1000200090939900809398003FBF0895862F0E9477
:10003000DE7F81E090E008951F920F920FB60F923D
:100040000BB60F9211242F933F934F935F936F93AF
:100050007F938F939F93EF93FF9340915012509112
:100060005112209198003091990060914C1270913A
:100070004D12809152121FC0260F371F952F91707D
:1000800056954F5F9817B9F0992321F08091900011
:10009000806C04C0809190008F7380688093900082
:1000A00030939900209398009093521250935112DC
:1000B000409350123BC04930F8F2493039F48AE09D
:1000C0008093501280919000806C28C080915312D0
:1000D000E09154128E1769F41092501280919000A2
:1000E0008F7380939000809171008D7F8093710059
:1000F0001DC081E080935012EF5FE43408F0E0E02F
:10010000E0935412F0E0EB5AFD4E8081809351123F
:1001100010925212809190008F73806880939000AB
:10012000260F371F3093990020939800FF91EF918D
:100130009F918F917F916F915F914F913F912F91FF
:100140000F900BBE0F900FBE0F901F9018958091CF
:1001500050128823E1F708950E94A78008951F9206
:100160000F920FB60F920BB60F9211241F932F937D
:100170003F934F935F936F937F938F939F93AF932F
:10018000BF93EF93FF932091960030919700909149
:100190004812992341F0809191008F7B80939100C8
:1001A0001092481208C08091910080648093910061
:1001B00080E88093481270914712772331F5992394
:1001C00009F06CC080914A1290914B12820F931FDC
:1001D00090939B0080939A0084E088BB809171008B
:1001E00084608093710080914C1290914D12280F81
:1001F000391F96958795280F391F30934F122093FA
:100200004E1281E08093471249C040914E125091A6
:100210004F1210914812E0914C12F0914D126091E2
:100220004912AA27BB27AE1BBF0BC901841B950B24
:1002300097FD2CC06695612B7F5F8A0F9B1F7930DD
:1002400018F44E0F5F1FF4CF609349128091710034
:100250008B7F809371009091F6119F5F903508F02D
:1002600090E08091F511981739F0E92FF0E0E9500E
:10027000FE4E60839093F611809191008F7B809366
:100280009100109248121092471208C060934912D0
:1002900050934F1240934E1270934712FF91EF917B
:1002A000BF91AF919F918F917F916F915F914F918E
:1002B0003F912F911F910F900BBE0F900FBE0F908B
:1002C0001F9018951F920F920FB60F920BB60F92B8
:1002D00011242F938F939F93EF93FF93809171003D
:1002E0008B7F80937100809191008F7B8093910030
:1002F000909147128091481280582091491203C072
:100300002695282B9F5F9930D8F32093491290911E
:10031000F6119F5F903508F090E08091F5119817E5
:1003200039F0E92FF0E0E950FE4E20839093F6116A
:1003300010924712809191008F7B809391001092D0
:100340004812FF91EF919F918F912F910F900BBECB
:100350000F900FBE0F901F9018958091F611E091AD
:10036000F5118E1719F42FEF3FEF0EC02E2F2F5FD0
:10037000203508F020E0E22FF0E0E950FE4E8081C9
:100380002093F511282F30E0C90108958091F611CE
:10039000E091F5118E1719F4EFEFFFEF06C0F0E0D2
:1003A000E950FE4E8081E82FF0E0CF010895909152
:1003B000F6118091F511292F30E0482F50E0981761
:1003C00010F4205B3F4F241B350BC9010895809129
:1003D000F5118093F61108950F931F9301E710E034
:1003E000F80180818B7F808380818F7D80830E9454
:1003F000E7810E94A780F80180818D7F80831F9113
:100400000F9108959B01AC012D3A8BE1380780E0F4
:10041000480780E0580730F4109271001092900065
:1004200081E814C063E056954795379527956A95FE
:10043000D1F72D3A8BE1380780E0480780E0580774
:10044000D0F5109271001092900082E88093910094
:1004500030934D1220934C12CA01B90125E230E0CD
:1004600040E050E00E94E6D152E09695879577955E
:1004700067955A95D1F770934B1260934A1287E1B2
:1004800062E00E941DC186E161E00E94A0C186E198
:1004900061E00E941DC1109247121092F611109255
:1004A000F51110925012109253121092541280E2D1
:1004B00088BB809371000895DF93CF9300D0CDB7B0
:1004C000DEB720919C1330919D13CE01019621152A
:1004D000310519F4865A934102C0821B930B9A830B
:1004E000898389819A810F900F90CF91DF91089530
:1004F0002F923F924F925F926F927F928F929F9234
:10050000AF92BF92CF92DF92EF92FF920F931F9321
:10051000DF93CF93CDB7DEB766970FB6F894DEBF03
:100520000FBECDBF69877A878B879C872D873E87D3
:100530004F87588BE98AFA8A0B8B1C8BC601B50151
:100540002FA438A849A85AA82DA92D8B3EA93E8BC7
:1005500029853A854B855C850E9466CF5B016C01DD
:100560006BA57CA58DA59EA52D853E854F855889BB
:100570000E9466CFA60195010E94CFCF3B014C019E
:10058000C801B701A80197010E9467CF7B018C01C8
:10059000C401B30120E030E040E450EC0E941ED1E1
:1005A0009B01AC01C801B7010E9467CFA201910174
:1005B0000E9467CF9058A60195010E94CFCF6D830E
:1005C0007E838F839887C401B30120E030E040E050
:1005D00050EC0E941ED19B01AC0169897A898B89FC
:1005E0009C890E9467CFA20191010E9467CFA6015A
:1005F00095010E94CFCFA60195010E94CFCF2B017C
:100600003C012D893E89C9019A8389831C821B8202
:1006100022243324AFC0E981FA8160817181828113
:10062000938129853A854B855C850E9466CF7B0145
:100630008C01CFA8D8ACC20CD31CA30192010E949C
:100640001ED19B01AC016D817E818F8198850E94B6
:1006500067CF9B01AC01C801B7010E941ED19B016D
:10066000AC0169897A898B899C890E9467CF9B013B
:10067000AC01C801B7010E941ED19B01AC016D8580
:100680007E858F8598890E9467CFF601608371838C
:10069000828393836D817E818F8198859B01AC01DC
:1006A0000E9467CF5B016C01E981FA8160817181F1
:1006B0008281938129853A854B855C850E9466CF2E
:1006C0007B018C0189AC9AAC820C931C20E030E059
:1006D00040E450E40E941ED1A30192010E941ED169
:1006E0009B01AC01C601B5010E9467CF9B01AC0123
:1006F000C801B7010E941ED19B01AC0169897A89AA
:100700008B899C890E9467CFF40160837183828307
:1007100093830BAD1CAD020D131DE981FA8161912C
:10072000719181919191FA83E98329853A854B856D
:100730005C850E9466CF20E030E040EC50E40E94EF
:100740001ED1A30192010E941ED19B01AC01C601E2
:10075000B5010E9467CFF801608371838283938320
:100760002B813C812F5F3F4F3C832B8384E090E0C3
:10077000280E391EEB81FC812BA93CA9E217F30757
:100780000CF449CF66960FB6F894DEBF0FBECDBF0E
:10079000CF91DF911F910F91FF90EF90DF90CF905D
:1007A000BF90AF909F908F907F906F905F904F9091
:1007B0003F902F9008954F925F926F927F928F9209
:1007C0009F92AF92BF92CF92DF92EF92FF920F93E0
:1007D0001F93CF93DF935C012B0169017A013801EC
:1007E00082E0A816B104A4F500D000D08091A41333
:1007F0009091A513EDB7FEB7928381838FE992E0C4
:10080000948383830E94FA0D8091A4139091A51381
:10081000EDB7FEB79283818381EA92E0948383836C
:100820000E94FA0D8091A4139091A513EDB7FEB725
:10083000928381838FEB92E0948383830E94FA0DED
:100840000F900F900F900F9081E090E00E94A6D241
:10085000F8012081318137FD05C0C50101972817B6
:1008600039073CF0C501019795958795F301918370
:100870008083F30100811181F801EE0FFF1FEE0F5D
:10088000FF1FE40DF51DC701B601208131814281B2
:1008900053810E94CBCF88230CF063C00115110552
:1008A00009F4D8C00130110519F1F8013197EE0FA4
:1008B000FF1FEE0FFF1FE40DF51D60817181828126
:1008C0009381A70196010E94CBCF181634F00150F6
:1008D0001040F30111830083BDC0C701B601F201CE
:1008E00024813581468157810E94CBCF181624F090
:1008F000F30111821082AEC05EEFA52E5FEFB52E20
:10090000A00EB11EC1E0D0E0CA15DB0521F4F30151
:10091000C083D1839FC0C50101968C0F9D1F62E0EB
:1009200070E00E9419D2972E062F172FF801EE0FB4
:10093000FF1FEE0FFF1FE40DF51D608171818281A5
:100940009381A70196010E94CBCF18162CF0802F1F
:10095000992D9C01E901D8CF58010894A108B1084C
:10096000D3CF48010894811C911CF401EE0FFF1FA6
:10097000EE0FFF1FE40DF51D60817181828193816F
:10098000A70196010E94CBCF88230CF063C0E5013C
:1009900022970C171D0709F45DC08DEF9FEFA80E7D
:1009A000B91E0A151B0599F00E5F1F4FF801EE0FD7
:1009B000FF1FEE0FFF1FE40DF51DC701B6012081DB
:1009C0003181428153810E94CBCF181624F0F3016C
:1009D000918280823FC0FE01EE0FFF1FEE0FFF1FCE
:1009E000E40DF51D6081718182819381A7019601DB
:1009F0000E94CBCF181624F4E801CA15DB0521F4B8
:100A0000F301D183C08326C0C50101968C0F9D1FC1
:100A100062E070E00E9419D2972E062F172FF8017E
:100A2000EE0FFF1FEE0FFF1FE40DF51D60817181BA
:100A300082819381A70196010E94CBCF18162CF0DA
:100A4000802F992D9C01E901D8CF58010894A10865
:100A5000B108D3CFDF91CF911F910F91FF90EF900D
:100A6000DF90CF90BF90AF909F908F907F906F90CE
:100A70005F904F9008952F923F924F925F926F92A6
:100A80007F928F929F92AF92BF92CF92DF92EF921E
:100A9000FF920F931F93DF93CF93CDB7DEB7669787
:100AA0000FB6F894DEBF0FBECDBF98878F837A87CD
:100AB00069875C874B873E872D87188B0F87DA8A7B
:100AC000C98ABC8AAB8A9E8A8D8AC80162E070E0BE
:100AD0000E9419D27A836983FC82EB821E821D8276
:100AE00022243324A3C0AB81BC812D913D914D9133
:100AF0005C918F81988569857A858E010F5F1F4F84
:100B00000E94DB83A981BA818D01000F111F000FA4
:100B1000111F1196AA0FBB1FAA0FBB1FEDB7FEB77F
:100B200072970FB6F894FEBF0FBEEDBF4DB65EB61E
:100B30000894411C511CE985FA85E00FF11F608182
:100B4000718182819381EB85FC85E00FF11F20810B
:100B5000318142815381ED85FE850E0F1F1FF80103
:100B6000E080F18002811381E985FA85EA0FFB1F9D
:100B7000A080B180C280D380EB85FC85EA0FFB1F8B
:100B80006080718082809380EDB7FEB7618272824F
:100B900083829482ED85FE85AE0FBF1F6D907D90A0
:100BA0008D909C90D20114966D927D928D929C9224
:100BB0001797E1E0F0E01996FC93EE931897EB811C
:100BC000FC811B96FC93EE931A97E989FA89E20D52
:100BD000F31D1D96FC93EE931C97EB89FC89E20DA7
:100BE000F31D1F96FC93EE931E97ED89FE89E20D8F
:100BF000F31D5196FC93EE9350970E9478822D81BD
:100C00003E812F5F3F4F3E832D838B819C810496D5
:100C10009C838B83A4E0B0E02A0E3B1EEDB7FEB7A9
:100C200072960FB6F894FEBF0FBEEDBF2D813E81C8
:100C30008F859889281739070CF455CF66960FB61B
:100C4000F894DEBF0FBECDBFCF91DF911F910F9102
:100C5000FF90EF90DF90CF90BF90AF909F908F90DC
:100C60007F906F905F904F903F902F90089580916C
:100C7000A0120895609311047093120480931304DA
:100C8000909314040895609111047091120480915E
:100C9000130490911404089590939D1280939C12D4
:100CA00070939F1260939E12089590939A1280936E
:100CB000991208958091991290919A1208958091B5
:100CC0009E1290919F1208959093080480930704B8
:100CD000089580910704909108040895FC0186818D
:100CE00097810895FC01808191810895FC01118212
:100CF00010820895FC01828193810895FC01138282
:100D000012820895DC0180919B128823D9F01496F9
:100D10008D919C911597880F991F880F991F1C968C
:100D2000ED91FC911D97E80FF91F40835183628379
:100D3000738314968D919C911597019615969C93AB
:100D40008E9314970895FC01848195810895FC0188
:100D5000158214820895660F771F660F771FDC01D6
:100D60001C96ED91FC911D97E60FF71F20813181B4
:100D700042815381B901CA01089560930D047093B3
:100D80000E0480930F049093100408956093090457
:100D900070930A0480930B0490930C0408956F924F
:100DA0007F928F929F92AF92BF92CF92DF92EF92FB
:100DB000FF920F931F93DF93CF9300D000D0CDB756
:100DC000DEB76C014A015B01FC0160847184F301B0
:100DD000E080F18002811381CB01BA01A801970163
:100DE0000E94CBCF8823BCF0F601808191810197CE
:100DF000880F991F880F991F680E791EF301E080F4
:100E0000F18002811381C501B401A80197010E94FC
:100E10001AD118162CF4E982FA820B831C8304C0C1
:100E200089829A82AB82BC82F60160857185428597
:100E3000538524853585A2E1AA2EB12CAC0CBD1CAE
:100E4000D60156968681978101E010E07E010894D4
:100E5000E11CF11CEEE0F0E0CE0EDF1E4D010E9421
:100E60003B850F900F900F900F90CF91DF911F91C6
:100E70000F91FF90EF90DF90CF90BF90AF909F9039
:100E80008F907F906F9008958F929F92AF92BF92B4
:100E9000CF92DF92EF92FF920F931F93CF93DF9346
:100EA0006C01DC0116968D919C9117970197880F24
:100EB000991F880F991F1896ED91FC911997E80FCB
:100EC000F91F608171818281938120E030E04AE7DF
:100ED00054E40E94CFCF20E030E040E85FE30E947E
:100EE00066CF4B015C01C0E0D0E0BE01882777FDF2
:100EF0008095982F0E946AD0A50194010E941ED16E
:100F0000AB01BC01C6010E94CF86F601E688F788D6
:100F1000008D118DC801B70120E030E040E050E0C5
:100F20000E941AD1181624F017FB109517F9109586
:100F3000C801B7012091090430910A0440910B04C3
:100F400050910C040E941AD1181614F480E006C0C7
:100F50002196F3E0C83EDF0741F681E0DF91CF91B3
:100F60001F910F91FF90EF90DF90CF90BF90AF90C7
:100F70009F908F9008958F929F92AF92BF92CF9241
:100F8000DF92EF92FF920F931F93CF93DF936C0149
:100F9000DC0116968D919C9117970197880F991FE8
:100FA000880F991F1896ED91FC911997E80FF91F7A
:100FB000608171818281938120E030E04AE754E4CE
:100FC0000E94CFCF20E030E040E85FE30E9466CF90
:100FD0004B015C01C0E0D0E0BE01882777FD809521
:100FE000982F0E946AD0A50194010E941ED1AB01E6
:100FF000BC01C6010E94CF86F601E288F38804890D
:101000001589C801B70120E030E040E050E00E94BF
:101010001AD1181624F017FB109517F91095C8016E
:10102000B70120910D0430910E0440910F045091AE
:1010300010040E941AD1181614F480E006C02196FC
:10104000F3E0C83EDF0741F681E0DF91CF911F91C9
:101050000F91FF90EF90DF90CF90BF90AF909F9057
:101060008F900895EF92FF920F931F93CF93DF938A
:10107000EC017A018B010E943786882339F0CE017A
:101080004A96B801A7010E94C39009C0CE01B801D9
:10109000A7010E94CF866E897F89888D998DDF9107
:1010A000CF911F910F91FF90EF900895EF92FF92D3
:1010B0000F931F93CF93DF93EC017A018B010E9472
:1010C0003786882339F0CE014A96B801A7010E94DD
:1010D000DB9009C0CE01B801A7010E94CF866A89C2
:1010E0007B898C899D89DF91CF911F910F91FF9012
:1010F000EF900895EF92FF920F931F93CF93DF939A
:10110000EC017A018B010E943786882339F0CE01E9
:101110004A96B801A7010E94F39009C0CE01B80118
:10112000A7010E94CF866E857F8588899989DF9186
:10113000CF911F910F91FF90EF9008950F931F9300
:10114000CF93DF938C01EB010E943786882331F027
:10115000C8014A96BE010E9477900FC0CC0FDD1FD8
:10116000CC0FDD1FD8011A96ED91FC911B97EC0F67
:10117000FD1F6081718182819381DF91CF911F91E9
:101180000F910895CF93DF93EC018091A0128823F3
:1011900029F0CE014A960E94C29112C080919B1202
:1011A000882399F08A819B81880F991F880F991F46
:1011B000EA85FB85E80FF91F4083518362837383BF
:1011C0008A819B8101969B838A83DF91CF910895C9
:1011D000CF93DF93EC0180919B12882371F0888577
:1011E00099850E945A0C8A859B850E945A0C8C8591
:1011F0009D850E945A0C10929B12CE014A960E9425
:101200000B91DF91CF9108950F931F93CF93DF93AD
:101210008C01EB010E943786882331F0C8014A9681
:10122000BE010E946A900FC0CC0FDD1FCC0FDD1FE6
:10123000D8011896ED91FC911997EC0FFD1F608174
:10124000718182819381DF91CF911F910F910895D8
:10125000CF93DF93EC018091A012882329F0CE0177
:101260004A960E94229212C080919B12882399F084
:1012700088819981880F991F880F991FE885F985C2
:10128000E80FF91F408351836283738388819981BA
:10129000019699838883DF91CF9108950F931F93CF
:1012A000CF93DF93EC018B0177FD37C00E94E88874
:1012B0001F830E830E943786882351F50230110563
:1012C00064F1C801880F991F880F991F0E94B00B05
:1012D000888799878E819F81880F991F880F991F12
:1012E0000E94B00B8A879B878E819F81880F991FF0
:1012F000880F991F0E94B00B8C879D8719821882D6
:101300001B821A821D821C8281E080939B1205C081
:10131000CE014A96B8010E948292DF91CF911F912F
:101320000F9108950F931F938C010E94E888C801C4
:101330004A960E9421911F910F9108950F931F9338
:101340008C014A960E945990F801118610861386E6
:1013500012861586148611821082138212821582DB
:101360001482178216821F910F9108950F931F9375
:10137000FC01408351836283738304831583268336
:1013800037831F910F910895AC01CB0116161706F4
:1013900014F481E090E097FF02C080E090E0FC014F
:1013A000EE0FFF1FEE0FFF1FE40FF51F20813181AD
:1013B00042815381B901CA010895FC012081318124
:1013C00042815381B901CA0108950F931F938C0183
:1013D000882777FD8095982F0E946AD0F801608356
:1013E0007183828393831F910F910895FC0124815F
:1013F000358146815781B901CA0108950F931F9322
:101400008C01882777FD8095982F0E946AD0F8017B
:1014100064837583868397831F910F9108958F92BC
:101420009F92AF92BF92CF92DF92EF92FF920F9373
:101430001F93DF93CF93CDB7DEB760970FB6F894C5
:10144000DEBF0FBECDBF4B01AA2797FDA095BA2FD7
:10145000BC01CD010E946AD07B018C01F401208186
:101460003181428153810E941ED15B016C01C80110
:10147000B701F40124813581468157810E941ED134
:101480008B019C017E010894E11CF11CC701B6018F
:10149000A5010E94B689DE011996F70188E0019046
:1014A0000D928150E1F729853A854B855C856D85E4
:1014B0007E858F85988960960FB6F894DEBF0FBE43
:1014C000CDBFCF91DF911F910F91FF90EF90DF90F3
:1014D000CF90BF90AF909F908F900895AF92BF92A2
:1014E000CF92DF92EF92FF920F931F93DF93CF93F0
:1014F000CDB7DEB760970FB6F894DEBF0FBECDBF95
:101500008C015B01FC016081718182819381F50115
:1015100020813181428153810E9467CF6B017C0120
:10152000F8016481758186819781F5012481358177
:10153000468157810E9467CF8B019C015E01089410
:10154000A11CB11CC501B701A6010E94B689DE012C
:101550001996F50188E001900D928150E1F72985F7
:101560003A854B855C856D857E858F8598896096EB
:101570000FB6F894DEBF0FBECDBFCF91DF911F91A4
:101580000F91FF90EF90DF90CF90BF90AF900895B4
:10159000EF92FF920F931F93DF93CF93CDB7DEB7F8
:1015A00060970FB6F894DEBF0FBECDBFFC0140813F
:1015B0005181628173817058048115812681378140
:1015C00030587E010894E11CF11CC7010E94B689C5
:1015D000DE011996F70188E001900D928150E1F744
:1015E00029853A854B855C856D857E858F859889B3
:1015F00060960FB6F894DEBF0FBECDBFCF91DF91DE
:101600001F910F91FF90EF900895FC017383628307
:101610000895FC01758364836115710521F0CB0188
:10162000BF010E94058B0895AF92BF92CF92DF92C7
:10163000EF92FF920F931F93DF93CF93CDB7DEB757
:10164000C056D0400FB6F894DEBF0FBECDBF8C01A0
:10165000F6E0CF2ED12CC80ED91EC6010E94C88A32
:10166000DE01A75ABF4F2C93FE01E65AFF4F30838D
:10167000FE01E55AFF4F4083FE01E45AFF4F5083BD
:10168000FE01E35AFF4F6083FE01E25AFF4F708371
:10169000FE01E15AFF4F8083FE01E05AFF4F908325
:1016A0009E012F5F3F4FFD0188E00190D9010D920F
:1016B0009D018150D1F7EEE0EE2EF12CE00EF11EEF
:1016C00083E090E0B7010E940F8ADE01A75ABF4F66
:1016D0002C93FE01E65AFF4F3083FE01E55AFF4F7F
:1016E0004083FE01E45AFF4F5083FE01E35AFF4F4F
:1016F0006083FE01E25AFF4F7083FE01E15AFF4F03
:101700008083FE01E05AFF4F90839E01275F3F4F89
:10171000FD0188E00190D9010D929D018150D1F722
:10172000CE010196BE01675F7F4F0E946E8ADE0187
:10173000A75ABF4F2C93FE01E65AFF4F3083FE019C
:10174000E55AFF4F4083FE01E45AFF4F5083FE01EC
:10175000E35AFF4F6083FE01E25AFF4F7083FE01A0
:10176000E15AFF4F8083FE01E05AFF4F90839E01B4
:101770002F5E3F4FFD0188E00190D9010D929D0140
:101780008150D1F776E1A72EB12CA00EB11E8DEFBE
:101790009FEFB5010E940F8ADE01A75ABF4F2C931D
:1017A000FE01E65AFF4F3083FE01E55AFF4F4083AA
:1017B000FE01E45AFF4F5083FE01E35AFF4F60835E
:1017C000FE01E25AFF4F7083FE01E15AFF4F808312
:1017D000FE01E05AFF4F90839E01275E3F4FFD01BF
:1017E00088E00190D9010D929D018150D1F7CE0181
:1017F0004196BE01675E7F4F0E946E8ADE01A75A46
:10180000BF4F2C93FE01E65AFF4F3083FE01E55A8D
:10181000FF4F4083FE01E45AFF4F5083FE01E35A1D
:10182000FF4F6083FE01E25AFF4F7083FE01E15AD1
:10183000FF4F8083FE01E05AFF4F90839E012F5D92
:101840003F4FFD0188E00190D9010D929D0181502B
:10185000D1F7B801625E7F4FCE0181960E946E8AF9
:10186000F80126A337A340A751A762A773A784A7AF
:1018700095A783E090E0B6010E940F8ADE01A75A87
:10188000BF4F2C93FE01E65AFF4F3083FE01E55A0D
:10189000FF4F4083FE01E45AFF4F5083FE01E35A9D
:1018A000FF4F6083FE01E25AFF4F7083FE01E15A51
:1018B000FF4F8083FE01E05AFF4F90839E01275D1A
:1018C0003F4FFD0188E00190D9010D929D018150AB
:1018D000D1F78AEF9FEFB7010E940F8ADE01A75A66
:1018E000BF4F2C93FE01E65AFF4F3083FE01E55AAD
:1018F000FF4F4083FE01E45AFF4F5083FE01E35A3D
:10190000FF4F6083FE01E25AFF4F7083FE01E15AF0
:10191000FF4F8083FE01E05AFF4F90839E012F5CB2
:101920003F4FFD0188E00190D9010D929D0181504A
:10193000D1F7CE018996BE016F5C7F4F0E946E8AFF
:10194000DE01A75ABF4F2C93FE01E65AFF4F3083AA
:10195000FE01E55AFF4F4083FE01E45AFF4F5083DA
:10196000FE01E35AFF4F6083FE01E25AFF4F70838E
:10197000FE01E15AFF4F8083FE01E05AFF4F908342
:101980009E01275C3F4FFD0188E00190D9010D9237
:101990009D018150D1F783E090E0B5010E940F8A4C
:1019A000DE01A75ABF4F2C93FE01E65AFF4F30834A
:1019B000FE01E55AFF4F4083FE01E45AFF4F50837A
:1019C000FE01E35AFF4F6083FE01E25AFF4F70832E
:1019D000FE01E15AFF4F8083FE01E05AFF4F9083E2
:1019E0009E012F5B3F4FFD0188E00190D9010D92D0
:1019F0009D018150D1F7CE01C996BE016F5B7F4F2B
:101A00000E946E8AF80126A737A740AB51AB62ABA4
:101A100073AB84AB95AB8DEF9FEFB6010E940F8A3D
:101A2000DE01A75ABF4F2C93FE01E65AFF4F3083C9
:101A3000FE01E55AFF4F4083FE01E45AFF4F5083F9
:101A4000FE01E35AFF4F6083FE01E25AFF4F7083AD
:101A5000FE01E15AFF4F8083FE01E05AFF4F908361
:101A60009E01275B3F4FFD0188E00190D9010D9257
:101A70009D018150D1F783E090E0B7010E940F8A69
:101A8000DE01A75ABF4F2C93FE01E65AFF4F308369
:101A9000FE01E55AFF4F4083FE01E45AFF4F508399
:101AA000FE01E35AFF4F6083FE01E25AFF4F70834D
:101AB000FE01E15AFF4F8083FE01E05AFF4F908301
:101AC0009E012F5A3F4FFD0188E00190D9010D92F0
:101AD0009D018150D1F7CE01875B9F4FBE016F5AA8
:101AE0007F4F0E946E8AF80126AB37AB40AF51AFF3
:101AF00062AF73AF84AF95AFD801DE96369688E0BB
:101B000001900D928150E1F7C05ADF4F0FB6F89463
:101B1000DEBF0FBECDBFCF91DF911F910F91FF9020
:101B2000EF90DF90CF90BF90AF900895EF92FF922B
:101B30000F931F93CF93DF93EC018A018091A11241
:101B40009091A2129983888301969093A212809318
:101B5000A112FE01369680E090E0AF017B01E80E15
:101B6000F91E28E0D7010D907D01DA010D92AD013B
:101B70002150C1F7089638968032910571F71B8283
:101B80001A82CE01B8010E94098BCE010E94148BEB
:101B9000DF91CF911F910F91FF90EF9008952F92B9
:101BA0003F924F925F926F927F928F929F92AF92ED
:101BB000BF92CF92DF92EF92FF920F931F93DF932A
:101BC000CF9300D00F92CDB7DEB79B838A835A01A3
:101BD0006B0181E0922F982799838A819B81CE9611
:101BE000698170E00E94C489A80197010E9466CFB4
:101BF0007B018C018A819B81C696698170E00E947D
:101C0000C4899B01AC01C601B5010E941ED19B0194
